:020000040800F2
:1000000000060020E1010008190E00081D0E00087E
:10001000750E00081D0E0008490E0008E3010008D7
:10002000E3010008E3010008E3010008452100089E
:10003000E3010008E3010008E3010008E301000810
:10004000E3010008E3010008E3010008E301000800
:10005000E3010008E30100082532000851320008DE
:100060007D320008A9320008D5320008E3010008FB
:10007000E3010008E3010008E3010008E3010008D0
:10008000E3010008E3010008E3010008E3010008C0
:10009000E3010008E3010008E30100080133000860
:1000A000E3010008E3010008E3010008E3010008A0
:1000B00099300008E3010008E3010008E3010008AB
:1000C000E3010008E3010008E3010008E301000880
:1000D000E3010008E3010008E3010008E301000870
:1000E00069330008E3010008E3010008E3010008A8
:1000F000E3010008E3010008E3010008E301000850
:10010000E3010008E3010008E3010008E30100083F
:10011000E3010008E3010008E3010008E30100082F
:10012000E3010008E3010008E3010008E30100081F
:10013000E3010008E3010008E3010008E30100080F
:10014000E3010008E3010008E30100088928000832
:10015000E3010008E3010008E3010008E3010008EF
:10016000E3010008E3010008E3010008E3010008DF
:10017000E3010008E3010008E3010008E3010008CF
:10018000E3010008E3010008E3010008E3010008BF
:10019000E3010008E3010008E3010008E3010008AF
:1001A000E3010008E3010008E3010008E30100089F
:1001B000E3010008E3010008E3010008E30100088F
:1001C000E3010008E3010008E3010008E30100087F
:1001D000E3010008E3010008E3010008E30100086F
:1001E00002E000F000F8FEE772B6394880F30888B4
:1001F000384880F3098838484EF60851CEF200019D
:10020000086040F20000CCF200004EF63471CEF2ED
:1002100000010860BFF34F8FBFF36F8F40F2000003
:10022000C0F2F0004EF68851CEF200010860BFF334
:100230004F8FBFF36F8F4FF00000E1EE100A4EF6C4
:100240003C71CEF200010860062080F31488BFF3F1
:100250006F8F01F0D5FF02F07BFE4FF055301F4944
:100260001B4A91423CBF41F8040BFAE71C49194A6A
:1002700091423CBF41F8040BFAE71A491A4A1B4B5A
:100280009A423EBF51F8040B42F8040BF8E70020F5
:100290001749184A91423CBF41F8040BFAE701F0B4
:1002A000B3FF02F0B1FE144C144DAC4203DA54F823
:1002B000041B8847F9E700F041F8114C114DAC429E
:1002C00003DA54F8041B8847F9E701F09BBF0000EC
:1002D000000600200022002000000008000000208E
:1002E0000006002078370008002200202822002085
:1002F00028220020942D0020E0010008E0010008E1
:10030000E0010008E00100082DE9F04F2DED108A12
:10031000C1F80CD0C3689D46BDEC108ABDE8F08FD3
:10032000002383F311882846A047002001F036FB04
:10033000FEE701F0B7FA00DFFEE700001A4B7A2271
:1003400070B500241A700F225C709C70DC701C71F8
:100350005C719C71DC711C725C729A72DC7201F0CF
:10036000C3FE064601F0E8FE054650B90F4B9E421B
:1003700017D001339E4241F2883412BF0546002453
:100380000125002001F0BAFE0DB100F059F800F08F
:1003900017FD00F09FFB204600F0B0F800F050F889
:1003A000F9E70446EDE700BF28220020010007B06E
:1003B00008B500F061FBA0F120035842584108BD88
:1003C00007B5054B02211B88ADF8043001A800F0E9
:1003D00071FB03B05DF804FB4C34000810B520231A
:1003E00083F311881248C3680BB101F073FB00233B
:1003F000104A0F484FF47A7101F01AFB002383F37F
:1004000011880D4C236813B12368013B2360636896
:1004100013B16368013B6360084B1B7833B96368B1
:1004200023B9022000F03AFC3223636010BD00BF04
:1004300034220020DD030008502300204822002041
:1004400010B5254B254953F8042F013200D110BDBA
:100450008B42F8D1224C234B22689A423AD9224B44
:100460009B6803F1006303F580339A4232D2002087
:1004700000F04AFB1D4B0220187000F007FC1C4BDB
:100480001A6C00221A64196E1A66196E596C5A6435
:10049000596E5A665A6E5A6942F080025A615A6918
:1004A00022F080025A615A691A6942F000521A61B8
:1004B0001A6922F000521A611B6972B60D4A0E4B7E
:1004C00013601B682268202181F311889D4683F305
:1004D0000888104710BD00BFFCFF00081C00010881
:1004E00004000108FFFF0008282200204822002005
:1004F0000038024008ED00E0000001082DE9F04F4F
:1005000099B0B94D00902022FF2110A8AC6800F0EE
:10051000F9FBB64A01951378A3B9B5480121C36028
:100520001170202383F31188C3680BB101F0D2FA54
:100530000023B04AAE484FF47A7101F079FA0023F3
:1005400083F31188009BAC4A03B11360AB4B009D51
:10055000029300261E705660B2463746B14601200F
:1005600000F094FB002D00F02582A34B1B68002BAC
:1005700040F0208219B0BDE8F08F0220FFF718FF8D
:10058000002840F01082009B002E08BF1D469C4BA7
:1005900002211B88ADF82C300BA800F08BFADEE7A7
:1005A0004FF47A7000F068FAB0F10008EBDB02203B
:1005B000FFF7FEFE0028E6D008F1FF38B8F1040F7F
:1005C00000F2F381DFE808F0031E2124270018A8B9
:1005D000052340F8343D042100F06CFA012303FAAE
:1005E00008F848EA0A0A5FFA8AFA4FF0000900F0B0
:1005F000DDFB27B10AF00B030B2B08BF0025FFF72B
:10060000DFFEACE704217848E6E704217D48E3E714
:1006100004217D48E0E74FF01C09484600F076FAD7
:1006200009F104090B9004210BA800F043FAB9F179
:100630002C0FF2D1D2E7002FA5D00AF00B030B2B21
:10064000A1D10220FFF7B4FE804600289BD00120F4
:100650006A4E00F059FA0220307000F017FB0027B4
:100660005FFA87FB584600F05FFA054688B15846A6
:1006700000F06AFA01370028F2D146460025634BA4
:1006800002211B88ADF82C300BA800F013FA474666
:1006900065E701230220337000F0EEFA2C46019B3F
:1006A0009B689C4206D2204600F030FA0130E4D12B
:1006B0000434F4E7029B00241C704F4B46465C60F8
:1006C0004746254693E7002F3FF45DAF0AF00B0342
:1006D0000B2B7FF458AF029B0220187000F0D6FA63
:1006E000322000F0C9F9B0F1000BFFF64CAF1BF05F
:1006F00003087FF448AF019B996804EB0B028A4220
:100700003FF641AFBBF5807F3FF63DAF404A0392D5
:10071000D8450FDA4FF47A7000F0AEF904900499DE
:100720000029FFF630AF039A049908F8021008F187
:100730000108ECE7C820FFF73BFE804600283FF4A5
:1007400022AF1F2C11D8C4F120075F4528BF5F4698
:1007500010AB24F003003A462D49184400F0A8FAE3
:100760003A46FF212A4800F0CDFA4FEAAB03DAB24D
:1007700027490393204600F0CDFA074600283FF4AE
:100780007EAF039B04EB830431E70220FFF710FEEA
:1007900000283FF4F8AE00F0FDF900283FF4F3AE76
:1007A0004FF000084346019A9268904532D2B8F162
:1007B0001F0F12D8109A01320FD028F0030218A987
:1007C0000A4452F8202C0B92184604220BA900F080
:1007D00065FB08F104080346E5E74046039300F093
:1007E00095F9039B0B90EFE7282200204C23002073
:1007F00034220020DD03000850230020482200207E
:100800004E3400082C2200203022002050340008F2
:100810004C22002018A8042140F84C3D00F04AF971
:10082000E5E618A8002340F8343D642100F038F9CB
:1008300000287FF4A8AE0220FFF7BAFD00283FF49D
:10084000A2AE0B9800F092F918AB43F8480D0421C2
:100850001846E3E718A8002340F8343D642100F06F
:100860001FF900287FF48FAE0220FFF7A1FD0028BA
:100870003FF489AE0B9800F087F918AB43F8440DAC
:10088000E5E70220FFF794FD00283FF47CAE00F07E
:1008900091F918AB43F8400DD9E70220FFF788FD26
:1008A00000283FF470AE0BA9142000F089F98046AF
:1008B00018A8042140F83C8D00F0FCF841460BA834
:1008C000ACE7322000F0D8F8B0F10008FFF65BAEDC
:1008D00018F0030F7FF457AE019A926808EB0903F2
:1008E00093423FF650AE0220FFF762FD00283FF42E
:1008F0004AAE28F00308C844C1453FF478AE4846E4
:1009000000F004F904210A900AA800F0D3F809F1D4
:100910000409F1E74FF47A70FFF74AFD00283FF42D
:1009200032AE00F037F9002842D0109B01330BD0D3
:10093000082210A9002000F0EDF9002838D020226C
:10094000FF2110A800F0DEF9FFF73AFD364801F06C
:100950002BF80FE6002F3FF416AE0AF00B030B2B1B
:100960007FF411AE18A8002340F8343D642100F054
:1009700097F8804600287FF406AE0220FFF718FDA6
:1009800000283FF400AE0390FFF71AFD41F28830D3
:1009900001F00AF80B9800F03DFA00F007FA039B0B
:1009A00045461F46DBE5074621E64FF00009EAE52C
:1009B000B84664E6002000F05FF80490049B002B2A
:1009C000FFF6D0AD012000F057F9049B213B122B1C
:1009D0003FF6C5AD01A252F823F000BF7B05000829
:1009E000A1050008370600085F0500085F0500083C
:1009F0005F050008C7060008C30800088B07000849
:100A00002308000855080008830800085F0500084F
:100A10009B0800085F05000815090008EF0500089D
:100A20005F05000855090008A086010070B50F4B4E
:100A30000C4619780131C9B2012906460FD80C4875
:100A400003681D6A4FF47A73534331462246A84720
:100A5000844204D1074B00221A70012070BD4FF46C
:100A6000FA7000F0A1FF002070BD00BF002200203E
:100A7000C02500208423002007B502AB002203F824
:100A8000012D012102461846FFF7D0FF20B19DF845
:100A9000070003B05DF804FB4FF0FF30F9E70000FA
:100AA0000A4608B50421FFF7C1FF80F00100C0B27B
:100AB000404208BD30B4054C2368DD69044B0A464A
:100AC000AC460146204630BC604700BFC025002030
:100AD000A086010070B501F00BFA094C094E208088
:100AE000002530682388834208D901F0FBF9336878
:100AF00005440133B5F5803F3360F2D370BD00BFCC
:100B0000862300205823002001F0A0BA00F10060E5
:100B100000F580300068704700F10060920000F539
:100B2000803001F02BBA0000054B1A68054B1B887A
:100B30009B1A834202D9104401F0D4B900207047B7
:100B4000582300208623002038B5074D0446286826
:100B5000204401F0CFF928B928682044BDE8384086
:100B600001F0E0B938BD00BF5823002010F00303A6
:100B700008D1B0F5047F05D200F10050A0F508407F
:100B80000068704700207047014BC058704700BF95
:100B9000107AFF1F064991F8243033B10023082250
:100BA000086A81F82430FFF7B7BF0120704700BF03
:100BB0005C230020014B1868704700BF002004E050
:100BC00070B52A4B1C68C4F30B03240C63B140F2CC
:100BD0001342934231D040F2194293422FD040F257
:100BE000214293422DD10323214A0C2505FB0323E7
:100BF0005D6893F9082042F201039C4224D0B4F5C9
:100C0000805F23D041F201039C4221D041F20303D3
:100C10009C421FD041F207039C4208BF3122441E70
:100C20000C44013D0B46A3421ED215F9016F581C1E
:100C300096B1034600F8016CF5E70123D4E70223DF
:100C4000D2E73F220B4DD6E73322E3E74122E1E72B
:100C50005A22E4E75922E2E72C2584421D7001D98B
:100C6000981C5A70401A70BD1846FBE7002004E03B
:100C70006034000854340008022802BF024B4FF4CD
:100C800000129A61704700BF00040240022802BFB0
:100C9000014B20229A61704700040240022801BFE4
:100CA000024A536983F020035361704700040240F5
:100CB00010B50023934203D0CC5CC4540133F9E750
:100CC00010BD000030B5441E14F9010F0B4660B191
:100CD00093F90050854201F1010106D11AB993F947
:100CE0000020801A30BD013AEEE7002AF7D1104605
:100CF00030BD000002460346981A13F9011B002973
:100D0000FAD1704702440346934202D003F8011B14
:100D1000FAE770472DE9F047234C94F82430054654
:100D20008846174683BB2E46DFF87C90C7B394F8FD
:100D300024302BB92022FF2148462662FFF7E2FF2C
:100D400094F82400C0F10805BD4228BF3D465FFA73
:100D500085FAAD0041462A4604EB8000FFF7A8FF64
:100D600094F82430A7EB0A079A445FFA8AFABAF19A
:100D7000080F2E44A844FFB284F824A0D6D1FFF770
:100D800009FF0028D2D108E0266A06EB8306B042AC
:100D9000CAD0FFF7FFFE0028C5D10020BDE8F087CC
:100DA0000120BDE8F08700BF5C230020024B1A78C9
:100DB000024B1A70704700BF8423002000220020DD
:100DC00038B5104D104C284600F004F9214628464D
:100DD00000F02CF924680D48626DD2F8043843F015
:100DE0000203C2F8043800F0DFFD0949204600F094
:100DF00029FA626DD2F8043823F00203C2F80438ED
:100E000038BD00BFC02500205435000840420F0007
:100E10007C35000870470000FEE7000000B59BB07D
:100E2000EFF3098168226846FFF742FFEFF305837D
:100E3000044B9A6BDA6A9A6A9A6A9A6A9A6A9A6A06
:100E40009B6AFEE700ED00E000B59BB0EFF309817F
:100E500068226846FFF72CFFEFF30583044B9A6B7B
:100E60009A6A9A6A9A6A9A6A9A6A9B6AFEE700BFC5
:100E700000ED00E000B59BB0EFF309816822684601
:100E8000FFF716FFEFF30583034B5A6B9A6A9A6AD2
:100E90009A6A9A6A9B6AFEE700ED00E030B5084D59
:100EA0000A4491420BD011F8013B09245840013CFF
:100EB000F7D040F300032B4083EA5000F7E730BD42
:100EC0002083B8ED002304491A465A50C818083345
:100ED000802B4260F9D17047882300200268436864
:100EE0001143016003B118477047000013B5446B0C
:100EF000D4F894341A681178042915D1217C022978
:100F000012D11979128901238B4013420CD101A906
:100F100004F14C0001F020FFD4F89444019B2179A6
:100F20000246206800F0DAF902B010BD143001F07A
:100F3000A3BE00004FF0FF33143001F09DBE00004F
:100F40004C3001F075BF00004FF0FF334C3001F022
:100F50006FBF0000143001F071BE00004FF0FF3190
:100F6000143001F06BBE00004C3001F041BF0000B6
:100F70004FF0FF324C3001F03BBF0000D0F894241A
:100F800038B5136819780429054601D0012038BD09
:100F9000017C0229FAD112795C8901209040044039
:100FA000F4D105F1140001F003FE02460028EDD053
:100FB000D5F894544FF480732868697900F07CF96F
:100FC000204638BD406BFFF7D9BF000000207047B6
:100FD000704700007FB5124B0360002343608360BD
:100FE000C360012502260F4B05740446029001934D
:100FF00000F18402294600964FF48073143001F00A
:10100000B3FD094B0193029400964FF4807304F5ED
:101010002372294604F14C0001F07AFE04B070BD41
:10102000B0340008C50F0008ED0E00080B68202240
:1010300082F311880A7903EB820290614A790932BE
:1010400043F822008A7912B103EB820398610223EC
:101050000374C0F89414002383F3118870470000D0
:1010600038B5037F044613B190F85430ABB9201D56
:1010700001250221FFF732FF04F1140025776FF0FC
:10108000010100F0B9FC84F8545004F14C006FF0F9
:101090000101BDE8384000F0AFBC38BD10B50121FA
:1010A00004460430FFF71AFF0023237784F85430F6
:1010B00010BD000038B504460025143001F06CFD69
:1010C00004F14C00257701F03BFE201D84F85450BC
:1010D0000121FFF703FF2046BDE83840FFF74EBF70
:1010E00090F8443003F06003202B19D190F845208C
:1010F000212A0AD0222A4FF000030ED0202A0FD135
:10110000084A82630722C26304E0064B8363072315
:10111000C36300230364012070478363C363F9E75B
:101120000020704701220020D0F8943437B51A68A7
:101130001178042904461AD1017C022917D11979A2
:10114000128901238B40134211D100F14C0528462E
:1011500001F0B6FE58B101A9284601F0FDFDD4F812
:101160009444019B21790246206800F0B7F803B04F
:1011700030BD000000EB8103F7B59C6905460E46C3
:10118000F4B1202383F3118805EB8607201D082185
:10119000FFF7A4FEFB685B691B684C3413B1204663
:1011A00001F0E8FD01A9204601F0D6FD024648B154
:1011B000019B3146284600F091F8002383F3118803
:1011C00003B0F0BDFB685A691268002AF5D01B8A8B
:1011D000013B1340F1D105F14402EAE7093138B58A
:1011E00050F82140DCB1202383F31188D4F89424F3
:1011F0001368527903EB8203DB689B695D6845B134
:1012000004216018FFF76AFE294604F1140001F07A
:10121000D9FC2046FFF7B2FE002383F3118838BDC6
:101220007047000001F082B801230370002343607F
:10123000C36183620362C3624362036303814381C8
:101240007047000038B50446202383F31188002539
:101250004160C56005614561856101F077F8022351
:10126000237085F3118838BD70B500EB8103054606
:101270005069DA600E46144618B110220021FFF7BB
:1012800041FDA06918B110220021FFF73BFD314656
:101290002846BDE8704001F023B90000028902F041
:1012A00001020281428902F00102428100220261B0
:1012B0004261826101F0A8B9F0B400EB8104478972
:1012C000E4680125A4698D403D43458123600023E6
:1012D000A2606360F0BC01F0C3B90000F0B400EBA1
:1012E00081040789E468012564698D403D430581D7
:1012F00023600023A2606360F0BC01F03DBA0000EF
:1013000070B50223002504460370A0F84C5080F805
:101310004E5080F84F5005814581C560056145619B
:10132000856180F8345001F077F863681B6823B159
:1013300029462046BDE87040184770BD037880F804
:1013400050300523037043681B6810B504460BB189
:101350000421984700232381638110BD436890F8DE
:1013600050201B6802700BB1052118477047000020
:1013700090F8343070B5044613B1002380F834304F
:1013800004F14402204601F061F963689B6863BB85
:1013900094F8445015F0600615D194F8453005F0E6
:1013A0007F0545EA032540F202339D4200F00E819D
:1013B0005BD8022D00F0DC803FD8002D00F0878044
:1013C000012D00F0CF800021204601F099FB002183
:1013D000204601F08BFB63681B6813B10621204691
:1013E0009847062384F8343070BD2046984700287B
:1013F000CED094F84B2094F84A3043EA0223E26BB3
:10140000934238BFE36394F94430E56B002B4FF00F
:10141000200380F2FD80002D00F0EC80092284F88A
:10142000342083F311880021E36BA26B2046FFF781
:1014300055FF002383F3118870BDB5F5817F00F05F
:10144000B180B5F5407F49D0B5F5807FBBD194F828
:101450004630012BB7D1B4F84C3023F00203A4F886
:101460004C30A663E6632664C3E740F201639D4205
:101470001ED8B5F5C06F3BD2B5F5A06FA3D1B4F8B7
:101480004430B3F5A06F0ED194F8463084F84E3056
:10149000204601F019F863681B6813B1012120464A
:1014A0009847032323700023A363E3632364A0E727
:1014B000B5F5106F32D040F602439D4252D0B5F5DB
:1014C000006F80D104F14F03A363012324E004F1F2
:1014D0004C03A3630223E36325648AE794F8463050
:1014E000012B7FF470AFB4F84C3043F00203B6E741
:1014F00094F84920616894F848304D6894F8471092
:1015000043EA0223204694F84620A84700283FF4E7
:101510005AAF4368A3630368E363A4E72378042B0B
:1015200010D1202383F311882046FFF7B7FE86F3FE
:101530001188636884F84F601B68032121700BB128
:101540002046984794F84630002BACD084F84F30B2
:101550000423237063681B68002BA4D0022120465B
:101560009847A0E7374BA3630223E36300239DE77B
:1015700094F8481011F0800F204601F00F010ED0B2
:1015800001F056F8012806D002287FF41CAF2E4B3C
:10159000A363E06367E72D4BA363E56363E701F0B3
:1015A00039F8EFE794F84630002B7FF40CAF94F84D
:1015B000483013F00F013FF476AF1A06204602D5EB
:1015C00001F0B2FA6FE701F0A5FA6CE794F8463043
:1015D000002B7FF4F8AE94F8483013F00F013FF47D
:1015E00062AF1B06204602D501F08AFA5BE701F0E4
:1015F0007DFA58E7142284F8342083F311882B46AF
:101600002A4629462046FFF757FE85F3118870BD0C
:101610005DB1152284F8342083F311880021E36B37
:10162000A26B2046FFF748FE03E70B2284F8342024
:1016300083F311882B462A4629462046FFF74EFEA3
:10164000E3E700BFE0340008D8340008DC340008C9
:1016500038B590F834300446152B29D8DFE803F06C
:101660003E28282828283E28280B293928282828D9
:10167000282828283E3E90F84B1090F84A20C36B4B
:1016800042EA01229A4214D9C268128AB3FBF2F5E7
:1016900002FB15356DB9202383F311882B462A46AA
:1016A0002946FFF71BFE85F311880A2384F834309E
:1016B00038BD142384F83430202383F311880023A9
:1016C0001A4619462046FFF7F7FD002383F31188D9
:1016D00038BD036C03B198470023E7E7002101F010
:1016E0000FFA0021204601F001FA63681B6813B16C
:1016F0000621204698470623D8E7000090F83420BA
:10170000152A38B5044622D80123934040F6416299
:1017100013421DD113F480150FD19B0217D50B2353
:1017200080F83430202383F311882B462A4629463B
:10173000FFF7D4FD85F3118838BDC3689B695B68EA
:101740002BB9036C03B19847002384F8343038BDBB
:10175000002101F0D5F90021204601F0C7F96368A6
:101760001B6813B10621204698470623EDE70000C9
:10177000024B00221B605B609A60704708240020C7
:10178000002303748268054B1B6899689142FBD261
:101790005A68036042601060586070470824002057
:1017A00008B5202383F31188037C032B05D0042B79
:1017B0000DD02BB983F3118808BD436900221A604C
:1017C0004FF0FF334361FFF7DBFF0023F2E790E8C0
:1017D0000C001A6002685360F2E7000000230374F3
:1017E0008268054B1B6899689142FBD85A68036070
:1017F000426010605860704708240020054B19694A
:101800000874186802681A60536018610123037431
:10181000FEF77ABD0824002030B54B1C87B0054682
:101820000A4C10D023690A4A01A800F001F92846A1
:10183000FFF7E4FF049B13B101A800F04BF9236903
:10184000586907B030BDFFF7D9FFF8E7082400203A
:10185000A117000838B50C4D41612B6981689A6861
:101860009142044603D8BDE83840FFF789BF1846C7
:10187000FFF7B4FF01232C61014623742046BDE825
:101880003840FEF741BD00BF08240020044B1A6811
:101890001B6990689B68984294BF002001207047A4
:1018A0000824002010B5084C236820691A682260BB
:1018B0005460012223611A74FFF790FF01462069EA
:1018C000BDE81040FEF720BD08240020FEE7000020
:1018D00010B50C4CFFF74CFF00F09CF880220A4931
:1018E000204600F021F8012344F8180C037400F09E
:1018F00039FC002383F3118862B60448BDE8104028
:1019000000F034B830240020E4340008EC3400083F
:1019100000F01AB9034B59685A68521A9042FBD822
:10192000704700BF001000E08260022202740022B3
:10193000427470478368A3F17C0243F80C2C02695F
:1019400043F83C2C426943F8382C074A43F81C2CD6
:10195000C26843F8102C022203F8082C002203F876
:10196000072CA3F1180070472103000810B52023AD
:1019700083F31188FFF7DEFF00210446FFF76AFFBB
:10198000002383F31188204610BD0000024B1B6921
:1019900058610F20FFF732BF08240020202383F373
:1019A0001188FFF7F3BF000008B50146202383F339
:1019B00011880820FFF730FF002383F3118808BD4A
:1019C00049B1064B42681B6918605A601360436056
:1019D0000420FFF721BF4FF0FF307047082400209C
:1019E0000368984206D01A68026050605961184630
:1019F000FFF7C6BE7047000038B504460D462068A4
:101A0000844200D138BD036823605C604561FFF704
:101A1000B7FEF4E7054B03F114025A619A614FF0E7
:101A2000FF32DA6100221A62704700BF08240020EA
:101A3000F8B5274F0361C2600D46044601F074FA01
:101A40003B46022D53F8142F294638BF02219A42F3
:101A50003E461D460AD138627C61BC610844226062
:101A60006260A160BDE8F84001F04CBAD7F820E010
:101A7000A0EB0E035F181FD300279068834217D88E
:101A8000376AAA421F44376201D0C01A9060736956
:101A90009A68914219D85A682360626014605C6049
:101AA000A1609868411A99604FF0FF33F361F8BD67
:101AB00097601B1A1268E0E793689F4203D20EEB0F
:101AC000070001F02DFA3946E1E7891A1B68DFE7C4
:101AD0000824002038B51B4B01685A6990421D4606
:101AE00003F114020CD04468216003680021934282
:101AF0005C60C16025D09A6881680A449A6038BDEC
:101B000059614A605B6900219342C16003D1BDE81D
:101B1000384001F0FFB99A6881680A449A602C6ADB
:101B200001F002FA6A699268001B824209D9111A0F
:101B3000012998BF821C286ABDE83840104401F092
:101B4000EFB938BD082400202DE9F84F204C0027BC
:101B5000656904F11406B84601F0E6F9236AA0EBC2
:101B6000030AAB6853451DD84FF02009236AAA68C1
:101B7000D5F80CB013442362AB68AAEB030A2B68B8
:101B8000B3425E606361EF6001D101F0C3F988F395
:101B900011882869D84789F311886569AB689A4527
:101BA000E4D2D9E76369B34210D020629A68A2EB0D
:101BB0000A029A60226AAB68821A9B1A022B2CBF17
:101BC000C0180230BDE8F84F01F0AAB9BDE8F88F9F
:101BD0000824002000207047FEE700007047000046
:101BE0004FF0FF3070470000022906D0032906D0CD
:101BF0000129064818BF0020704705487047032A8E
:101C00009ABF044800EBC20000207047D835000896
:101C10008C3500080822002070B59AB001AD064648
:101C200008462946144600F095F82846FFF762F862
:101C3000C0B2431C5B0086E8180023700323637066
:101C4000002302341946DAB2904204F1020401D8AA
:101C50001AB070BDEA5C04F8022C04F8011C0133D0
:101C6000F1E7000008B5202383F311880348FFF74C
:101C70005BFA002383F3118808BD00BFC025002054
:101C800010B50446052916D8DFE801F0161503162D
:101C9000161D202383F311880E4A0121FFF7E4FA71
:101CA00020460D4A0221FFF7DFFA0C48FFF702FA3F
:101CB000002383F3118810BD202383F31188074884
:101CC000FFF7CEF9F4E7202383F311880348FFF7E9
:101CD000E5F9EDE70C35000830350008C025002097
:101CE00038B50C4D0C4C0D492A4604F10800FFF79D
:101CF00093FF05F1CA0204F110000949FFF78CFFB8
:101D000005F5CA7204F118000649BDE83840FFF72E
:101D100083BF00BF882A0020082200205C3500080D
:101D2000663500087135000870B5044608460D4652
:101D3000FEF7E0FFC6B22046013403780BB918461F
:101D400070BD32462946FEF7BDFF0028F3D10120C1
:101D500070BD00002DE9F84F05460C46FEF7CAFF9E
:101D60002A49C6B22846FFF7DFFF08B10136F6B2AE
:101D700027492846FFF7D8FF08B11036F6B2632E80
:101D80000DD8DFF88890DFF888A0224FDFF88CB0FC
:101D9000DFF88C802E7846B92670BDE8F88F29468A
:101DA0002046BDE8F84F01F049BB252E29D1072276
:101DB00049462846FEF786FF40B9D8F80030236030
:101DC000D8F80430636007350834E3E70822514649
:101DD0002846FEF777FFA0B90F4BA21C13F8011F8E
:101DE00009095B45C95D02F8021C197801F00F0171
:101DF00002F10202C95D02F8031CEFD11834083564
:101E0000C8E7267001350134C4E700BFF835000883
:101E100071350008093600080F7AFF1F1B7AFF1F73
:101E200000360008BFF34F8F024AD368DB03FCD4AF
:101E3000704700BF003C024008B5094B1B7873B9DE
:101E4000FFF7F0FF074B1A69002ABFBF064A5A6026
:101E500002F188325A601A6822F480621A6008BD62
:101E6000E62C0020003C02402301674508B50B4BDF
:101E70001B7893B9FFF7D6FF094B1A6942F000426D
:101E80001A611A6842F480521A601A6822F4805269
:101E90001A601A6842F480621A6008BDE62C0020BD
:101EA000003C02400B2870B513D80B4A0B4C13783A
:101EB00063B90B4E4FF0006144F8231056F82350DD
:101EC00001330C2B2944F7D10123137054F820005F
:101ED00070BD002070BD00BF182D0020E82C002030
:101EE0001C360008014B53F8200070471C360008D0
:101EF0000C2070470B2810B5044601D9002010BDF6
:101F0000FFF7D0FF064B53F824301844C21A0BB920
:101F1000012010BD12680132F0D1043BF6E700BF8A
:101F20001C3600080B2810B5044621D8FFF77AFFAD
:101F3000FFF782FF0F4AF323D360C300DBB243F401
:101F4000007343F002031361136943F48033136198
:101F5000FFF768FFFFF7A6FF074B53F8241000F0C8
:101F6000DDF8FFF783FF2046BDE81040FFF7C2BF52
:101F7000002010BD003C02401C3600082DE9F8434B
:101F800012F00103154640D18218B2F1016F3CD224
:101F90002C4B1B6813F0010337D02B4CFFF74CFF81
:101FA000F323E360FFF73EFF40F20127032D01D941
:101FB000830713D0244C0F46401A40F20118EB1B44
:101FC0000B44012B00EB0706236924D823F00103FF
:101FD0002361FFF74BFF0120BDE8F883236923F459
:101FE0004073236123693B43236151F8046B06600E
:101FF000BFF34F8FFFF716FF03689E4208D0236997
:1020000023F001032361FFF731FF0020BDE8F883CF
:10201000043D0430CAE723F440732361236943EA93
:1020200008032361B94637F8023B3380BFF34F8F73
:10203000FFF7F8FE3688B9F80030B6B2B342BED02A
:10204000DDE700BF00380240003C0240084908B507
:102050000B7828B153B9FFF7EFFE01230B7008BDD1
:1020600023B1BDE808400870FFF700BF08BD00BFFE
:10207000E62C002010B50244064B0439D2B290423F
:1020800000D110BD441C00B253F8200041F8040FE9
:10209000E0B2F4E750280040104B30B51C6F240428
:1020A00007D41C6F44F400741C671C6F44F4004494
:1020B0001C670B4C236843F4807323600244094B74
:1020C0000439D2B2904200D130BD441C00B251F864
:1020D000045F43F82050E0B2F4E700BF003802404C
:1020E000007000405028004007B5012201A90020DF
:1020F000FFF7C0FF019803B05DF804FB13B5044679
:10210000FFF7F2FFA04206D002A9012241F8044DD8
:102110000020FFF7C1FF02B010BD000070470000B3
:10212000034B1B689B0042BF024B01221A70704791
:1021300074380240192D0020014B1878704700BFF9
:10214000192D0020EFF3098305494A6822F00102A6
:102150004A60683383F30988002383F3118870474A
:1021600030EF00E0202080F3118862B60B4B0C4A60
:10217000D96821F4E0610904090C0A430949DA60CD
:10218000CA6842F08072CA6007490A6842F00102D8
:102190000A601022DA7783F82200704700ED00E031
:1021A0000003FA05F0ED00E0001000E010B5202378
:1021B00083F311880E4B5B6813F4006314D0F1EEC7
:1021C000103AEFF30984683C4FF08073E361094BE8
:1021D000DB68236684F30988FFF758FB10B1064BD0
:1021E000A36110BD054BFBE783F3118810BD00BF51
:1021F00000ED00E030EF00E0330300083603000894
:1022000070470000FEE70000084A094B09498B426D
:1022100004D3094A0021934205D3704752F8040FB2
:1022200043F8040BF3E743F8041BF4E79C3700087A
:10223000942D0020942D0020942D0020836D70B5E6
:10224000446D9E6800214FF0FF354A01A31801310B
:10225000D3F800090028BEBFD3F8000940F0804041
:10226000C3F80009D3F8000B0028BEBFD3F8000B59
:1022700040F08040C3F8000BA3188E42C3F8085901
:10228000C3F8085BE1D24FF00113C4F81C3870BDED
:10229000890141F02001016103699B06FCD41220F1
:1022A000FFF738BB204B03EB80022DE9F047D2F853
:1022B0000CE05D6DDEF81420461CD2F800C005EB82
:1022C000063605EB4018516861450BD3D5F8342824
:1022D000012303FA00F022EA0000C5F8340818468A
:1022E000BDE8F087BEF81040ACEB0103A34228BF65
:1022F0002346D8F81849A4B2B3EB840F10D89468D9
:102300001F46A4F1040959F804AFC6F800A0042F31
:1023100001D9043FF7E71C440B4494605360D2E7B3
:102320000020BDE8F08700BF1C2D002010B5054C33
:102330002046FEF779FF4FF0A0436365024BA3658B
:1023400010BD00BF1C2D0020703600080378012B43
:1023500070B5054650D12A4B446D98421BD1294B8C
:102360005A6B42F080025A635A6D42F080025A65FD
:102370005A6D5A6942F080025A615A6922F080020D
:102380005A610E2143205B6900F0D8FB1E4BE360CD
:102390001E4BC4F800380023C4F8003EC02323605D
:1023A0006E6D4FF40413A3633369002BFCDA012331
:1023B00033610C20FFF7AEFA3369DB07FCD412203F
:1023C000FFF7A8FA3369002BFCDA0026A66028463E
:1023D000FFF734FF6B68C4F81068DB68C4F8146852
:1023E000C4F81C684BB90A4BA3614FF0FF3363611B
:1023F000A36843F00103A36070BD064BF4E700BF80
:102400001C2D002000380240401400400300200230
:10241000003C30C0083C30C0F8B5446D0546002192
:102420002046FFF735FFA96D00234FF001128F689A
:10243000C4F834384FF00066C4F81C284FF0FF3061
:1024400004EB431201339F42C2F80069C2F8006BEB
:10245000C2F80809C2F8080BF2D20B686A6DEB6586
:10246000636210231361166916F01006FBD1122067
:10247000FFF750FAD4F8003823F4FE63C4F80038AC
:10248000A36943F4402343F01003A3610923C4F874
:102490001038C4F814380A4BEB604FF0C043C4F84E
:1024A000103B084BC4F8003BC4F81069C4F800396D
:1024B000EB6D03F1100243F48013EA65A362F8BDEB
:1024C0004C36000840800010426D90F84E10D2F853
:1024D000003823F4FE6343EA0113C2F80038704762
:1024E0002DE9F0410EB200EB86080D46D8F80C102D
:1024F0000F6807F00303022B50D0032B50D03D4A46
:102500003D4F012B18BF1746446D4FEA451E04EBA3
:102510000E030022C3F8102B8A6905F1100C002A63
:1025200040D04A8A05F158035B013A43E250012347
:10253000D4F81C2803FA0CF31343A6444A69C4F8E0
:102540001C380023CEF8103905F13F03002A39D09A
:102550000A8A898B9208012988BF4A43C16D04EB1E
:102560008303561841EA0242C66529465A6020464E
:10257000FFF78EFED8F80C301B8A43EA85531F43C1
:1025800005F148035B01E7500123D4F81C2803FA46
:1025900005F51543C4F81C58BDE8F081174FB3E7A3
:1025A000174FB1E704EB4613D3F8002B22F4004297
:1025B000C3F8002BD4F81C28012303FA0CF322EAF9
:1025C0000303BAE704EB83030E4A5A6004EB461692
:1025D00029462046FFF75CFED6F8003923F4004375
:1025E000C6F80039D4F81C38012202FA05F523EAAE
:1025F0000505CFE70080001000800410008008105F
:1026000000800C1000040002826D1268C265FFF7A2
:1026100015BE00005831436D49015B5813F400406A
:1026200004D013F4001F14BF0120022070470000E3
:102630004831436D49015B5813F4004004D013F452
:10264000001F14BF012002207047000000EB810131
:10265000CB68196A0B6813604B68536070470000C1
:1026600000EB810330B5DD68AA691368D36019B93E
:10267000402B84BF402313606B8A1468426D1C4456
:10268000013CB4FBF3F46343033323F0030302EB95
:10269000411043EAC44343F0C043C0F8103B2B68E9
:1026A00003F00303012B09B20ED1D2F8083802EB74
:1026B000411013F4807FD0F8003B14BF43F08053E7
:1026C00043F00053C0F8003B02EB4112D2F8003B4C
:1026D00043F00443C2F8003B30BD00002DE9F04157
:1026E000244D6E6D06EB40130446D3F8087BC3F807
:1026F000087B38070AD5D6F81438190706D505EB34
:1027000084032146DB6828465B689847FA072FD583
:10271000D6F81438DB072BD505EB8403D968CCB980
:102720008B69488A5E68B6FBF0F200FB12628AB9D8
:102730001868DA6890420DD2121A83E81400202338
:1027400083F311880B482146FFF78AFF84F3118831
:10275000BDE8F081012303FA04F26B8923EA020346
:102760006B81CB6823B121460248BDE8F041184790
:10277000BDE8F0811C2D002000EB810370B5DD6801
:10278000436D6C692668E6604A0156BB1A444FF4F3
:102790000020C2F810092A6802F00302012A0AB2D6
:1027A0000ED1D3F8080803EB421410F4807FD4F85C
:1027B000000914BF40F0805040F00050C4F80009F8
:1027C00003EB4212D2F8000940F00440C2F80009BD
:1027D000D3F83408012202FA01F10143C3F8341896
:1027E00070BD19B9402E84BF4020206020682E8A19
:1027F000841940F00050013C1A44B4FBF6F440EA5E
:10280000C440C6E7F8B504461E48456D05EB4413C1
:10281000D3F80869C3F80869F10717D5D5F8103857
:10282000DA0713D500EB8403D9684B691F68DA68AF
:10283000974218D2D21B00271A605F60202383F3CF
:1028400011882146FFF798FF87F31188330617D5C3
:10285000D5F834280123A340134211D02046BDE807
:10286000F840FFF71FBD012303FA04F2038923EAAE
:10287000020303818B68002BE8D021469847E5E7E7
:10288000F8BD00BF1C2D002097482DE9F84F456D7D
:102890006E69AB691E4016F4805F6E61044605D018
:1028A000FEF72EFDBDE8F84FFFF780BC002E12DAD0
:1028B000D5F8003E8C489B071EBFD5F8003E23F09C
:1028C0000303C5F8003ED5F8043823F00103C5F82A
:1028D0000438FEF743FD370505D58348FFF7AEFC06
:1028E0008148FEF72BFDB0040CD5D5F8083813F05D
:1028F000060FEB6823F470530CBF43F4105343F4FA
:10290000A053EB60310704D56368DB680BB17648F0
:102910009847F2025AD4B3020CD5D4F85480DFF8A9
:10292000C8A100274FF00109A36D9B68F9B28B4243
:1029300080F08780F70619D5616D0A6AC2F30A171D
:1029400002F00F0302F4F012B2F5802F00F0A18024
:10295000B2F5402F0AD104EB830301F58051DB6807
:10296000186A00231A469F4240F087803003D5F84A
:10297000184813D5E10302D50020FFF7AFFEA203EC
:1029800002D50120FFF7AAFE630302D50220FFF75C
:10299000A5FE270302D50320FFF7A0FE750381D50E
:1029A000E00702D50020FFF72DFFA10702D5012087
:1029B000FFF728FF620702D50220FFF723FF230756
:1029C0007FF570AF0320FFF71DFF6BE7D4F854804D
:1029D000DFF814A100274FF00109A36D9B685FFA8F
:1029E00087FB5B4597D308EB4B13D3F8002902F420
:1029F0004022B2F5802F22D1D3F80029002A1EDA16
:102A0000D3F8002942F09042C3F80029D3F80029F6
:102A1000002AFBDB5946606DFFF73AFC228909FA70
:102A20000BF322EA0303238104EB8B03DB689B682F
:102A300013B15946504698475846FFF733FC0137C3
:102A4000CBE708EB4112D2F8003B03F44023B3F587
:102A5000802F10D1D2F8003B002B0CDA628909FAE2
:102A600001F322EA0303638104EB8103DB68DB6883
:102A70000BB150469847013756E79C0708BF0A68D4
:102A8000072B98BF027003F101039CBF120A0130AB
:102A900069E7023304EB830201F5805152689069C3
:102AA0000268D0F808C04068A2EB000E0022104671
:102AB00097420AD104EB830463689B699A683A449D
:102AC0009A605A6817445F6050E712F0030F08BF1E
:102AD0000868964588BF8CF8000002F1010284BFA7
:102AE000000A0CF1010CE3E71C2D0020436D03EB01
:102AF0004111D1F8003B43F40013C1F8003B70478B
:102B0000436D03EB4111D1F8003943F40013C1F8D0
:102B100000397047436D03EB4111D1F8003B23F4BA
:102B20000013C1F8003B7047436D03EB4111D1F82E
:102B3000003923F40013C1F80039704700F16043F5
:102B400000F01F02400903F5614309018000C9B28A
:102B500000F1604083F8001300F5614001239340C9
:102B6000C0F880310360704730B5039C01720433B4
:102B700004FB0325C361049B03630021059B0060E4
:102B80004060C160426102618561046242628162AB
:102B9000C162436330BD00000022416A41610161AE
:102BA000C2608262C2626FF00101FEF725BF0000C1
:102BB00003694269934203D1C2680AB10020704799
:102BC000181D704703691960C2680132C260C2698A
:102BD000134482690361934224BF436A0361002165
:102BE000FEF7FEBE38B504460D46E3683BB16269A8
:102BF000131D1268A3621344E362002038BD237AD8
:102C000033B929462046FEF7DBFE0028EDDA38BD51
:102C10006FF00100FBE70000C368C269013BC360BD
:102C20004369134482694361934224BF436A436109
:102C300000238362036B03B11847704770B52023EC
:102C4000044683F31188866A3EB9FFF7CBFF054639
:102C500018B186F31188284670BDA36AE26A13F89A
:102C6000015BA362934202D32046FFF7D5FF002306
:102C700083F31188EFE700002DE9F84F04460E4674
:102C800090469946202787F311880025AA46D4F854
:102C900028B0BBF1000F09D149462046FFF7A2FF3B
:102CA00020B18BF311882846BDE8F88FA16AE36A4A
:102CB000A8EB050B5B1A9B4528BF9B46BBF1400F59
:102CC0001BD9334601F1400251F8040B43F8040BC1
:102CD0009142F9D1A36A40334036A3624035A26ADB
:102CE000E36A9A4202D32046FFF796FF8AF31188DF
:102CF0004545D8D287F31188C9E730465A46FDF7D3
:102D0000D7FFA36A5B445E44A3625D44E7E700002B
:102D100010B5029C0172043303FB0421C36100233C
:102D20008362C362039B0363049B00604060C460D2
:102D300042610261816104624262436310BD00002E
:102D4000026AC260426A4261026100228262C26219
:102D50006FF00101FEF750BE436902699A4203D148
:102D6000C2680AB100207047184650F8043B0B6057
:102D700070470000C368C2690133C36043691344EC
:102D800082694361934224BF436A43610021FEF795
:102D900027BE000038B504460D46E3683BB1236901
:102DA0001A1DA262E2691344E362002038BD237A4F
:102DB00033B929462046FEF703FE0028EDDA38BD78
:102DC0006FF00100FBE7000003691960C268013A77
:102DD000C260C269134482690361934224BF436A9B
:102DE000036100238362036B03B11847704700003F
:102DF00070B5202304460E4683F31188856A35B9E1
:102E00001146FFF7C7FF10B185F3118870BDA36AA3
:102E10001E70A36AE26A01339342A36204D3E1699C
:102E200020460439FFF7D0FF002080F3118870BDE1
:102E30002DE9F84F04460D4691469A464FF020087A
:102E400088F311880026B346A76A4FB95146204639
:102E5000FFF7A0FF20B187F311883046BDE8F88F57
:102E6000A06AE76AA9EB06033F1A9F4228BF1F46E4
:102E7000402F1BD905F1400355F8042B40F8042BD3
:102E80009D42F9D1A36A4033A3624036A26AE36A45
:102E90009A4204D3E16920460439FFF795FF8BF38A
:102EA00011884E45D9D288F31188CDE729463A4694
:102EB000FDF7FEFEA36A3B443D44A3623E44E5E7C2
:102EC000026943699A4203D1C3681BB91846704727
:102ED0000023FBE7836A002BF8D0043B9B1AF5D054
:102EE0001360C368013BC360C3691A44836902610C
:102EF0009A4224BF436A0361002383620123E5E70A
:102F000000F090B84FF08043002258631A6102220B
:102F1000DA6070474FF080430022DA6070470000AB
:102F20004FF08043586370474FF08043586A7047B2
:102F30004B6843608B688360CB68C3600B694361F7
:102F40004B6903628B6943620B6803607047000042
:102F500008B5224B22481A6940F2FF110A431A6150
:102F60001A6922F4FF7222F001021A611A691A6BBF
:102F70000A431A631A6D0A431A651A4A1B6D1146F1
:102F8000FFF7D6FF184802F11C01FFF7D1FF1748E1
:102F900002F13801FFF7CCFF154802F15401FFF7A9
:102FA000C7FF144802F17001FFF7C2FF124802F197
:102FB0008C01FFF7BDFF114802F1A801FFF7B8FF30
:102FC0000F4802F1C401FFF7B3FF0E4802F1E00120
:102FD000FFF7AEFFBDE8084000F0AAB80038024095
:102FE000000002407C360008000402400008024055
:102FF000000C024000100240001402400018024081
:10300000001C02400020024008B500F007FAFEF75D
:103010005FFCFFF785F8BDE80840FEF761BE0000E1
:1030200070470000104B1A6C42F001021A641A6ECD
:1030300042F001021A660D4A1B6E936843F00103C9
:1030400093604FF0804353229A624FF0FF32DA626E
:1030500000229A615A63DA605A6001225A6108219B
:103060001A601C20FFF76ABD00380240002004E00F
:103070004FF0804208B51369D1680B40D9B2C943FB
:103080009B07116107D5202383F31188FEF740FCCD
:10309000002383F3118808BD08B5FFF7E9FFBDE8F9
:1030A0000840FFF783B800001F4B1A696FEAC2524D
:1030B0006FEAD2521A611A69C2F308021A614FF01C
:1030C000FF301A695A69586100215A6959615A6971
:1030D0001A6A62F080521A621A6A02F080521A6208
:1030E0001A6A5A6A58625A6A59625A6A1A6C42F0E3
:1030F00080521A641A6E42F080521A661A6E0B4A97
:10310000106840F480701060186F00F44070B0F5E3
:10311000007F1EBF4FF4803018671967536823F48F
:103120000073536000F05AB900380240007000404C
:10313000334B4FF080521A64324A4FF440411160D1
:103140001A6842F001021A601A689207FCD59A6860
:1031500022F003029A602A4B19469A6812F00C0278
:10316000FBD1186800F0F90018609A601A6842F400
:1031700080321A600B689B03FCD54B6F43F0010350
:103180004B671F4B5A6F9007FCD51F4A5A601A684D
:1031900042F080721A601B4A53685904FCD5184BE0
:1031A0001A689201FCD5194A9A60194B1A68194B92
:1031B0009A42194B21D1194A1168194A91421CD1DE
:1031C00040F205121A60144A136803F00F03052B2E
:1031D000FAD10B4B9A6842F002029A609A6802F0A8
:1031E0000C02082AFAD15A6C42F480425A645A6E90
:1031F00042F480425A665B6E704740F20572E1E726
:10320000003802400070004008544007009488389D
:10321000002004E011640020003C024000ED00E0CA
:1032200041C20F41084A08B5536911680B4003F0C9
:103230000103536123B1054A13680BB150689847E5
:10324000BDE80840FEF7B2BF003C014088230020E3
:10325000084A08B5536911680B4003F00203536133
:1032600023B1054A93680BB1D0689847BDE8084080
:10327000FEF79CBF003C014088230020084A08B5A7
:10328000536911680B4003F00403536123B1054AED
:1032900013690BB150699847BDE80840FEF786BF37
:1032A000003C014088230020084A08B55369116892
:1032B0000B4003F00803536123B1054A93690BB136
:1032C000D0699847BDE80840FEF770BF003C014058
:1032D00088230020084A08B5536911680B4003F0A1
:1032E0001003536123B1054A136A0BB1506A984722
:1032F000BDE80840FEF75ABF003C0140882300208B
:10330000174B10B55C691A68144004F478725A615E
:10331000A30604D5134A936A0BB1D06A9847600696
:1033200004D5104A136B0BB1506B9847210604D596
:103330000C4A936B0BB1D06B9847E20504D5094A50
:10334000136C0BB1506C9847A30504D5054A936CD8
:103350000BB1D06C9847BDE81040FEF727BF00BF07
:10336000003C0140882300201A4B10B55C691A68A4
:10337000144004F47C425A61620504D5164A136D68
:103380000BB1506D9847230504D5134A936D0BB1CB
:10339000D06D9847E00404D50F4A136E0BB1506E00
:1033A0009847A10404D50C4A936E0BB1D06E984790
:1033B000620404D5084A136F0BB1506F9847230479
:1033C00004D5054A936F0BB1D06F9847BDE8104004
:1033D000FEF7ECBE003C014088230020062108B522
:1033E0000846FFF7ABFB06210720FFF7A7FB0621E6
:1033F0000820FFF7A3FB06210920FFF79FFB06210A
:103400000A20FFF79BFB06211720FFF797FB0621F9
:103410002820BDE80840FFF791BB000008B5FFF782
:1034200043FEFDF74FFDFDF7FDFEFDF7D1FDFFF774
:10343000F7FDBDE80840FFF763BD0000034611F843
:10344000012B03F8012B002AF9D170471210121337
:103450001211000053544D3332463F3F3F000000ED
:1034600000000000543400083F0000001304000076
:10347000903400083F000000190400009A3400084E
:103480003F00000021040000A43400083F000000B9
:1034900053544D3332463430780053544D33324612
:1034A0003432780053544D33324634343658580051
:1034B00000000000490F0008350F0008710F0008D8
:1034C0005D0F0008690F0008550F0008410F000844
:1034D0002D0F0008CD0F00080000000001000000C3
:1034E000000000006D61696E0000000004350008F6
:1034F00048240020C025002001000000CD1800084D
:103500000000000069646C6500000000020000001B
:103510000000000075110008DD11000840004000A7
:10352000582A0020682A0020020000000000000045
:10353000030000000000000021120008000000004D
:1035400010000000782A00200000000001000000A8
:10355000000000001C2D0020010102004172647572
:1035600050696C6F740025424F415244252D424CE6
:10357000002553455249414C25000000811C00089C
:10358000E91B0008E1100008651C0008430000006A
:103590009435000809024300020100C0320904000A
:1035A00000010202010005240010010524010001B0
:1035B000042402020524060001070582030800FF17
:1035C00009040100020A0000000705010240000092
:1035D000070581024000000012000000E0350008ED
:1035E00012011001020000400912415700020102BD
:1035F000030100000403090425424F415244250001
:103600004B616B7574654634003031323334353676
:10361000373839414243444546000000004000002D
:1036200000400000004000000040000000000100D9
:103630000000020000000200000002000000020082
:103640000000020000000200000002000000000074
:103650007113000851160008FD16000840004000D4
:103660007C2D00207C2D0020010000008C2D0020EE
:103670008000000040010000030000000000800204
:1036800000000000AAAAAAAA00000000FFFF000094
:103690000000000000A00A0040040010000000002C
:1036A000AAAAAAAA40000010DFFF00000000000044
:1036B000000000000001040000000000AAAAAAAA5D
:1036C00000010800FFFD00000000000000000000F5
:1036D0000000000000000000AAAAAAAA0000000042
:1036E000FFFF0000000000000000000000000000DC
:1036F00000000000AAAAAAAA00000000FFFF000024
:1037000000000000000000000000000000000000B9
:10371000AAAAAAAA00000000FFFF00000000000003
:10372000000000000000000000000000AAAAAAAAF1
:1037300000000000FFFF000000000000000000008B
:1037400000000000000000000A000000000000006F
:103750000300000000000000000000000000000066
:103760000000000000000000000000000000000059
:103770000000000000000000FF00960000000008AC
:1037800004000000F4350008000000000000000004
:103790000000000000000000000000000000000029
:1037A000FFFFFFFFFFFFFFFFFFFFFFFFFFFFFFFF29
:1037B000FFFFFFFFFFFFFFFFFFFFFFFFFFFFFFFF19
:1037C000FFFFFFFFFFFFFFFFFFFFFFFFFFFFFFFF09
:020000040801F1
:1000000000060020A5120108450E0908A10D0908E7
:100010000D0E0908A10D0908D90D0908A71201083C
:10002000A7120108A7120108A712010851FC0A082B
:10003000A7120108A7120108A7120108A7120108B8
:10004000A7120108A7120108A7120108A7120108A8
:10005000A7120108A71201086D0E0B08950E0B08D8
:10006000BD0E0B08E50E0B080D0F0B08F5B70A08BF
:100070001DB80A0849B80A0875B80A08A1B80A08DC
:10008000C9B80A08F5B80A0879B70A08A71201081A
:10009000A7120108A7120108A7120108350F0B08C3
:1000A000A7120108A7120108A7120108A712010848
:1000B0006D100B0881100B0895100B0881BE0A0803
:1000C00029C00A08A7120108A7120108A7120108EF
:1000D000A712010809100B08A71201081D100B0830
:1000E000990F0B08A7120108A7120108B9100B08F5
:1000F000BD100B08D1100B08D5100B0821B90A0848
:10010000A7120108A7120108A5100B08A7120108E1
:1001100031100B0845100B08A7120108A71201089F
:100120004DB90A0875B90A08A1B90A08CDB90A0873
:10013000F9B90A08A7120108A7120108A7120108B5
:10014000A7120108A7120108A71201087D030B08D6
:1001500021BA0A084DBA0A0879BA0A0859100B08D8
:10016000A7120108A7120108A7120108A712010887
:10017000A7120108A7120108A7120108A712010877
:10018000A7120108A7120108A7120108A712010867
:10019000A7120108A7120108A7120108A712010857
:1001A000A7120108A7120108A7120108A712010847
:1001B000A7120108A7120108A7120108A712010837
:1001C000A7120108A7120108A7120108A712010827
:1001D000A7120108A7120108A7120108A712010817
:1001E000F55601080D7B020879E90308FDA605080C
:1001F00021AD050829F70508F1470608B54F06089F
:10020000ED5206084DB8060869DF060861B4070814
:10021000CD0D08080507090869D80908C5330A087B
:10022000255A0A08A1640A0825940A08ED990A08C3
:1002300081F0004102E000BF83F0004330B54FEA97
:1002400041044FEA430594EA050F08BF90EA020F04
:100250001FBF54EA000C55EA020C7FEA645C7FEA97
:10026000655C00F0E2804FEA5454D4EB5555B8BFBA
:100270006D420CDD2C4480EA020281EA030382EA2B
:10028000000083EA010180EA020281EA0303362DBD
:1002900088BF30BD11F0004F4FEA01314FF4801C90
:1002A0004CEA113102D0404261EB410113F0004FA2
:1002B0004FEA03334CEA133302D0524263EB430359
:1002C00094EA050F00F0A780A4F10104D5F1200EF7
:1002D0000DDB02FA0EFC22FA05F2801841F1000152
:1002E00003FA0EF2801843FA05F359410EE0A5F126
:1002F00020050EF1200E012A03FA0EFC28BF4CF057
:10030000020C43FA05F3C01851EBE37101F000450C
:1003100007D54FF0000EDCF1000C7EEB00006EEB19
:100320000101B1F5801F1BD3B1F5001F0CD34908A3
:100330005FEA30004FEA3C0C04F101044FEA4452FA
:1003400012F5800F80F09A80BCF1004F08BF5FEA81
:10035000500C50F1000041EB045141EA050130BD61
:100360005FEA4C0C404141EB0101013C28BFB1F573
:10037000801FE9D291F0000F04BF01460020B1FABE
:1003800081F308BF2033A3F10B03B3F120020CDA91
:100390000C3208DD02F1140CC2F10C0201FA0CF06F
:1003A00021FA02F10CE002F11402D8BFC2F1200CD4
:1003B00001FA02F120FA0CFCDCBF41EA0C0190408A
:1003C000E41AA2BF01EB0451294330BD6FEA0404D3
:1003D0001F3C1CDA0C340EDC04F11404C4F12002BE
:1003E00020FA04F001FA02F340EA030021FA04F3D0
:1003F00045EA030130BDC4F10C04C4F1200220FA27
:1004000002F001FA04F340EA0300294630BD21FA64
:1004100004F0294630BD94F0000F83F4801306BF2A
:1004200081F480110134013D4EE77FEA645C18BF1E
:100430007FEA655C29D094EA050F08BF90EA020FB5
:1004400005D054EA000C04BF1946104630BD91EAAD
:10045000030F1EBF0021002030BD5FEA545C05D1B0
:100460004000494128BF41F0004130BD14F58004EF
:100470003CBF01F5801130BD01F0004545F0FE4163
:1004800041F470014FF0000030BD7FEA645C1ABF98
:10049000194610467FEA655C1CBF0B46024650EACF
:1004A000013406BF52EA033591EA030F41F40021FB
:1004B00030BD00BF90F0000F04BF0021704730B581
:1004C0004FF4806404F132044FF000054FF0000156
:1004D00050E700BF90F0000F04BF0021704730B517
:1004E0004FF4806404F1320410F0004548BF4042EC
:1004F0004FF000013EE700BF42004FEAE2014FEA41
:1005000031014FEA02701FBF12F07F4393F07F4F1B
:1005100081F06051704732F07F4208BF704793F01E
:100520007F4F04BF41F40021704730B54FF4607431
:1005300001F0004521F000411CE700BF50EA010234
:1005400008BF704730B54FF000050AE050EA0102DD
:1005500008BF704730B511F0004502D5404261EB4D
:1005600041014FF4806404F132045FEA915C3FF48E
:10057000D8AE4FF003025FEADC0C18BF03325FEA2B
:10058000DC0C18BF033202EBDC02C2F1200300FADC
:1005900003FC20FA02F001FA03FE40EA0E0021FA01
:1005A00002F11444BDE600BF70B54FF0FF0C4CF4EF
:1005B000E06C1CEA11541DBF1CEA135594EA0C0FA1
:1005C00095EA0C0F00F0DEF82C4481EA030621EADC
:1005D0004C5123EA4C5350EA013518BF52EA033517
:1005E00041F4801143F4801338D0A0FB02CE4FF0C9
:1005F0000005E1FB02E506F00042E0FB03E54FF0F9
:100600000006E1FB03569CF0000F18BF4EF0010EF0
:10061000A4F1FF04B6F5007F64F5407404D25FEAEC
:100620004E0E6D4146EB060642EAC62141EA55519F
:100630004FEAC52040EA5E504FEACE2EB4F1FD0CE1
:1006400088BFBCF5E06F1ED8BEF1004F08BF5FEA5F
:10065000500E50F1000041EB045170BD06F0004611
:1006600046EA010140EA020081EA0301B4EB5C04BE
:10067000C2BFD4EB0C0541EA045170BD41F48011B6
:100680004FF0000E013C00F3AB8014F1360FDEBFDB
:10069000002001F0004170BDC4F10004203C35DAB7
:1006A0000C341BDC04F11404C4F1200500FA05F33A
:1006B00020FA04F001FA05F240EA020001F00042DB
:1006C00021F0004110EBD37021FA04F642EB060151
:1006D0005EEA430E08BF20EAD37070BDC4F10C047B
:1006E000C4F1200500FA04F320FA05F001FA04F23F
:1006F00040EA020001F0004110EBD37041F100012B
:100700005EEA430E08BF20EAD37070BDC4F1200535
:1007100000FA05F24EEA020E20FA04F301FA05F29D
:1007200043EA020321FA04F001F0004121FA04F245
:1007300020EA020000EBD3705EEA430E08BF20EA15
:10074000D37070BD94F0000F0FD101F0004640004F
:1007500041EB010111F4801F08BF013CF7D041EAD1
:10076000060195F0000F18BF704703F000465200D5
:1007700043EB030313F4801F08BF013DF7D043EAA6
:100780000603704794EA0C0F0CEA135518BF95EA5C
:100790000C0F0CD050EA410618BF52EA4306D1D1E3
:1007A00081EA030101F000414FF0000070BD50EA02
:1007B000410606BF1046194652EA430619D094EA8C
:1007C0000C0F02D150EA013613D195EA0C0F05D176
:1007D00052EA03361CBF104619460AD181EA0301CA
:1007E00001F0004141F0FE4141F470014FF0000082
:1007F00070BD41F0FE4141F4780170BD70B54FF01D
:10080000FF0C4CF4E06C1CEA11541DBF1CEA13559C
:1008100094EA0C0F95EA0C0F00F0A7F8A4EB05047E
:1008200081EA030E52EA03354FEA013100F0888075
:100830004FEA03334FF0805545EA131343EA12633E
:100840004FEA022245EA111545EA10654FEA0026F3
:100850000EF000419D4208BF964244F1FD0404F5AC
:10086000407402D25B084FEA3202B61A65EB030508
:100870005B084FEA32024FF480104FF4002CB6EBC5
:10088000020E75EB030E22BFB61A754640EA0C0045
:100890005B084FEA3202B6EB020E75EB030E22BF85
:1008A000B61A754640EA5C005B084FEA3202B6EBC6
:1008B000020E75EB030E22BFB61A754640EA9C0085
:1008C0005B084FEA3202B6EB020E75EB030E22BF55
:1008D000B61A754640EADC0055EA060E18D04FEA13
:1008E000051545EA16754FEA06164FEAC30343EAB3
:1008F00052734FEAC2025FEA1C1CC0D111F4801F80
:100900000BD141EA00014FF000004FF0004CB6E778
:1009100011F4801F04BF01430020B4F1FD0C88BF17
:10092000BCF5E06F3FF6AFAEB5EB030C04BFB6EB22
:10093000020C5FEA500C50F1000041EB045170BD15
:100940000EF0004E4EEA113114EB5C04C2BFD4EB42
:100950000C0541EA045170BD41F480114FF0000EC6
:10096000013C90E645EA060E8DE60CEA135594EA42
:100970000C0F08BF95EA0C0F3FF43BAF94EA0C0F45
:100980000AD150EA01347FF434AF95EA0C0F7FF4BA
:1009900025AF104619462CE795EA0C0F06D152EA0E
:1009A00003353FF4FDAE1046194622E750EA4106F2
:1009B00018BF52EA43067FF4C5AE50EA41047FF403
:1009C0000DAF52EA43057FF4EBAE12E74FF0FF3C68
:1009D00006E000BF4FF0010C02E000BF4FF0010C39
:1009E0004DF804CD4FEA410C7FEA6C5C4FEA430CB2
:1009F00018BF7FEA6C5C1BD001B050EA410C0CBF01
:100A000052EA430C91EA030F02BF90EA020F002062
:100A1000704710F1000F91EA030F58BF994208BFC9
:100A200090422CBFD8176FEAE37040F00100704786
:100A30004FEA410C7FEA6C5C02D150EA013C07D1DD
:100A40004FEA430C7FEA6C5CD6D152EA033CD3D028
:100A50005DF8040B704700BF8446104662468C4622
:100A60001946634600E000BF01B5FFF7B7FF002855
:100A700048BF10F1000F01BD4DF808EDFFF7F4FF7E
:100A80000CBF012000205DF808FB00BF4DF808ED09
:100A9000FFF7EAFF34BF012000205DF808FB00BF2C
:100AA0004DF808EDFFF7E0FF94BF012000205DF84E
:100AB00008FB00BF4DF808EDFFF7CEFF94BF012003
:100AC00000205DF808FB00BF4DF808EDFFF7C4FFFC
:100AD00034BF012000205DF808FB00BF4FEA410C45
:100AE0007FEA6C5C02D150EA013C0AD14FEA430C28
:100AF0007FEA6C5C02D152EA033C02D14FF0000065
:100B000070474FF0010070474FEA410212F50012A2
:100B100015D211D56FF47873B3EB625212D94FEA44
:100B2000C12343F0004343EA505311F0004F23FA2E
:100B300002F018BF404270474FF00000704750EA83
:100B4000013005D111F0004008BF6FF00040704740
:100B50004FF00000704700BF4A0011D212F500129A
:100B600011D20DD56FF47873B3EB62520ED44FEA05
:100B7000C12343F0004343EA505323FA02F0704785
:100B80004FF00000704750EA013002D14FF0FF30C3
:100B900070474FF0000070474FEA4102B2F1E04366
:100BA00024BFB3F5001CDCF1FE5C0DD901F0004C54
:100BB0004FEAC0024CEA5070B2F1004F40EB8300A4
:100BC00008BF20F00100704711F0804F21D113F1D0
:100BD0003872BCBF01F00040704741F480114FEA09
:100BE0005252C2F11802C2F1200C10FA0CF320FA92
:100BF00002F018BF40F001004FEAC1234FEAD323AF
:100C000003FA0CFC40EA0C0023FA02F34FEA430318
:100C1000CCE77FEA625307D150EA01331EBF4FF0A1
:100C2000FE4040F44000704701F0004040F0FE40BC
:100C300040F40000704700BF80F0004002E000BFB9
:100C400081F0004142001FBF5FEA410392EA030FB7
:100C50007FEA226C7FEA236C6AD04FEA1262D2EB01
:100C60001363C1BFD218414048404140B8BF5B4206
:100C7000192B88BF704710F0004F40F4000020F09F
:100C80007F4018BF404211F0004F41F4000121F0B5
:100C90007F4118BF494292EA030F3FD0A2F10102FF
:100CA00041FA03FC10EB0C00C3F1200301FA03F13D
:100CB00000F0004302D5494260EB4000B0F5000F60
:100CC00013D3B0F1807F06D340084FEA310102F11F
:100CD0000102FE2A51D2B1F1004F40EBC25008BFD1
:100CE00020F0010040EA03007047490040EB00009B
:100CF000013A28BFB0F5000FEDD2B0FA80FCACF19C
:100D0000080CB2EB0C0200FA0CF0AABF00EBC250C8
:100D100052421843BCBFD0401843704792F0000FB6
:100D200081F4000106BF80F400000132013BB5E709
:100D30004FEA41037FEA226C18BF7FEA236C21D07F
:100D400092EA030F04D092F0000F08BF08467047E4
:100D500090EA010F1CBF0020704712F07F4F04D1B2
:100D6000400028BF40F00040704712F100723CBFC5
:100D700000F50000704700F0004343F0FE4040F4EF
:100D8000000070477FEA226216BF08467FEA2363AD
:100D90000146420206BF5FEA412390EA010F40F498
:100DA000800070474FF0000304E000BF10F00043E4
:100DB00048BF40425FEA000C08BF704743F09643CB
:100DC00001464FF000001CE050EA010208BF7047E6
:100DD0004FF000030AE000BF50EA010208BF70476D
:100DE00011F0004302D5404261EB41015FEA010C82
:100DF00002BF84460146002043F0B64308BFA3F17A
:100E00008053A3F50003BCFA8CF2083AA3EBC2535B
:100E100010DB01FA02FC634400FA02FCC2F120027A
:100E2000BCF1004F20FA02F243EB020008BF20F0B1
:100E30000100704702F1200201FA02FCC2F1200217
:100E400050EA4C0021FA02F243EB020008BF20EA0C
:100E5000DC7070477BB972B90029BEBF00204FF02B
:100E6000004106E008BF00281CBF6FF000414FF0B2
:100E7000FF3000F015BAADF1080C6DE904CE002981
:100E800009DB002B1ADB00F0A3F8DDF804E0DDE954
:100E9000022304B07047404261EB4101002B1BDB91
:100EA00000F096F8DDF804E0DDE9022304B04042EA
:100EB00061EB4101524263EB43037047524263EBE3
:100EC000430300F085F8DDF804E0DDE9022304B017
:100ED000404261EB41017047524263EB430300F033
:100EE00077F8DDF804E0DDE9022304B0524263EB59
:100EF0004303704753B94AB9002908BF00281CBFF3
:100F00004FF0FF314FF0FF3000F0CAB9ADF1080CDF
:100F10006DE904CE00F05CF8DDF804E0DDE90223C1
:100F200004B0704730B1012390FAA0F0B0FA80F01D
:100F30001844704708460029FBD02123F4E700BF7E
:100F4000430803F05533C01A830803F0333300F02D
:100F50003330184400EB101000F00F3000EB00208D
:100F600000EB0040000E704707EE900AF5EEC07AE5
:100F7000F1EE10FA01D400F00BB8F1EE677A08B583
:100F800017EE900A00F004F8404261EB410108BD01
:100F9000D0B5FFF7B1FA0C4B002206460F46FFF71B
:100FA00003FBFFF7D9FD0446FFF784FA074B002245
:100FB000FFF7FAFA02460B4630463946FFF73CF98E
:100FC000FFF7CAFD2146D0BD0000F03D0000F04112
:100FD0002DE9F047089D04468E46002B4DD18A42EC
:100FE000944669D9B2FA82F252B101FA02F3C2F11F
:100FF000200120FA01F10CFA02FC41EA030E9440B0
:101000004FEA1C48210CBEFBF8F61FFA8CF708FBD0
:1010100016E341EA034306FB07F199420AD91CEBA8
:10102000030306F1FF3080F01F81994240F21C81DA
:10103000023E63445B1AA4B2B3FBF8F008FB103322
:1010400044EA034400FB07F7A7420AD91CEB040457
:1010500000F1FF3380F00A81A74240F20781644427
:10106000023840EA0640E41B00261DB1D4400023AC
:10107000C5E900433146BDE8F0878B4209D9002D10
:1010800000F0EF800026C5E9000130463146BDE89A
:10109000F087B3FA83F6002E4AD18B4202D3824204
:1010A00000F2F980841A61EB030301209E46002DB3
:1010B000E0D0C5E9004EDDE702B9FFDEB2FA82F208
:1010C000002A40F09280A1EB0C014FEA1C471FFA66
:1010D0008CFE0126200CB1FBF7F307FB131140EA4D
:1010E00001410EFB03F0884208D91CEB010103F11A
:1010F000FF3802D2884200F2CB804346091AA4B2DC
:10110000B1FBF7F007FB101144EA01440EFB00FEAF
:10111000A64508D91CEB040400F1FF3102D2A64514
:1011200000F2BB800846A4EB0E0440EA03409CE7B3
:10113000C6F12007B34022FA07FC4CEA030C20FA60
:1011400007F401FA06F31C43F9404FEA1C4900FA80
:1011500006F3B1FBF9F8200C1FFA8CFE09FB1811FD
:1011600040EA014108FB0EF0884202FA06F20BD970
:101170001CEB010108F1FF3A80F08880884240F2C0
:101180008580A8F102086144091AA4B2B1FBF9F004
:1011900009FB101144EA014100FB0EFE8E4508D9FF
:1011A0001CEB010100F1FF346CD28E456AD9023884
:1011B000614440EA0840A0FB0294A1EB0E01A14269
:1011C000C846A64656D353D05DB1B3EB080261EBD7
:1011D0000E0101FA07F722FA06F3F1401F43C5E9B1
:1011E000007100263146BDE8F087C2F12003D840E7
:1011F0000CFA02FC21FA03F3914001434FEA1C4729
:101200001FFA8CFEB3FBF7F007FB10360B0C43EA1A
:10121000064300FB0EF69E4204FA02F408D91CEBCA
:10122000030300F1FF382FD29E422DD902386344C8
:101230009B1B89B2B3FBF7F607FB163341EA034168
:1012400006FB0EF38B4208D91CEB010106F1FF38B7
:1012500016D28B4214D9023E6144C91A46EA0046AE
:1012600038E72E46284605E70646E3E61846F8E640
:101270004B45A9D2B9EB020864EB0C0E0138A3E789
:101280004646EAE7204694E74046D1E7D0467BE76A
:10129000023B614432E7304609E76444023842E7E2
:1012A000704700BF02E000F000F8FEE772B6374872
:1012B00080F30888364880F3098836483649086044
:1012C00040F20000CCF200004EF63471CEF2000184
:1012D0000860BFF34F8FBFF36F8F40F20000C0F282
:1012E000F0004EF68851CEF200010860BFF34F8F38
:1012F000BFF36F8F4FF00000E1EE100A4EF63C7125
:10130000CEF200010860062080F31488BFF36F8FCF
:101310009EF0FCFC9FF046FC4FF055301F491B4AE5
:1013200091423CBF41F8040BFAE71D49184A91422B
:101330003CBF41F8040BFAE71A491B4A1B4B9A427F
:101340003EBF51F8040B42F8040BF8E7002018499F
:10135000184A91423CBF41F8040BFAE79EF0DAFCD0
:101360009FF074FC144C154DAC4203DA54F8041B86
:101370008847F9E701F0F4F8114C124DAC4203DA5A
:1013800054F8041B8847F9E79EF0C2BC0006002011
:10139000002200200000010808ED00E0000000200D
:1013A0000006002090B40D0800220020242C00200C
:1013B000282C002010470120E0010108300201081C
:1013C00030020108300201082DE9F04F2DED108A9E
:1013D000C1F80CD0C3689D46BDEC108ABDE8F08F03
:1013E000002383F311882846A04700209DF0C6FB08
:1013F000FEE79DF023FA00DFFEE7000001F0FF01A9
:10140000102A2BDB10F0070F08D010F8013B013A2F
:101410008B422DD010F0070F42B3F6D1F0B441EA61
:10142000012141EA014122F007047FF00007002377
:10143000F0E80256083C85EA010586EA010685FACD
:1014400047F5A3FA87F586FA47F6A5FA87F68EB927
:10145000EED1F0BC01F0FF0102F0070232B110F84A
:10146000013B013A83EA010313B1F8D10020704730
:1014700001387047002D06BF35460338073815F090
:10148000010F07D1013015F4807F02BF013015F440
:10149000C03F0130F0BC0138704700BF10F8012B8D
:1014A00011F8013B012A28BF9A42F7D0D01A7047A1
:1014B000034613F8012B002AFBD1181A0138704794
:1014C00038B50022002304460D46FFF7DFFA28B99D
:1014D00020462946BDE8384000F00AB8204605F10C
:1014E000004100F005F8404261EB410138BD00BF0A
:1014F000D0B50C4B002206460F46FFF755F8FFF714
:101500002BFB0446FEF7D6FF074B0022FFF74CF8F3
:1015100002460B4630463946FEF78EFEFFF71CFBAF
:101520002146D0BD0000F03D0000F04103680022DC
:101530001B68184710B503685B680446984708B1F4
:1015400094F84D0010BD000038B5044678F018F846
:101550000E4B1D680146E86A0268126890474FF01A
:101560002FFFEB6A93F89C104FF064F894F8373033
:101570005BB17FF099FCEB6AD3F8A030C01AB0F5EC
:10158000FA6F24BF002384F8373038BD342C002094
:1015900070B50E4605465AF079FB5AF03BFB10B980
:1015A0000124204670BD0A4B93F91633012BF7D165
:1015B0005AF06CFB437A002BF2D15AF067FB847A25
:1015C000002CEDD1034A3146284678F01FFAE8E7AF
:1015D000384C0020F8800B0877F088BF2DE9F043E5
:1015E0002DED028BC47F91B006460F468CB990F961
:1015F0000430002B00F0FE807F4B1D68A86A036852
:101600005B6B9847044650B97C4A3946304678F0BF
:10161000FDF9204611B0BDEC028BBDE8F083B36844
:101620004BB933685B6B3946304611B0BDEC028B69
:10163000BDE8F0431847E86AFFF77CFF044600283E
:10164000E7D13946304679F095F8DFF8E481054670
:101650003946304678F002FA98EDCA7AD8EDC97A60
:10166000B4EEE77A2840F1EE10FAC5B209D598F940
:101670002033032B05D0624A3946304678F0C6F94C
:101680002546D8EDB27AB0EE088AF4EEC87AF1EECB
:1016900010FA0BD517EE900AFEF72EFF594ACDE946
:1016A00000013946304678F0B1F90025D8EDB37A1B
:1016B000F4EEC87AF1EE10FA0BD517EE900AFEF7A9
:1016C0001BFF514ACDE900013946304678F09EF9BA
:1016D0000025D8EDB47AB8EE087AF4EEC77AF1EEC8
:1016E00010FA0BDD17EE900AFEF706FF474ACDE928
:1016F00000013946304678F089F90025B8F9B4324E
:10170000042B07DC052200923946414A304678F026
:101710007DF90025D8F85C0B5AF014FB80B198F9DC
:1017200016336BB1D8F85C3BB8F91823B3F90E3017
:101730009A4205DA374A3946304678F067F900258B
:10174000DFF8F09039463046FFF722FF99F8213D47
:10175000002B48D100EA05042F484FF4806100F0C7
:10176000F5FE78B1D8F85C3BB3F90C30A3F2E24255
:1017700092B2B2F5FA7F05D9284A3946304678F058
:1017800045F90024264890F8BC335BB100F56D7034
:101790002CF072F9054628B9224A3946304678F0CD
:1017A00035F92C4600212E2204A80DF10C080391D6
:1017B000A2F070FAD9F80C0D4246322107F0DCFD98
:1017C000054600287FF425AFD9F80C0D03689B6807
:1017D0009847154ACDF8008003463946304678F0E0
:1017E00015F92C4615E7114A3946304678F00EF9BE
:1017F0000024B1E701240CE7342C002008810B08F9
:101800001F810B0842810B0862810B0884810B0841
:10181000A6810B08C5810B08382C002000820B081C
:10182000387C002028820B0838320C08EB810B082A
:10183000384C0020386C002070B505460E46FFF786
:10184000A7FE31460446284678F04CFE2040C0B240
:1018500070BD0000F0B591B005460E4678F09EF9D7
:101860000446D8B11021284677F0A6FEB0B1002179
:101870002E2204A803AF0391A2F00CFA0FF06CFD26
:1018800032233A4601210FF075F8044630B9054B72
:10189000009732461021284677F096FE204611B078
:1018A000F0BD00BF3C820B0870B505460E46B1B9CD
:1018B00090F910408CB116480AF08EFCDFED157AD5
:1018C000B0EEC00AB4EEE70AF1EE10FA07D4124AFD
:1018D0000121284678F09AF83446204670BDAB685E
:1018E0009BB10E4B1B68D86AFFF724FE044630B14B
:1018F00058F0DAFC0A4A042151F00AFEEDE73146BD
:101900002846BDE8704078F015BC0124E5E700BF2B
:10191000382C00200000003448820B08342C0020B2
:101920005A820B0838B5044678F0E4FF0546A8B1A2
:101930000B4804F0F7FF38B10A490B480FF05AF989
:1019400010B1074800F0D4FD2046FFF7FDFD01234C
:10195000064984F83730204678F0DCFE284638BD4A
:10196000382C00202C820020E83E00207C820B08CE
:10197000F8B505460E461746C2B1232901D0012904
:1019800014D81E4807F088F8044668B100242046A1
:10199000F8BD95F91030022B08D058F085FC184A94
:1019A000062151F0B5FDF2E7002EF2D03A4631465D
:1019B000284679F04BF804460028E7D0114ED6F8B7
:1019C0000C2D06F54A639A4203D003F214702CF0F2
:1019D00089FCD6F80C0D03689B6B98470A4B83F87B
:1019E00088032846FFF7B0FD4FF0FF330749C6F8DC
:1019F0003C3D284678F08EFEC9E700BF382C002019
:101A00008C820B08386C0020387C0020A4820B08E4
:101A1000F8B505460E4677F07BFE104B93F9EB7256
:101A20000446CFB90E48BD212CF0F2FB38B10D4B66
:101A300032464FF48041284677F0C6FD3C460848C0
:101A4000BC212CF0E5FB38B1074B32464FF4804106
:101A5000284677F0B9FD00242046F8BD384C002018
:101A6000EC7F0020B8820B08E4820B08002070474E
:101A7000014800F0E5BC00BF382C002003685B681B
:101A8000184700000CF0C8BC61F0B0BC5AF04CB86C
:101A900024F01ABF4EF04CBF07F034B909F09CBED9
:101AA00002F0BEBD4CF000BE13F036BC5DF0B6BC1B
:101AB0005DF034B90BF0ACBD45F022BC0AF00ABCB5
:101AC00012F0AABF63F012BA59F050BD57F05ABED7
:101AD00006F044BB04F09CB909F034BA09F0EABD41
:101AE0000BF0CABB0BF042BE0AF02CBA0BF0EABCFA
:101AF00001F01EB900F2845016F0A6BC06F06EBECE
:101B000090F8F432B02202FB030390F8382393F8E4
:101B1000D13012B1012B28BF0123184670470000B5
:101B2000034808602B21117008221A60704700BF1B
:101B300028860B0870B5044604F5955500F5AD40B0
:101B400074301035FFF700FD002128460FF08AFBA6
:101B5000802120460CF078F818B126F0A9FA24F07C
:101B600041FB04F50053D3EDB27ADFED236A93ED28
:101B7000B47A67EEA67A04F58052FDEEE77A02F2B7
:101B8000FC41D1ED006AF8EEE77A02F59F6267EE5C
:101B9000A67A03F53763FDEEE77A05F5457017EE93
:101BA000901A43F8041CD2ED007AF0EEE77A67EE63
:101BB000877A04F5AF51C3ED007A083129F050FA65
:101BC00004F5A04694ED467AD6EDC17AE7EE007AA8
:101BD000C6EDC17AB0EE670A26F092FF4FF400110D
:101BE00086EDC10A20460CF02FF820B12846BDE84A
:101BF00070400DF06DBE70BD0000C842FFF79ABF87
:101C000010B500F580430446D3F80C0D03689B6BB8
:101C1000984704F5A04393F843333BB930B104F53A
:101C200030500830BDE810407DF0C6B810BD00004F
:101C3000FFF7E6BF38B54FF4801104460CF004F806
:101C4000054620B9012120460BF0FEFF0546022182
:101C500020460BF0F9FF48B115B9204602F088FC88
:101C600004F5955010300DF031FD01E0002DF7D155
:101C70004FF4805120460BF0E7FF30B104F5AC4043
:101C80007030BDE838405DF0EFBC38BDFFF7D2BF23
:101C900038B54FF4801104460BF0D6FF01210546FC
:101CA00020460BF0D1FF18B115B9204602F060FCB8
:101CB000102120460BF0C8FF60B1204602F0C8FC9E
:101CC0004FF4800120460BF0BFFF18B926F0F0F961
:101CD00024F07AFB202120460BF0B6FF28B12046E5
:101CE00002F02CFD204602F045FE4FF40051204644
:101CF0000BF0AAFF10B1204602F024FE80212046FE
:101D00000BF0A2FF28B126F0D3F9BDE8384024F04B
:101D10008DBA38BDFFF7BCBF00F5804300F5AA407F
:101D2000D3F8301D58307AF089BA0000FFF7F4BFBD
:101D300010B5044616F078FC90F921308BB190F87C
:101D4000403373B194F9A8355BB1064B1B68DB6A6D
:101D500093F89C302BB904F28450BDE8104016F083
:101D60008BB910BD342C0020FFF7E2BF2DE9F843FA
:101D7000434B1B68DB6A93F89C300446002B7DD0F4
:101D800000F5805797F8B935002B77D006F084FE20
:101D9000002873D004F5FC5507F58059183599F8DB
:101DA000E61028460DF036F8002867D004F5907646
:101DB0003046FFF7A5FE022860D994F814344FF09E
:101DC000B00808FB034393ED837AF1EE007AB4EE9A
:101DD000E77AF1EE10FA51D499F8E61028460DF0A2
:101DE000C9FA04F50053B3F9B42207EE902AB8EE0D
:101DF000E77AB4EEC07AF1EE10FA0CDD94F8142410
:101E000008FB0242F8EE677A92ED837AF4EEC77A25
:101E1000F1EE10FA32DCD7F8A824D3F86C1B002AB4
:101E2000B8BF52428A4229DC07F2AC42D2ED007AB6
:101E3000D3EDB36A9FED136AF8EEE77A66EE866A31
:101E4000F4EEE67AF1EE10FA18DC03F5376292ED63
:101E5000007A27EE067AF4EEC77AF1EE10FA0DD486
:101E600094F81414B02202FB01612846B3F9B6229B
:101E700001F58271BDE8F8430CF0B6BEBDE8F88309
:101E8000342C00200000C842FFF770BF2DE9F0415C
:101E900090F814342D4D00EB03132F68D3F8C48150
:101EA00000F5907604463046FFF72AFE474514D0E9
:101EB000022814D904F58047C5F8008097F8343D0E
:101EC000012B15D817D104F5A045D5F8FC35E3B999
:101ED000D5F80036CBB905230BE0022810D804F55D
:101EE000804393F8342D5AB1052283F8342D07E04E
:101EF000013B87F8343D04F5B7500C3010F0ACFBD3
:101F00002046BDE8F04109F0C5B9114B1B68D86AFD
:101F100003685B68984780460028ECD194F8141455
:101F2000B02303FB0161DC31204604F06DFDD5F8E0
:101F3000E0350FCB05F2E45605F2046586E80F00A4
:101F400085E80F0087F8348DD5E700BF282C0020E6
:101F5000342C0020FFF79ABF10B500F5A04300F520
:101F6000805493F843231AB1002384F8B9350AE06A
:101F7000D3F89033042B07D100F5A9404C307DF005
:101F8000B9F984F8B90510BD0123EEE710B500F5E5
:101F9000804400F59943D4F80C1D2033994200F594
:101FA000A04308D000F59942643291421CBF4FF023
:101FB000FF32C3F8FC22074AC3F8EC22064AC3F8F2
:101FC000F022FFF7C9FFD4F80C0D0368BDE81040FC
:101FD0001B6918470000C8420000C8C2FFF7D6BFFF
:101FE000F7B500F5A0460446D6F890338B420D466F
:101FF0003FD00B1F00F5A947594207F14C07594143
:10200000384601917DF066F8019938467DF062F816
:10201000042D02D1184869F0E5FDD6F89033012B64
:1020200018D1032D16D104F5AD40743077F0B2FA13
:1020300040B1204606F030FD20B104F52C500430AC
:1020400069F0CAFD2046C6F8905303B0BDE8F040E1
:1020500002F0DEBB072DF5D104F54C50D6F80C2369
:102060006423052192FBF3F31830044A51F050FA2F
:10207000E8E703B0F0BD00BF3C57002088830B08A1
:1020800038B500F580450446D5F80C0D03689B6B08
:102090009847002840D004F5A04393F88823DABB82
:1020A000D5F80C1D04F599422032914236D193F8AF
:1020B0003C232AB901212046BDE83840FFF790BFF4
:1020C000B3F8F223152A27D193F8D01411F00101A7
:1020D00020D1D3F89023072A1CD093F946350BB9A9
:1020E0000421E8E720460AF077F8DFED0F7AB4EE36
:1020F000E70AF1EE10FAF3DB04F5A9404C307DF06D
:1021000039F80028ECD004F54C50084A0621183064
:1021100051F0FEF90721CEE70321CCE704F59943FE
:1021200064339942F8D138BD0000B442AC830B0847
:1021300038B5214CD4F80C2D04F54A639A422DEDA4
:10214000028BB0EE408A03D00020BDEC028B38BD7C
:1021500004F58055D5F89033042B23D194F8353D00
:1021600033B11649A1F510702CF034FB0028ECD1E6
:102170009FED137AF0EEC87AF4EEC77AF1EE10FA1A
:1021800007D49FED100A28EE008ABDEEC88A85EDBF
:10219000C38A0D487CF0EEFF0028D5D0002385F8D7
:1021A0003F33D2E7B5F8F213A4F5804005F036FED0
:1021B0000028D3D1C8E700BF386C00202C82002053
:1021C000000000340000C8420481002010B52DED4D
:1021D000028B00F5A0430446D3F89023042A0BD1C8
:1021E00004F0C4F82046B0EE408A04F0F3F838EE6C
:1021F000400ABDEC028B10BD03F2246393ED000A8C
:10220000F7E700002DE9F0412DED028B00F58C651C
:102210008AB00446284611F0D9FB04F595500023F6
:1022200007A910300793089309930EF0A7FE002822
:1022300000F081809DED090ADFED567A04F5A04596
:1022400095EDC77A20EE270ADFED537AA7EE270A2D
:1022500004F5A9402C3004F5804685EDC70A63F0EB
:1022600059F82046FFF70CFFD6F80C0D03689B6B5E
:10227000984795F84333002B58D1002856D095F84D
:102280008833002B52D1D5F89033042B6AD09FEDC0
:10229000438A204604F0C0F8C5F8AC07D6F80C2DE8
:1022A00004F5994338339A4204F500581AD195F849
:1022B0006836BBB9B8F93C3B002B04DC384AD2F88D
:1022C000FC2AD2060ED5D5F8E015D5F8E8254968E0
:1022D0000A33521A64214B438242ACBF9B181B182D
:1022E000C5F8AC37D6F8382DD5F8AC17D5F89033FB
:1022F00005912046049203930BF00CFFB6F9466D4E
:1023000007462046FFF762FFCDE9007604F530501E
:10231000F0EE400ADDE90332D8EDD41A95EDEB1A60
:102320000599B0EE480A08307CF0EAF90AB0BDEC35
:10233000028BBDE8F08104F59070FFF7E1FB022805
:102340000AD994F81434B02202FB034393F84022D4
:1023500012B193ED8B0A6FE7284611F0D1F9B1EE77
:10236000400A69E704F5AB4704F5AC48743708F157
:10237000040804F5AB4142466431384615F098FA3A
:10238000002884D04146384615F026FBB0EE408A3E
:102390007FE700BFCDCC4C3ECDCC4C3F00000000D1
:1023A000384C0020FFF72EBF00F5804200F599431E
:1023B000D2F80C2D5C339A421FBF00F5A040D0F834
:1023C00024330B60012008BF0020704710B500F5D2
:1023D000804200F59943D2F80C2D5C339A420C46AA
:1023E00012D000F54050D0F8400503681B699847AB
:1023F00007EE900A9FED057AF8EEE77A012067EE86
:10240000877AC4ED007A10BD0020FCE70AD7233C90
:1024100010B500F5804200F59943D2F80C2D5C33DD
:102420009A420C460AD000F54050D0F840050368A7
:102430005B699847012084ED000A10BD0020FCE78D
:1024400030B505460FC985B06C4684E80F0040F2F0
:1024500079322146284604F06BF90C4B03F6C8424A
:10246000D3F80C3D93420ED19DF8001011F00401F9
:1024700002D1204615F018F80548214604F012FA5A
:10248000012005B030BD0020FBE700BF386C002004
:10249000382C002000F58040D0F80C0D03689B6CB0
:1024A0001847000000F58040D0F80C0D0368DB6C85
:1024B0001847000010B500F5805303F5976403F248
:1024C000B443246814601B680B6000F50050D0F81A
:1024D000FC3A9B0509D4D0EDD46AD2ED007A9FED89
:1024E000037AE6EEC77AC2ED007A10BD35FA8E3C6B
:1024F00038B50D4D044629460C480EF08DFC04F508
:10250000804305F1300183F8350D04F59550103006
:102510000EF01AFB04F5AC40D0ED097AF1EE677AC3
:10252000C0ED097A38BD00BF2C820020E83E0020B3
:1025300010B5044600F590701EF020FC2046BDE862
:102540001040FFF7D5BF0000FFF7F2BF00F50050C5
:10255000D0F8FC3A194214BF012000207047000057
:1025600038B5054B1C6823680A461D68034B0146B5
:102570002046A847002038BD342C0020382C0020ED
:1025800070B52DED028B0446036804F500559B6D74
:102590009847D5F8FC3A1B0618D5B5F9B432B5F909
:1025A000B612CA1A0B4402EBD27203EBD373521069
:1025B0005B1000EE902A00EE103A04F59550F8EE0C
:1025C000E00AB8EEC00A10300EF07CF8554BB5F8B2
:1025D000E6221A7004F5AD455BF0C0FC74355BF083
:1025E0000FF900212846FEF7F9FF4F4E0123B07185
:1025F0002846F37176F0C4FF28B9284678F09EF893
:10260000B0FA80F040093071284676F0B9FFE8B999
:1026100094F8143404F5A04504EB031341F2883216
:10262000D3F8C461D5F86C36F31A93420ED904F589
:102630009070FFF765FA022808D9C5F86C66204645
:1026400005F2CC4504F06EF900232B60B4F9A430F8
:102650001BB9B4F8A230A4F8A430B4F8A430DFED6C
:10266000338A07EE903AF8EEE77AB7EE008A88EE02
:10267000270AD4ED2B7AF0EEE77AF4EEE87AF1EE61
:1026800010FA09D5B4F9A23007EE903AF8EEE77ADD
:1026900088EE277A84ED2B7AD4ED2B0A26F032F9D6
:1026A00020BB4DF0D1F940F27D124FF480114DF076
:1026B00083F94CF0AFF84BF017FD04F53B500430B4
:1026C000B0EE408A70F0BCF804F54050B0EE480A15
:1026D000203070F0B5F8B0EE480ABDEC028B04F57E
:1026E00045501430BDE8704070F0AAB8D4ED2B7A94
:1026F00094ED460AF0EEE77AF4EEE87AF1EE10FA9D
:1027000009D5B4F9A23007EE903AF8EEE77A88EEF0
:10271000277A84ED2B7AD4ED2B0A26F0F3F80028E3
:10272000BFD0C6E77D230020958400200000003440
:10273000FFF726BF70B500F5A046044696F944356C
:10274000002B28DD06F0A8F928BB04F5AD4574354B
:10275000284677F0F3FFF0B1284676F011FFD0B1AC
:102760007EF0A2FBD6F82C33C01A96F944354FF40C
:102770007A72534398420ED301221C212846FFF758
:10278000F7F840B104F54C50034ABDE8704006210B
:10279000183050F0BDBE70BDCC830B0830B52DEDA8
:1027A000028B044683B000F5955001A910300EF05D
:1027B000B7FB002871D004F5A04595EDC57ADDED95
:1027C000017AB4EEE77AF1EE10FA08D504F5AD40DF
:1027D000743076F0DFFE10B1019BC5F8143304F5B8
:1027E0000054D4EDC26AB4F9B432052BB8BF052346
:1027F00007EE903AB4F9B63207EE103AB8EEC77A5F
:10280000F8EEE77A37EE077A1820C6EE870AB6EEBA
:10281000007AF4EE470AF1EE10FAC8BFF0EE470A6C
:102820009FED2D7A67EE877A9FED2C7A86EEA71AB8
:10283000F0EE007AB4EE671AF1EE10FA48BFB0EE8F
:10284000671ADDED017AF4EEC77AF1EE10FACCBF2B
:1028500086EEA70AB0EE410A26F066F9B0EE408A8D
:102860001F480DF067FB90B91E484021FFF76EFE30
:1028700068B11D4BD3F89033012B08D1F7EE007AE5
:10288000B4EEE78AF1EE10FA58BFB0EE678AB0EE08
:10289000480A03B0BDEC028B30BD04F5AD40743086
:1028A00076F078FEB7EE008A0028D9D046205AF09C
:1028B000F7FDB4EEC80ADFED0D7AF1EE10FAD8BFDD
:1028C000B0EE480A87EE800A9FF038F92F209FED7E
:1028D000081ADFED080ABFE73333333F17B7D138A3
:1028E000E83E0020382C0020387C002000003442D4
:1028F0008FC2D53F9A99193FF8B5044659F0C6F9E9
:102900000368DB689847054610B900252846F8BDDE
:10291000204605F051FF04F580460746D6F80C0D19
:1029200003689B6B984780B10E4BD3F80C0D03687E
:102930005B6B984748B104F5005494F95D33002B64
:10294000E3D0032BE1D03D46E0E796F8203D002B95
:10295000DCD004F5005494F92053023D18BF012542
:10296000D4E700BF386C002073B500F5804202F652
:10297000545393ED000AD2F80C2D00F598433C33E4
:102980009A422BD100F50053D3F8543BB3F90840D9
:10299000003C18BF012400F5A04300F53A5500F5AE
:1029A0008050D3F8A463D0F8A82493F8A0330C3552
:1029B000B61A5BB10A488DED010A4FF40061FFF7CA
:1029C000C5FD9DED010A80F00100C3B222463146EB
:1029D000284602B0BDE8704078F054BD0024DAE724
:1029E000382C002010B5044605F010FB98B104F512
:1029F000A042D2F8A43303F58C415031C2F8A4139D
:102A000004F58051D1F8A8140029BEBFA3F58C436A
:102A1000503BC2F8A4332046FFF7A6FFBDE81040A4
:102A200004205AF029BD00002DE9F0412DED048B62
:102A300000F5005696EDD48ADFED378A28EE288A15
:102A400000F58048BDEEC88A00F5A04708F654534B
:102A500093ED009AD7F8A83318EE102A1A4408EE1E
:102A6000102A054646205AF01BFDB8EEC88AD6ED5E
:102A7000BE7AD8F80C0DA0EE278A05F598433C33B2
:102A80009842FDEEC87A17EE904A42D1D6F8583BEC
:102A9000B3F90860003E18BF012603685B699847D8
:102AA000C0B9D8F80C0D03689B6B984790B9D7F85C
:102AB000A437022B0ED1284609F0E2F950B107F2F3
:102AC0002453D3ED007A67EEA87AFDEEE77A17EE8D
:102AD000903A1CB205F53F5805F5805508F12408D9
:102AE000D5F8AC34E41A97F8A0333BB10B484FF457
:102AF0000061FFF72BFD80F00100C3B2B0EE490A80
:102B0000BDEC048B324621464046BDE8F04178F0EA
:102B1000F5B90026C1E700BF0000C842382C0020EC
:102B200010B504460BF034FC68B100B200EB400075
:102B3000C0EB001300EE103AB8EEC00ABDE810403A
:102B400013205AF099BC2046FFF76EFFF6E700000D
:102B500010B50E48FFF7D0FEB0B10D4C04205AF06E
:102B60009FFCD4F8540B59F001FB04205AF084FC6C
:102B700013205AF095FCD4F8580B59F0F7FABDE839
:102B8000104013205AF078BC10BD00BF382C002034
:102B9000384C0020F8B52DED028B0446FFF7ACFE53
:102BA000002800F0818004F5804704F59842D7F8AA
:102BB0000C3D4C32934277D004F5984274329342E4
:102BC00072D004F59942183293426DD004F59842C0
:102BD0007C32934268D004F599420432934263D028
:102BE00004F59842443293425ED004F50055F6EE67
:102BF000008AD5F8540B59F079F9B4EEE80AF1EEF1
:102C000010FA3EDDB0EE087AFFEE007AE0EE077AC9
:102C1000B0EE670AD5F86C2B07EE902A04F5A046B3
:102C2000B8EEE77AD6EDE97AF8EEE77A5142E7EEC8
:102C3000007AFDEEE77A17EE900AC6EDE97A26F003
:102C400013F8C6F8A403D7F80C2D04F599434033C4
:102C50009A4222D0D5F8580B59F048F9B4EEE80A58
:102C6000F1EE10FAB0EE408A21DCFEEE007AB4EE0E
:102C7000E70AF1EE10FA22D5B0EE087AF7EE007A04
:102C800019E0FEEE007AB4EEE70AF1EE10FAC1D5D3
:102C9000B0EE087AF7EE007AB8E723484FF4805197
:102CA000FFF754FC0028D5D0BDEC028BF8BDB0EE88
:102CB000087AFFEE007AE8EE077AB0EE678A2046DF
:102CC00005F0A4F908B1B1EE488AD5EDB36AD6EDA6
:102CD000EA7A9FED166A05F5376595ED007AB5EE4F
:102CE000C08AF1EE10FACCBF28EE268A27EE488A79
:102CF000F8EEE77A66EE866AE8EE067A27EE067A5E
:102D0000FDEEE77AFDEEE66ABDEEC77A16EE902A92
:102D100017EE101A17EE900AC6EDEA7A25F0A4FF16
:102D2000C6F8A803C0E700BF382C00200000C84246
:102D300070B5044604F580457EF0B6F8D5F81C3D24
:102D4000C31AB3F5FA6F064603D9D5F80C0D06F091
:102D50002DFB2E4BC5F81C6DD3F80C0D02681368C3
:102D600098470021204609F037FADFED297AB0EEC6
:102D7000C00AB4EEE70AF1EE10FA45D504F5AC430B
:102D8000D3ED097AB1EE047AF0EEE77AF4EEC77A81
:102D9000F1EE10FA38D504F58C6010F0B1FCF6EEC7
:102DA000007AB0EEC00AB4EEE70AF1EE10FA2BD5C5
:102DB00004F5B55595ED057AF0EE087AB4EEE77AAC
:102DC000F1EE10FA05F114051ED504F53A500C3059
:102DD00078F0C8FB04F53F50243078F03FF904F553
:102DE00044503C3079F06CF895ED007AF7EE007ABB
:102DF000B4EEE77AF1EE10FA06D504F54A50303019
:102E0000BDE8704078F0B2BD70BD00BF386C0020E6
:102E10000000003400F5005090F9AB32012BC3BF25
:102E200000F6084090ED290ADFED047A9FED040AD0
:102E3000C8BF20EE270A46205AF01EBB0000C84239
:102E4000000000002DE9F8432DED028B00F58049CC
:102E500009F65453D3ED008A054608F02FFE0746C5
:102E6000D9F80C0D03681B6A984705F544563C36A3
:102E700098B14B4CD4F86833002B0EDD7EF014F87B
:102E8000D4F86833C01A40F6B733984205D8B4F97D
:102E90005C43304679F020F874E005F5A04805F56C
:102EA000005498F8993743B1B4F93C33002B04DD52
:102EB00005F5405393F9523103BBD9F80C3D05F5A4
:102EC00098453C35AB4267D00021B0EE680A3046E9
:102ED00078F09AFD054604205AF0E2FA2BB207EE8C
:102EE000903A94EDBC7AF8EEE77AE0EE077AFDEEE0
:102EF000E77A17EE904A3C4424B2CAE701212846FB
:102F000008F0B4FF9FED277AB4F93C33C0EE077A9E
:102F100008EE103AB8EEC88A9FED230A28EE278AF9
:102F2000D8EDE97AF8EEE77A67EE807A9FED1F0A2E
:102F300027EE800A9EF026FCB4F9B432DFED1C7A4D
:102F400098EDEC7A20EE270A07EE903AF8EEE77A51
:102F50000021B4EEE77AF1EE10FA58BFF0EE477AAE
:102F600080EE277A3046DFED137AB0EE480AA7EEFE
:102F7000270AF0EE680A78F0A3FEBDEEC00A10EE54
:102F8000103A1CB2BDEC028B20460B49BDE8F84359
:102F900041F2941225F078BE391E18BF012194E742
:102FA000387C002000A08C450AD7233C35FA8E3CA3
:102FB0000AE81C41E02E65426CEEFFFF38B500F5D3
:102FC00040530546D3F840050368DB68984701463F
:102FD00005F54A50303078F0ABFC04B22846FFF7D4
:102FE0008BFC70B107EE904A05F50055B8EEE70A84
:102FF000D5F8600B59F0BAF8BDEEC00A10EE103AE1
:103000001CB220460349BDE8384041F2941225F035
:103010003BBE00BF6CEEFFFF38B590F81434B02211
:1030200002FB030393ED837AF7EE007AB4EEE77ABE
:10303000F1EE10FA044600F5A0451CD5002109F078
:10304000CBF8DFED407AB0EEC00AB4EEE70AF1EE5D
:1030500010FA10D5D5F89033012B0CD0072B0AD0DD
:10306000002385F800330023C5F804332046BDE86B
:10307000384008F023BD7DF017FFD5F80833C5F8B8
:103080000803C31AB3F57A7F84BF002385F80033A1
:10309000204608F013FDD5F89033012B07EE100AF7
:1030A0002DD0072B2BD0B8EEC77ADFED276AC7EEFD
:1030B000267A04F50052B2F9002300EE102AB8EE89
:1030C000C00A27EE800ADFED1F7AB0EEC07AB4EEB8
:1030D000E77AF1EE10FA14D4002385F8003395F85E
:1030E000003304F54A503030D3B978F009FBBDE81D
:1030F0003840164900B241F2941225F0C5BD9FED4B
:10310000140A95F80023002AE9D10122934285F898
:103110000023E4D0072B1CBF0023C5F80433DEE7EF
:1031200095EDC17ADFED0B7A67EEC77A9FED0A7AEB
:1031300067EE877AFDEEE77A17EE901A78F0F8FBE3
:10314000D5E700BF0000003400A08C456CEEFFFF07
:1031500000000000E02E65420000C84270B52DED71
:10316000028B00F5A9464C3682B0054630467BF00E
:1031700031FF0446D8B905F50052D2F8543BB3F9F3
:10318000083073B905F5AC43D3ED097A92EDBF7AF7
:10319000F0EEE77AF4EEC77AF1EE10FA4CBF0124B4
:1031A000002430467BF02AFF002808BF0024304668
:1031B0007BF010FF28BB05F5A043D3F8FC320133A8
:1031C00019D0F4B99FED1A8A2846FFF73BFE07EEA7
:1031D000900AB8EEE70A8DED010AD4B915205AF02D
:1031E0004BF99DED010A1A2002B0BDEC028BBDE83F
:1031F00070405AF041B9002CE4D02846FFF70CFF8C
:1032000002E02846FFF7DAFE07EE900AB8EEE78AFA
:10321000DAE71A205AF0D2FB9DED010A08B9B0EEA8
:10322000480A15205AF028F9B0EE480ADBE700BF3B
:103230000000000010B500F5005303F53762D3ED30
:10324000B36ADFED127A92ED007A9FED116A03F610
:10325000084366EEA76A27EE277AD3ED2A7A67EE4F
:10326000867AFDEEE66ABDEEC77AFDEEE77A0446A1
:1032700016EE902A17EE101A17EE900A25F0F4FCBD
:1032800004F5A044C4F8A80310BD00BF0000C84264
:10329000A00CB34510B504460AF0DAFC031E26DB89
:1032A00004F5005191F9AB229A4220DD04F5A040CB
:1032B000D0F89043022C1AD0D1EDC17ADFED0C6A20
:1032C000D31A66EEE76A07EE102A07EE903AB8EED8
:1032D000C77AF8EEE77A87EE876AD0EDEA7AF8EEF9
:1032E000E77AE6EE867AFDEEE77AC0EDEA7A10BD7F
:1032F0000000C84270B52DED028B00F5A045D5ED5C
:10330000E97A9FED400A9FED407AF8EEE77A0446AD
:1033100067EE807A9FED3D0AF0EEE76AF4EE476AC9
:10332000F1EE10FAC8BFF0EE477A27EE800A9EF061
:1033300069F825F01BFBB7EE008AC8EE007A04F5A9
:103340000056C5EDEB7A96F9DC3243B3204604F023
:103350005DFE20BBB6F9B432D5EDEC6A012BB8BFE7
:10336000012307EE903AF8EEE77A86EEA77AB4EEFC
:10337000C87AF1EE10FA15D840F6C4122449D5F8EF
:10338000A40325F071FCC5F8A403D6F86C2B40F615
:10339000C4139A42D4BFC6F86C2BC6F86C3BBDEC84
:1033A000028B70BDD5EDEB7AB4EEE77AF1EE10FA50
:1033B000F5D588EE070A20EE000A9EF00DFADFED43
:1033C000157AD5F8A40320EE270ADFED137A20EE54
:1033D000270A40F6C413FDEEC07A17EE904A9C42CD
:1033E000B8BF1C462246614225F03EFCC5F8A40346
:1033F000D6F86C3BA342D4BFC6F86C3BC6F86C4B06
:10340000CDE700BF0AD7233C0000AA4235FA8E3C24
:103410003CF6FFFFE02E65420000C84210B500F503
:1034200040530446D3F8400503681B68984704F5E9
:103430000053D3F86C2B514225F016FC04F5A04341
:10344000C3F8A4032046BDE81040FFF753BF0000B7
:103450007047000001207047082070470120704726
:1034600070470000014B93F8E8027047384C002089
:10347000034B93F9F00A003818BF0120704700BFD2
:10348000384C0020014B93F9EA027047384C002079
:1034900013B5064BD3F80C0D4B6904680093083143
:1034A0000EC9646CA04702B010BD00BF386C00208C
:1034B00070470000002070477047000038B5254D68
:1034C000D5F80C0D03685B6898470F2834D80F288F
:1034D00039D8DFE800F00836080808080808083876
:1034E00036363636363610241B4B93F8112312B17C
:1034F00093F810330BB944F01004184BD5F80C2D89
:103500009A42A3F1080303D09A4218BF44F0100472
:10351000134991F95D13C1B19A4218D0032902D120
:10352000104B9A4201D144F040040F4876F028F83D
:1035300068B144F080040AE0182814BF012418245C
:10354000D2E71824D0E70124CEE79A42EDD144F027
:10355000010038BD386C0020385C00201479002050
:10356000384C0020D87800202C83002008B504486F
:1035700005F092FA00280CBF0120022008BD00BF10
:10358000382C0020F0B52DED028B8BB005460DF0E8
:10359000E3FE4FF48071D0F8047290ED828AD0F887
:1035A0000C6204461448FEF7D1FF30B9134BDFED2F
:1035B000147A93EDD47AA7EE678A2D7C7DF074FCA3
:1035C000D4F81823D4F81C33D4F8141308920993B0
:1035D00027221C23CDE900320390079103AA1E2164
:1035E000284604978DED058A069650F0C5FF0BB06E
:1035F000BDEC028BF0BD00BF382C0020384C002001
:1036000035FA8E3C2DE9F0432DED068B3F4ED6F872
:103610000C2D06F6DC439A428BB071D0A6F5805390
:1036200006F58059D3F84075D9EDE97A3B6890F8F2
:1036300010809B689FED369AB8EEE7AAD9EDEA7A3A
:103640003846F8EEE79A984707EE900AF8EEE77AE0
:10365000384667EE897A2AEE09AAFDEEE77A69EE26
:10366000899A17EE903A1DB23B681B69984707EE9E
:10367000900AF8EEE77AD9EDC98A67EE897AA6F55D
:103680008040FDEEE77A06F5546617EE903ADFEDDE
:10369000217AF4EEE78AF1EE10FA58BFF0EE678A6D
:1036A0001CB202F069FD3B68D6ED00AADFED1A7A84
:1036B0005B6908EE100A38466AEEA7AA9847FCEE46
:1036C000E88AB8EEC88A18EE903AB72228EE098A3E
:1036D000ADF824301A23CDE900323E2103AA40463A
:1036E0008DED03AACDED049A8DED058ACDED06AAE8
:1036F0008DED070AADF82050ADF8224050F03CFFA8
:103700000BB0BDEC068BBDE8F08300BF386C002029
:103710000AD7233C00FF7F470000C84208B5024893
:103720000AF096FA00B208BD382C002052F0E6B933
:1037300037B50D46134840F2EF2202F0F9FF2C781E
:1037400014F004040AD0696803220F4813F01AFE2B
:103750000C4803B0BDE8304002F06ABC01AA214623
:10376000284613F0B1FE0028F2D0DDED017A9FED7E
:10377000077A67EE877A2246FDEEE77A17EE901A0F
:10378000E3E700BF382C00203C8200200000C84244
:1037900010B5054C012384F8133352F0EFFB0023DE
:1037A00084F8133310BD00BF385C002055F08ABE8A
:1037B0002DE9F0412DED028B4FF0000882B0CDE9EC
:1037C00000281E4F9FED1E8A0C461546B0EE480A93
:1037D000B1F90220D7F8541B4FF47A73064656F01D
:1037E00059F90123CDE90053B4F90020D7F8581B4B
:1037F000B0EE480A30464FF47A7356F04BF9B4F9FC
:103800000420D7F85C1B9FED0F0A43463046CDE9F4
:10381000005856F03FF9CDE90058B4F90620D7F822
:10382000601BB0EE480A4FF47A73304656F032F916
:1038300002B0BDEC028BBDE8F08100BF384C002027
:103840000000FA4400007A4438B5C5780B46352D9F
:10385000044628BF3525352200211846A0F01AFA63
:103860002A4604F10C01BDE83840A0F0C9B90000B7
:1038700008B552F0CBF940F4A67040F0010008BD45
:1038800010B5044614F050F9204610BD10B50C4C8C
:10389000002384F83F3353F06BF8A4F58052A4F56D
:1038A0005873D2F80C2D9A4208D194F8B8332BB93A
:1038B00004F56D70BDE810402AF0E6BE10BD00BFF3
:1038C000387C002013B5124C94F8E610A4F168007F
:1038D0000BF0A0FA78B194F8E610A4F168000BF0B0
:1038E00007FD40B194F8E610A4F1680002B0BDE80D
:1038F00010400BF03FBD0DF02FFD01A90DF010FBA6
:1039000018B19DED010A02B010BD9FED020AFAE761
:10391000384C00200000000008B51248D0F80C2DEB
:1039200000F6D4439A4216D0B0F9243DABB900F565
:10393000805393F8C92282B990F8212D6AB993F87F
:10394000793363B9A0F5804005F0A6F800280CBFD4
:103950000320042008BD0220FCE70520FAE706202A
:10396000F8E700BF386C002010B5224B03F6DC42AC
:10397000D3F80C3D934290B0044639D0002302F6B0
:103980002810029313F0E8FC014618B91A4802AA5D
:1039900013F02EFD247C7DF087FA184BDDED027AC2
:1039A000D3F80C26D3F8103605930023F8EEE77A07
:1039B0009FED137A0793089309930A930B930C9343
:1039C0000D930E934FF6F853ADF83C300023CDE93C
:1039D000030267EE877A96228DF83E303323CDE9D5
:1039E0000032572103AA2046CDED067A50F0C4FDDF
:1039F00010B010BD386C00203C820020387C0020C4
:103A00000AD7233C10B552F0FBFA044688B90A489D
:103A1000A0F58052A0F55873D2F80C2D80F83F43E2
:103A20009A4206D190F8B8331BB900F56D702AF0B0
:103A30002BFE204610BD00BF387C002001207047BF
:103A400008B5034BD3F80C0D03685B68984708BDB5
:103A5000386C002030B587B005460DF07DFC04467B
:103A60002D7C7DF019FAD4F88422D4F8883204929F
:103A7000059300211023CD22CDE90032029003915D
:103A800002AA42F60C31284650F076FD07B030BD50
:103A900030B52DED028B89B005460DF05DFC00F5CB
:103AA0005A7393E8070002AC84E80700DDED020AD0
:103AB0009DED030A2D7CF1EE600AB1EE400A9DF007
:103AC000F3FE2046B0EE408A27F0B0FEDFED0B7A21
:103AD000049B079328EE278A0C230122CDE90032AC
:103AE000A82105AA28468DED058A8DED060A50F01D
:103AF00043FD09B0BDEC028B30BD00BFE02E654236
:103B0000422938B505461BD00AD824290CD04029B3
:103B100024D01B2922D02846BDE8384056F016B9DB
:103B2000432917D05329F5E70C214FF023FF044612
:103B300010B90024204638BD2846FFF7A9FFF9E751
:103B400010214FF017FF04460028F2D02846FFF757
:103B500081FFEFE7017C02487BF03AFA0124E9E7B4
:103B600004810020F0B52DED028B05468DB0164680
:103B7000B0EE408A0C46002930D0007C50F092FC18
:103B80000746287C51F092FB00F121039F4207D2A7
:103B9000287C0DB0BDEC028BBDE8F0404FF0D8BEE4
:103BA00063690893636A2269CDF82530236AA069A6
:103BB000E1680792CDF82930622221232768059019
:103BC000CDE900320691287C0397192303AAC2216C
:103BD0008DED048A8DF8246050F0CEFC0DB0BDEC64
:103BE000028BF0BD70B52E4CD4F80C2D04F6DC43DE
:103BF0009A42054652D0A4F50054B4F88633DE0745
:103C000008D504F6B87393ED000A012204F6B471E6
:103C1000FFF7A8FFB4F88633980708D52149022298
:103C200091ED450A284601F58871FFF79BFFB4F82E
:103C30008633590708D51B49032291EDA20A28466D
:103C400001F52171FFF78EFFB4F886331A0708D506
:103C50001449052291EDB90A284601F53871FFF79C
:103C600081FFB4F88633DB0618D50F4ED6F89033B3
:103C7000042B13D10DF070FB044606F2CC407BF010
:103C8000D7F994EDC70ADFED097A014620EE270A3D
:103C900028460622BDE87040FFF764BF70BD00BF34
:103CA000386C0020385C0020387C0020E02E654213
:103CB00070B504460E461DF09FF890F8F412B0233C
:103CC00003FB0101DC31204602F09EFE054698B15F
:103CD0003EB10DF041FB90F87C3243F0020380F8D6
:103CE0007C3204F5804304F59944D3F80C0D383444
:103CF000A04201D105F0ACFA284670BD73B5164656
:103D0000019104460DF028FB01990CF073FF054664
:103D100098B13EB10DF020FB90F87C3243F00203E5
:103D200080F87C3204F58043D3F80C0D04F59943F8
:103D30003833984201D105F08BFA284602B070BDA5
:103D400030B5054685B00C46D1E9040125F056F999
:103D500040B1684613F010FB6A462146284655F0EC
:103D600009FE08B9022067E0344840F24F32694644
:103D700002F0DEFCD4ED037AF4EE677AF1EE10FA8D
:103D800022D69FED2F7AF0EEE77AF4EEC77AF1EEC5
:103D900010FA54BF012200229DF80030294962F335
:103DA000410368468DF8003013F01EFC0028D9D17D
:103DB0002548694665F0B6FF40B94DF001FB052284
:103DC00016214DF059FACDE70022E5E7D4ED017A4E
:103DD000FDEEE77A17EE903ADB0706D41B4B03F6AD
:103DE000C842D3F80C3D934225D119491348022209
:103DF00009F03CFD9DF8001011F0040102D1684665
:103E000013F052FB0D48694602F04CFD94ED020A96
:103E1000B4EE400AF1EE10FA0BD6B5EEC00AF1EEA0
:103E200010FA06DD9DF800100948C1F3400106F0C4
:103E30005BFA002000E0042005B030BD382C0020E3
:103E4000000000342C820020884D0020386C0020B7
:103E50000079002010B52DED028BD1ED017A91EDA6
:103E6000008AFCEEE77A8AB0CDED037A9DF80C105B
:103E700005AA044655F068FDC8B1DFED0E7A059B32
:103E8000009368EE277A0022FDEEE77A114617EEDE
:103E9000903A06A813F090FA23682046D3F8CC3065
:103EA00006A9984700200AB0BDEC028B10BD022085
:103EB000F9E700BF0000C84237B5124DD5F80C0D28
:103EC00003681B6A0C46984740B9D5F80C2D05F5D8
:103ED0004A639A4202D0042003B030BDD4ED007A88
:103EE000D4ED020A94ED010A0748FCEEE77ACDED25
:103EF000017A9DF8041003F02DFB0028EBD0002080
:103F0000EAE700BF386C0020382C002008B5D1ED5E
:103F1000007A9FED087A0848F0EEE77AF4EEC77A67
:103F2000F1EE10FA54BF0121002104F069F80020DD
:103F300008BD00BF00000034382C002010B5D1EDC2
:103F4000007AFCEEE77A17EE903A9CB2012C02D090
:103F5000022C06D084B91148214661F049F90020AD
:103F600010BD0F4890F8C0345B0707D556F09CF998
:103F70000C4A05214FF0CCFA0420F1E790F9AC345B
:103F80001BB956F091F9084AF3E7A0F5A04007F0F5
:103F900055FC002814BF00200420E1E7E480002045
:103FA000387C00208C890B08A7890B0838B58B8BCF
:103FB000C02B05460C4631D8B12B0BD8112B00F085
:103FC0009680142B00F0968021462846BDE83840A4
:103FD00056F0AEBFB23B0E2BF6D801A151F823F03C
:103FE0004F400108C93F0108C93F0108C93F010806
:103FF000C93F0108C93F0108C93F0108C93F01087D
:1040000045400108C93F010869400108A540010871
:10401000C93F0108594001083B400108D42B08D092
:10402000B3F5967F49D0D02BCED1BDE83840FFF70D
:1040300085BFBDE83840FFF769BF2146BDE838407D
:10404000FFF77EBE2146BDE83840FFF703BF21469B
:10405000BDE83840FFF730BF94ED000A2848FEF76E
:1040600067F8E8B100201CE0264C94F8353DBBB160
:104070002549A1F510702AF005FC88B104F580539C
:10408000012283F8ED2304F54A610222A4F5804061
:1040900009F0ECFB0028E5D11C4B002283F8ED234E
:1040A000042038BD174C94F8353D002BF8D0164944
:1040B000A1F510702AF06AFBDFE7D1ED007A9FEDE1
:1040C000147AF0EEE77AF4EEC77AF1EE10FA14D52E
:1040D000D1ED017AF0EEE77AF4EEC77AF1EE10FA5C
:1040E0000BD50C490222064809F0C0FBBAE70A4981
:1040F0000222F8E709490222F5E70220D1E700BFD2
:10410000382C0020386C00202C820020387C0020C5
:1041100000000034D8780020F8780020F0780020E3
:1041200070B53F4B03F6C842D3F80C3D93428EB0B6
:104130000C4673D1CD78272D28BF272527220021B3
:1041400004A89FF0A7FD2A4604F10C0104A89FF0E3
:1041500057FD059B9DF836400093069B0193E44371
:10416000079B0293E4B2089B03938DF836407CF0E2
:104170009BFE14F0810F04F08705064601D1802DC7
:1041800011D1684626F0D0FADFED267A264B20EED4
:10419000270ADFED267AC3F8606320EE270ABDEE1A
:1041A000C00A83EDD50A14F0820F01D1802D11D100
:1041B000684626F0D3FADFED1B7A1B4B20EE270A68
:1041C000DFED1A7AC3F8646320EE270ABDEEC00A59
:1041D00083EDD60A14F0840F01D1802D11D16846E9
:1041E00026F0CCFADFED0F7A0F4B20EE270ADFED39
:1041F0000F7AC3F8686320EE270ABDEEC00A83ED8C
:10420000D70A63060AD5DDED0C7A9FED087A064BD6
:1042100067EE877AC3F87063C3EDDB7A0EB070BDCA
:10422000386C0020E02E6542387C00200000C84237
:1042300030B5214C91B0084602A9FFF705FBD4F830
:104240000C2D04F6C8439A4233D19DF83C30072B1D
:104250002FD104F58054DDED056AD4F808369FEDC2
:10426000177A07EE903AF8EEE77AE6EEC77AFDEEB7
:10427000E77A17EE903AC4F8083656F015F8D4F8F5
:10428000E025D4F8083652689FED0D7A9B1A07EEA8
:10429000903AF8EEE77A054667EE877A17EE900ACD
:1042A000FCF72AF9074ACDE90001062128464FF01C
:1042B0002FF911B030BD00BF386C00200000C8429B
:1042C0000AD7233CC0890B0810B51D4B03F6C84222
:1042D000D3F80C3D9342044696B008460FD108A986
:1042E000FFF7B2FA9DF8541003AA204655F02CFBB4
:1042F00038B955F0D9FF134A04214FF009F916B027
:1043000010BDBDF8503023F004039BB2002BF6D053
:10431000DDED0B7A9FED0C7A039B009367EE877AB5
:104320000022FDEEE77A114617EE903A04A813F04A
:1043300043F8236804A9D3F8CC3020469847DEE739
:10434000386C0020D4890B080000C84230B48D7A44
:104350004B7A43EA0523CD7A43EA0543562B0446BC
:104360000A4618D008D8522B0FD0542B10D0204614
:10437000114630BC55F0B8BF03F18073863B23F083
:104380007F43012BF3D830BC704730BCFFF7C8BE69
:1043900030BCFFF74DBF30BCFFF796BF0020704721
:1043A000C8207047012070470020704700207047E8
:1043B00090F89C308B4286BF283150F821000020B5
:1043C0007047000090F89C308B4286BF283150F82F
:1043D000210000207047000003207047014B93F834
:1043E000E6027047384C002070B504463D4807F09F
:1043F000EDFE18B1E36A43F40003E362394807F0C5
:10440000E5FE88B1462059F04BF8DFED377AB4EE7F
:10441000E70AF1EE10FA07D8236B43F40003236395
:10442000636B43F400036363E36A43F4F843E362BA
:104430002E4BD3F80C0D03685B689847013817289A
:1044400014D8DFE800F0333B0C3D3B3B3B3B1333E0
:104450003333333333131313131313131333244A24
:1044600092F8103353B392F8112352B3214B1D68C5
:10447000DDB1214E284696F84A1B46F0C5FDA0B195
:10448000E36A43F48073E36296F984331BB1236BD0
:1044900043F48073236396F84A1B284646F0ECFDEC
:1044A00018B1636B43F48073636370BDD4E90C236C
:1044B00042F4E04243F4E04322636363012300E0FB
:1044C0000023216B41F480622263626B42F48060BE
:1044D0006063002BCAD041F4406142F44062216322
:1044E0006263C3E7382C0020000000B4386C002061
:1044F000385C00204C850020384C002013B54FF468
:104500004470CDE9002113F007FB044628B1DDE932
:10451000002156F009F9024B2360204602B010BD7D
:10452000D08B0B0800207047002070470020704798
:104530000020704700F50D50083070470048704764
:1045400064B10B0800F58040D0F80C0D03685B687F
:104550001847000000F5804300F59940D3F80C3D62
:1045600020301B1A58425841704700009B2070476A
:1045700030B500F5A043D3EDE97ADFED286AB8EE57
:10458000E77AD3EDEA7AF8EEE77A85B0044627EECB
:10459000267A67EEA67A00F59550002301A910301F
:1045A00003938DED017ACDED027A04F57F650BF072
:1045B000B5F804F53E523432692128464BF022FF0B
:1045C00004F5445210326A2128464BF01BFF04F5D3
:1045D000405393F9522132B9D3ED527AF5EEC07AB5
:1045E000F1EE10FA06DD04F54A5204326B2128463A
:1045F0004BF008FF04F54A543034204677F0BAF9FE
:1046000028B104F130026D2128464BF0FBFE0CF07E
:10461000A3FE0CF0EBFB05B030BD00BF0AD7233C76
:1046200010B54FF48011044609F00EFB10B120467E
:10463000FFF79EFF4FF48001204609F005FB28B1EB
:1046400023F036FDBDE8104021F0BEBE10BD0000D5
:1046500030B500F5955591B000231035029302A9AD
:10466000002304460DF1070228468DF807300CF0B0
:104670005DFC03A928460BF0ADFC08B92D4B039354
:104680003022002104A89FF005FBA3238DF81030F1
:1046900095238DF811307CF00FFC04F5A042CDF885
:1046A0001300D2F8A433ADF81B3004F58053D2F8D0
:1046B000A823CDF817104620D3F8A814D3F8AC34AB
:1046C000ADF81D10ADF81F20ADF8213058F0E8FE10
:1046D00010EE103A1520CDF8233058F0E1FE10EE20
:1046E000103ACDF8273004F530539FED137AD3ED0F
:1046F0002B7A67EE877A284617EE903ACDF82B3062
:10470000029BCDF82F309DF807308DF83330039B96
:104710000D930CF011FE04F580433022D3F8483D90
:104720008DED0E0A04A904F57F600F934BF09AFFFC
:1047300011B030BD2292CA7F0000C84270B58EB061
:1047400035220446002168469FF0A4FAA3238DF881
:10475000003095238DF8013001238DF802307CF074
:10476000ABFB04F5A04504F54056D5F82433CDF84D
:104770000300D6F84005CDF80710CDF80B300368DC
:104780001B699847ADF80F00D6F8400503689B6891
:104790009847ADF811001D4801F0EEFCADF813008C
:1047A000D6F8400503685B69984710EE103AD6F8D2
:1047B0004005CDF8153003689B69984710EE103A14
:1047C000CDF8193004F5804303F5546135220968AA
:1047D000CDF81D10D5F80C16CDF82110D5F810160F
:1047E000CDF82510D5F80816CDF82910D5F8AC1756
:1047F000D3F8383DCDF82D1004F57F606946CDF82B
:1048000031304BF02FFF0EB070BD00BF382C0020B0
:1048100030B587B016220446002168469FF03AFA68
:10482000A3238DF8003095238DF8013002238DF8F5
:1048300002307CF041FB04F5A045CDF80300204692
:10484000CDF8071004F028F9D5F894330393144BEE
:104850008DF80B001B68D86A90F89C308DF81030EA
:104860000368DB69984795F879338DF812308DF835
:10487000110023F01DFC22F06BFDD5F890338DF86C
:1048800013008DF81430162295F87A338DF8153010
:10489000694604F57F604BF0E5FE07B030BD00BF10
:1048A000342C002010B58AB0272204460021684627
:1048B0009FF0F0F9A3238DF8003095238DF8013097
:1048C00009238DF802307CF0F7FACDF803000420BC
:1048D000CDF8071058F0E4FD10EE103A1320CDF893
:1048E0000B3058F0DDFD10EE103A4620CDF80F30B9
:1048F00058F0D6FD10EE103A1520CDF8133058F0D0
:10490000CFFD10EE103A0320CDF8173058F0D8FD47
:1049100010EE103A1A20CDF81B3058F0C1FD10EE01
:10492000103ACDF81F3004F59A43543327221B6800
:10493000CDF82330694604F57F604BF093FE0AB052
:1049400010BD000013B5044600F57F6001904BF0E8
:10495000C7F901984BF05EFA04F58053019893F97A
:10496000C4300BB14BF0FEFA204602B0BDE8104057
:10497000FFF798BF7047000010B500F5804304466C
:10498000D3F80C0D03685B68984704F500530146A3
:1049900093F8682204F57F604CF024F804F59550F4
:1049A00010300CF025FF04F59070BDE810401BF0AE
:1049B0008DBA00009FED020A002244F0FDBC00BF4A
:1049C0000AD7233C184B70B5044640F8043B56F018
:1049D000DDFF164E164B63605425601957F08CF9B5
:1049E00066513035B5F5557FF7D104F5557059F05E
:1049F0004BF904F27C75FF2384F88C3784F89437E4
:104A00000C49284645F0D6F80B4B1A6812B10B48F2
:104A10007CF01CFA1D6001232046094984F8C13747
:104A200045F0C8F8204670BDA838002098DB0B0878
:104A3000ACDB0B08543F0D08148F0020ACC80B08EA
:104A4000D0CB0B082DE9F04100F50B519AB00D22A7
:104A5000243104464AF002FA0022BE48BE4E272105
:104A600044F022FC0421002059F0E8F81321012031
:104A700059F0E4F84621022059F0E0F8152103200E
:104A800059F0DCF858F046FE45F09AFAB34A13881C
:104A900043F0040313804FF000080AAF00211022F6
:104AA00038469FF0F7F801238DF830303388ADF8A1
:104AB000283005A973680B93384644F0FDFAC8B155
:104AC0009DF91430002B15DD57F0E0F89DF8141017
:104AD000036801391B68C9B2984758B1051D2846BB
:104AE00044F088FA30B9B368ADF8183006A9284602
:104AF00045F00CFF08F10608B8F12A0F06F10C0684
:104B0000CCD1974800220DF10B0144F05BF806ADC3
:104B1000064620B344F06EFA08BB924B0FCB85E8F3
:104B20000F0004A9284644F0C7FA002840F0098184
:104B30004FF004088C4B0FCB87E80F0005A93846CF
:104B400044F0BAFA28B105A844F054FA08B148F084
:104B5000010803A930468DF80C8045F085FE834B93
:104B60000FCB85E80F0003A9284644F0A5FA0028DA
:104B700046D00998002204A944F024F806460028EB
:104B80003ED044F037FA0546002839D19DF80C3064
:104B9000013BDBB2032B96BF754A0346D35C8DF80D
:104BA00028303046394645F05FFE7248002205A99C
:104BB00044F008F8064665F0F7FA78B165F0F2FAC5
:104BC00090F8302090F8281090F84830114490F870
:104BD00040200A44D34214BF0125002586B1304647
:104BE0009DF90C8044F006FA50B91DB1B8F10005EA
:104BF00018BF0125394630468DF8285045F034FE5F
:104C000004F50C500022B7EE000A02211C3044F0DB
:104C1000D3FB012304F5FC510093574A00231831BC
:104C20008E2044F045FB94F9A4C9BCF1000F1AD1C1
:104C3000524E0FCE3D460FC50FCE0FC50FCE0FC53E
:104C400096E80F0085E80F0062460421384644F0DC
:104C50002BFB9FED4B0A4B4845F054FB4A48B7EEFF
:104C6000000A45F04FFB012504F50551474A009520
:104C70000023103140F2051044F01AFB04F50D50EA
:104C800002211030FFF796FE04F50A500321383058
:104C9000FFF790FE032104F50B50FFF78BFE04F5A0
:104CA0000D5003210C30FFF785FE04F50D50022155
:104CB0001430FFF77FFE04F50B5002210C30FFF794
:104CC00079FE04F50B5002211030FFF773FE04F556
:104CD0000B5002210830FFF76DFE04F5A9404C305F
:104CE0007AF00CFB2A4A1368D90709D429491560C0
:104CF00004F5035338330B6004F585530833CB6058
:104D000004F50E50234902220830012544F022FB0D
:104D1000214A0095002304F57F61FD2044F0C8FA84
:104D20001E4B1A68D20705D41D4A1D6004F58E5427
:104D3000183414601A48012144F028FB1AB0BDE869
:104D4000F08104A844F056F900283FF4F1AE4FF08A
:104D50000C08EFE60CC90B087CCB0B08248500205F
:104D6000D0C80B08A87E0B08B87E0B08C87E0B08BD
:104D700008C90B08DBC80B084CEF0B08D87E0B08E2
:104D800000000000E8C80B08F7C80B08883A0D08B7
:104D90002C2C002000220020F47E0C08302C002057
:104DA0001822002000207047002070470020704724
:104DB00000207047002070477047000000207047B7
:104DC0000020704784B001A880E80E0004B00020E5
:104DD00070470000002070477047000010207047A7
:104DE00000487047BCD70B0800487047CCD70B0869
:104DF0000020704770470000012070470120704775
:104E000000207047002343608360C36003614361F7
:104E1000002303767047000010B50446FFF7F2FF49
:104E20000023637610BD0000027E531CDBB2042B0E
:104E3000037600EB820288BF002382ED010A88BF5F
:104E40000376704710B50446FFF7EEFFD4ED017A04
:104E50009FED107A94ED020A637E77EE877A042B39
:104E600077EE807A94ED030A94BF0133052377EE41
:104E7000807A94ED040A637677EE807A637E94ED0F
:104E8000050A77EE807A00EE103AB8EEC00A87EE97
:104E9000800A10BD0000000003F03CBB02F04EBDD4
:104EA00002F0A0BF02F058BD01F070B901F020B8C7
:104EB00001F04AB901F0E0B9FDF73CBCFDF7E0B8FC
:104EC00070B51F4B036000F540530446D3F8D4047B
:104ED0001C4AC3F8182308B112F02AFE1A4B2360AB
:104EE00004F5805393F8342F42B9D3F8305F2DB1D5
:104EF000284620F0F1FA284612F016FE04F58D50EF
:104F00001C3073F099FD04F5865004305AF03AF9DC
:104F100004F6F44504F69446B54204D0183D2846FC
:104F20001FF030FFF8E7094BC4F8C83804F6C41086
:104F30004DF054FB04F513604DF050FB204670BD5E
:104F40005CBF0B08B0970C087C780C08D0410C08AB
:104F500038B54B4B044640F8043B5EF067FB04F168
:104F600010000FF07FFE04F1680049F02BF904F502
:104F700090701AF065FB04F58C600EF097FB04F25C
:104F8000845012F0D7FD04F6C80021F041FB04F56F
:104F900047605EF029F904F5546045F05BFF04F5C5
:104FA0007F604BF0A7FA04F58550083064F036F8BE
:104FB00004F5865004305AF0CDF804F5885011F00D
:104FC0008FFB04F58D501C3073F022FD04F58E50DC
:104FD000183049F0B9FC04F591500C305FF0D0FC6A
:104FE00004F580530025274A83F8505204F5925364
:104FF000103304F59350136040F0E2FD04F5955032
:10500000294610300AF0CEFC04F5C8506DF01EFEA3
:1050100004F5EE50043070F02DFD04F5F6501C3010
:1050200072F050FE04F5FA5073F086FA04F5FC5065
:10503000183009F0EFFD04F5035038306EF0E8FA4F
:1050400004F50550103064F085FB04F5085010306D
:1050500074F07AF804F5005304F50A5083F86852A6
:10506000094D74F093F92B6813B108487BF0EEFEFC
:105070002046074944F09EFD2C60204638BD00BF05
:105080007C780C087C8E002080850020D4D70B080B
:1050900084770C082DE9F04F2DED028B04469FB06C
:1050A000FFF756FFE44B236004F50E500830FFF77E
:1050B00089FC04F52D500C3004F5005775F0E6FC22
:1050C00004F50C532E33C7F8743B04F52E50062319
:1050D00087F8783B203059F04FFC04F5A9434C3356
:1050E000C7F8203C0E934FF40063C7F8243C5A23C2
:1050F00087F8A43C04F50A5807F6084304F59556CA
:1051000008F12808CD4ADFEDCE8AC7F81C8C10368E
:10511000C7F8186CB7EE008AC3F8602104F5375061
:10512000C84AC3F86821C3F8CC2183ED578AC3ED80
:10513000598A24304DF072FD04F5375030304DF06F
:105140006DFD4FF00009C04BC7F8003E87F8189E70
:1051500004F5385004F5305AFFF754FE0AF1080AF6
:10516000BA4BBB49C7F8003E87F8199E504644F039
:1051700021FDB84BC7F8203E07F562630022C7F84F
:10518000246EC7F828AE04F538555A63DA6304F57F
:105190003950012387F8643E2035383012F0ECF89E
:1051A00087F8889EAC49284644F004FD04F53A503F
:1051B00041460C3076F020F804F53F50414624304B
:1051C00075F07EFC04F54450414604F540573C30F0
:1051D00076F0DCFB2C22494607F538709EF05AFD2C
:1051E00004F54A509D49303004F54C5944F0E2FC36
:1051F00009F118099A4BC7F8183309F114007BF02C
:1052000007F804F54D5B04F54E530BF1100B3433E6
:1052100058460F9352F07EFB0F9B0BF1140B5B452E
:10522000F6D10723C7F8D8340023A7F8DC344FF4AD
:10523000CB7012F077FCC7F8D40404F5535020303B
:105240007AF0E6FF04F5545024307AF0E1FF854B04
:105250001A680AB9C3F80090834BC7F8183304F5ED
:1052600055504FF48051C7F8405504300FF0DAFD27
:1052700004F55750043042F001F804F5585004305A
:1052800045F0FAFB04F55850183066F0B1FC04F50F
:10529000984004F58045343003F0BCFF734BC5F8EB
:1052A000343C04F598403C3003F0B4FF704BC5F833
:1052B0003C3C04F59840443003F0ACFF6D4BC5F81E
:1052C000443C04F598404C3003F0A4FF6A4BC5F809
:1052D0004C3C05F54663002204F59840DA609A607C
:1052E0005A6083ED008A743003F094FF634BC5F875
:1052F000743C04F598407C3003F08CFF604BC5F89B
:105300007C3C04F59940043003F084FF5D4BC5F804
:10531000843C04F59940183003F07CFF5A4BC5F8E3
:10532000983C04F59940203003F074FF574BC5F8C2
:10533000A03C04F59940383003F06CFF544BC5F89D
:10534000B83C04F59940403003F064FF514BC5F878
:10535000C03C04F59940483004F5994903F05AFFE0
:1053600009F154094C4BC5F8C83C484603F052FFBC
:105370004A4BC5F8D43C04F599405C3003F04AFF31
:10538000474BC5F8DC3C04F59940643005F0CAFC95
:10539000FE2385F8183D052385F8343D4FF0FF3B8B
:1053A000404BC5F80C9DC5F8109DC5F83CBD119348
:1053B00005F654553C4B85ED008A04F59A4022468B
:1053C0004FF4007100935830364B109404F5A0450B
:1053D0000EF030FF0023C5E9D533C5E9D733C5E961
:1053E000D9330323C5F89033304BC5F8FCB2C5E977
:1053F000F5342F4BC5EDC68AC5E9F73404F5A7404F
:105400002C4BC5F8E43385EDEB8AC5F8D0437830F2
:1054100011F0B2FF04F5A840143011F0ADFF04F50F
:10542000A84004F5A749303011F0A6FF09F134096E
:10543000214BC5F8443441E05CBF0B08000080BF3D
:105440000000B4420000B4C240D80B0850D80B088A
:1054500014790D0888760D0830760D08CC700D088B
:10546000B0970C08C8880020AC8C0B08BCE10B0876
:10547000A0E50B0888E70B0810E00B08C4E20B0856
:1054800048E30B0830E20B0840E10B08C0E00B08D2
:1054900028E50B0838E40B08C4E30B0878D80B08A0
:1054A000B4E40B08994E010884890B089D4E01084D
:1054B000A14E0108A54E01080000FFFFA5F848B461
:1054C00009F1980011F058FF6E4B6F49C5F8A8B468
:1054D0004846C3F8009044F06DFB4FF6FF73A5F803
:1054E000F03304F5A940694B6949A5F80CB42C3098
:1054F000186044F05FFB674BD7F840251294CDE964
:105500001334654BCDE91534644BCDE91734644B46
:10551000CDE91934634BCDE91B34634B1D931EA9B0
:1055200011E903000CAB83E80300DDE91A010AABC3
:1055300083E80300DDE9180108AB83E80300DDE937
:10554000160106AB83E80300DDE9140104AB83E830
:105550000300DDE9120102AB83E80300CDE9002876
:105560004946324653460E9804F5AA4879F0CEFCD7
:1055700008F158084D4BC5F8583508F13C0011F0BA
:10558000FBFE4B49404644F015FB4A4B1F6817B1E0
:1055900049487BF05BFCC3F8008006F51B76474B5F
:1055A000C5F8583504F5AB40C5F8E06585F85C757D
:1055B00085F8617585F88575643011F0DDFE04F5B8
:1055C000AB40743011F0D8FE04F5AC40043011F05B
:1055D000D3FE1022394605F214609EF05BFB04F501
:1055E000AD4604F5AC407436703059F001FF3046DA
:1055F00073F086FF324B3349C5F8F436304644F039
:10560000D9FA314A3149116004F5AE432C331426DE
:10561000B8B206FB00120137127C002AF8D12C4ADE
:1056200010802C4A16680EB12B48B2E704F5AE4044
:105630003030136073F04EFF284BC5F83037284BDD
:10564000C5F84037642385F84437264BC5F87837CA
:1056500004F5AE40244BC5F87C372449403044F073
:10566000A9FA234BC5F8403720460123C5F8A067A7
:1056700085F8A86785F83C331FB0BDEC028BBDE808
:10568000F08F00BF648400202C4F0C08848E002013
:10569000E8AD0C08A94E0108AD4E0108B14E010855
:1056A000B54E0108B94E0108BD4E010828D80B08B7
:1056B000AC740D0834960020E8D70B08D0DB0B083B
:1056C00040830B0818830B083C85002080CD0B0815
:1056D00038850020F084002004D80B0880830B0854
:1056E00060D80B0898EB0B08F0EB0B080C9F0C082C
:1056F00070ED0B0810B57BF001F8064C064B1860F6
:105700002046FFF7C7FC2046044A0549BDE8104083
:105710009BF052BD382C0020342C002024E20020C5
:10572000C14E01080069C0F3401070470F299DBFAA
:10573000302303FB0100503000207047014B93F9E8
:105740002D037047384C0020014BD3F8600B704795
:10575000384C002008B503689B68984730B9044B63
:1057600093F8260DB0FA80F0400908BD0020FCE750
:10577000386C002008B5044806F0BCFA10B9034B99
:1057800093F8200D08BD00BF382C0020386C002095
:10579000022A10B50C4605D1BDE810400948352253
:1057A00008F040B9084BD3F80C0D03685B689847C4
:1057B000A04205D156F06AFABDE8104056F0F0B9A3
:1057C00010BD00BF382C0020386C0020012910B516
:1057D0000C4614D0022907D0D1B90E4BC3F8A0173C
:1057E00054F062FD0C4A05E00A4BC3F8A01754F0D0
:1057F0005BFD0A4ABDE8104006214DF089BE54F019
:1058000053FD074A06214DF083FE024BC3F8A04723
:1058100010BD00BF387C00208FD90B0864D90B085D
:1058200078D90B08012902D0022900D011B9024B06
:10583000C3F8A417704700BF387C0020622910B459
:1058400000F3888047291ADC402900F0958008DCA5
:10585000162951DC032904DD4F4B01248C402340E1
:1058600053B95DF8044B57F0E3B8A1F19604012356
:10587000A3404A4C2342F4D05DF8044B7047A1F199
:1058800048031A2BEDD801A454F823F079580108E5
:1058900063580108635801086358010863580108F8
:1058A00079580108635801086358010863580108D2
:1058B00063580108635801086358010863580108D8
:1058C000635801086F5901086F5901086F590108A1
:1058D00079580108635801086F590108795801087F
:1058E000635801086358010879580108795801087C
:1058F0006358010879580108A1F12703112BB0D88A
:10590000112BAED801A454F823F000BF7958010838
:105910006358010863580108635801087958010861
:105920006358010863580108635801086358010867
:105930006358010863580108635801087958010841
:10594000795801086358010863580108795801081B
:1059500079580108B02904DC952986DC6B2980D1AF
:105960008AE7A1F1D003022B3FF67BAF84E75DF815
:10597000044B002357F02EB8094B012283F89C27D3
:10598000A3F54053D3F85C0B00283FF475AF5DF8E6
:10599000044B642156F0C0B910004100A1008004FE
:1059A000387C002038B50B46622B0446114600F3C4
:1059B0009580472B13DC382B7ADC262B4CDC102B04
:1059C00000F0B680162B00F00781042B00F0C78092
:1059D0000A4620461946BDE8384056F067BDA3F197
:1059E00048021A2AF4D801A050F822F0395B0108C5
:1059F000D1590108D1590108D1590108D1590108DB
:105A0000635B0108D1590108D1590108D159010836
:105A1000D1590108D1590108D1590108D1590108BA
:105A2000D15901086F5B0108AF5B0108D15901082A
:105A3000D15B0108D1590108B75B0108695B010816
:105A4000D1590108D15901081F5B0108E55B010824
:105A5000D1590108475B0108A3F12702112AB7D8E1
:105A600001A050F822F000BF1F5B0108D1590108C6
:105A7000D1590108D1590108235B0108D159010806
:105A8000D1590108D1590108D1590108D15901084A
:105A9000D1590108D1590108595B0108415B01083E
:105AA000D1590108D1590108535B01084D5B010828
:105AB000402B8DD1931E5942644C594184F89B1759
:105AC00054F0F2FB624A94F89B17624B002908BF1E
:105AD0001346614A06214DF01BFD20E09B2B00F090
:105AE0008E8007DC6B2B00F09480962B7FF470AFD8
:105AF00007211EE0AD2B7AD00CDC9D2B7FF468AF24
:105B00000124002A00F08180022A5BD14F4B83F8E8
:105B10009A4757E0A3F1D002022A3FF659AF012479
:105B200050E08A1E4D4B5142514183F8191DF6E752
:105B30000A21FFF72DFEF2E70A4601212046F8E789
:105B40000A460421FAE70A460321F7E70A460C2130
:105B5000F4E70A460F21F1E70A460021EEE70B21A0
:105B6000E7E70A460D21E9E70A460521E6E7374C53
:105B7000D1B102290DD1012384F89837A4F58053BF
:105B8000D3F80C0D03685B6A984710B1344800F0F5
:105B90008DF954F089FB334A94F89817324B002959
:105BA00008BF1346314A95E784F89817E6E7204680
:105BB000FFF70CFEB3E7012431B1022902D12C4BCF
:105BC00083F8E440204638BD294B83F8E410F9E718
:105BD0002046FFF727FEA2E7022AA0D1204805F0C1
:105BE0002DFE9CE756F052F855F0DAFF97E7022AAF
:105BF00095D19FED200A1A48FCF79AFA8FE7022AFE
:105C00008DD1174805F084FF89E7104B83F89A2758
:105C1000D8E7022A14D1114DD5F80C0D0368DB6BBF
:105C20009847044628B10121A5F5804002F0E8F923
:105C3000C8E754F039FB104A04214DF069FC6EE7C7
:105C40000748002102F0DCF969E700BF387C00203A
:105C5000A4D90B08EFC10B08ACD90B08386C002095
:105C6000382C002048AD0B0808E60B08BCD90B08FF
:105C7000384C002000000000CFD90B0810B5084CAC
:105C8000D4F80C0D03689B6B984738B9D4F80C0D09
:105C900004F6DC44001B18BF012010BD0220FCE705
:105CA000386C002008B50221032057F011FF0221B3
:105CB000084657F00DFF0121042057F009FF02218B
:105CC000152057F005FF1320022157F001FF12485D
:105CD00006F07CFAA8B10021462057F0F9FE002119
:105CE000492057F0F5FE00214A2057F0F1FE00212F
:105CF000012057F0EDFE0021BDE80840084657F0AE
:105D0000E7BE0121462057F0E3FE0121492057F06C
:105D1000DFFE0121E8E700BF382C002002490348DC
:105D2000052207F0A3BD00BFD8780020382C002042
:105D300038B5304B01241C7090F90A302B2B0CD154
:105D40002D4879F0D9FA2D4807F070FBBDE83840AE
:105D50002B4801220921FBF70BBE284D9FED290A94
:105D6000D5ED460A6421032057F07CFCD5ED460AA8
:105D70009FED240A6421022057F074FC9FED220A53
:105D8000032057F079FB9FED200A022057F074FBA7
:105D90009FED1E0A042057F06FFB9FED1C0A152093
:105DA00057F06AFB13209FED190A57F065FB284650
:105DB00006F00CFAA0B10021462057F0B7FE0021F2
:105DC000492057F0B3FE00214A2057F0AFFE0021D2
:105DD000012057F0ABFE0021084657F0A7FEB2E7BE
:105DE0002146462057F0A2FE2146492057F09EFE4C
:105DF0002146E9E72889002004810020382C002072
:105E00002C830020000000000000C84200A08C4548
:105E100000F58040D0F80C0D03681B6C184700009B
:105E200000F5005393EDD37A00F5A040B5EEC07AAB
:105E3000F1EE10FA5DBFD0F8E035DFED086AD3ED82
:105E4000017AD0F8F8055FBFF8EEE77AE7EE267A38
:105E5000FDEEE77A17EE900A704700BF0000C842D7
:105E600000F5005090F8840328B141F00101084288
:105E700014BF01200020704708B50346FFF7F0FF6C
:105E800050B103F5005292F87C1BC90704D502F605
:105E9000983292ED000A08BD03F5AC4090ED090A76
:105EA000F9E700000022FFF7E7BF000000F5A0407F
:105EB000D0F8F835C0F814360023C0F8183670470B
:105EC00000F5A0404A68C0F814260B78DB0741BFF4
:105ED000D0F8E0355B689B18C0F8143670470000B6
:105EE00000F5A040D0F814361944C0F814167047D5
:105EF00010B54B68516800F5A0448B42D8BF0A46E4
:105F0000D4F81406CCBF1A46194622F0ADFEC4F8E8
:105F1000140610BD10B50446414863F077FD10F03B
:105F2000080217BF3F4BDFED407A93ED577AD3ED70
:105F3000597A1FBF77EE877A9FED3C7A012267EE90
:105F4000877A10F0010317BF364B9FED377AD3EDF8
:105F5000596A93ED567A1CBF37EE667ADFED336AE5
:105F600004F5005118BF27EE267AD1EDD56AF5EE7B
:105F7000C06A18BF0123F1EE10FA4BDD294A9FEDEC
:105F80002B6AD2EDD56A66EE866AF4EE676AF1EEA8
:105F900010FA58BFF0EE667AF3B11A4604F5A04342
:105FA000D3F8E015D1ED016AD3F81416F8EEE66ADD
:105FB00076EE876A07EE101AB8EEC77AF4EEC76A73
:105FC000F1EE10FAD8BFB0EE667ABDEEC77A17EEE2
:105FD000101AC3F814160AB304F5A044D4F8E03537
:105FE00093ED017AD4F81436B8EEC77A77EE277AB3
:105FF00007EE103AB8EEC77AF4EEC77AF1EE10FA6F
:1060000058BFB0EE677ABDEEC77A17EE103AC4F803
:10601000143603E0002ABFD1002BBFD110BD00BF52
:10602000884D0020384C0020000000000000C842CD
:1060300000F5A0400023C0F81836704713B50023C0
:106040000446104601AA019311F052FA034648B1E2
:10605000DDED017A9FED177A67EE877AFDEEE77A3C
:1060600017EE903A04F5A041D1F89023C1F8183604
:10607000042A1DD004F50054B4F97E23002A14DD4F
:1060800083EAE370A0EBE37007EE900A9FED0A7AD3
:10609000F8EEE77A67EE877A07EE102AB8EEC77A4D
:1060A000F4EEC77AF1EE10FA02D50023C1F81836E3
:1060B00002B010BD0000C8420AD7233C0B78D1EDD6
:1060C000017A00F5A04013F0010F1CBFD0F8E035B5
:1060D00093ED017AF8EEE77A18BFB8EEC77A00F5CB
:1060E000BF6318BF77EE877A93ED007AB8EEC77A70
:1060F000B4EEE77AF1EE10FACCBF01200020704731
:106100007047000000F5005300F58042B3F93633C4
:10611000D2F80C2D00EE103A00F5994320339A4244
:10612000B8EEC00A0ED100F5A040D0F89033042B91
:1061300002D090F83D332BB100F2CC40D0ED007A84
:1061400030EE270A70470000014608B501F5A0416E
:10615000FFF7D8FF01F5BF63D3ED007A9FED057A15
:10616000F8EEE77AE0EE477AFDEEE77A17EE900A6E
:1061700008BD00BF0000C84210B5044604F5A044A5
:10618000FFF7E2FFD4F81436181A10BD70B50446B4
:106190002DED028B04F5A045FFF792FEDFED340AEA
:1061A00040F24310B7EE001A0E4622F0BDFCD5F8BF
:1061B0001826534207EE903AF8EEE77AD5F81436EF
:1061C00067EE807AB0EE408AFDEEE77A17EE901A1D
:1061D0001944C5F8141604F50053D3EDE06AF5EE42
:1061E000C06AF1EE10FA3FDD002A3DDD2046FFF7E0
:1061F000C3FF9FED207A07EE900A66EE876AF8EEFD
:10620000E77AF4EEE67AF1EE10FA2DD53146204623
:10621000FFF756FE04F5AB41324674312046FFF7D6
:106220000DFFD5F81826534207EE903AF8EEE77ABC
:10623000D5F8143667EE887AB5EEC08AFDEEE77AB7
:10624000F1EE10FA17EE901A1944C5F814160BDD8A
:1062500007EE902AF8EEE77A87EE887ABDEEC77AE5
:1062600017EE103AC5F81836BDEC028B70BD00BFB2
:10627000000000000000C8C2014608B5FFF742FF59
:1062800001F5AC40D0ED097A37EEC00ADFED047AB3
:1062900020EE270AFDEEC07A17EE900A08BD00BF77
:1062A0000000C8422DE9F04100F5AB4800F5AC45CF
:1062B00008F17408043504462946404611F08CFB69
:1062C00004F5AB4604F5A04764362A4631464046FD
:1062D00087EDC90A11F0B6FADFED220A87EDCA0A86
:1062E000B7EE001A762022F01FFC04F5305383ED40
:1062F000730A2046FBF7C4FE04F58043D3F80C0D67
:1063000003685B6898470B280BD006D80A280FD083
:106310000023C7F81836BDE8F0810E38C0B2012856
:10632000F6D829462046FFF7C9FE0028F0D011E034
:1063300029462046FFF7C2FE30B90B484FF4804192
:10634000FCF704F90028E3D12046FFF795FFB0F5EC
:10635000FA6FE6DD2A4631462046BDE8F041FFF7F8
:106360006DBE00BF00000000382C002010B500F505
:10637000A04300F58054D3F8082693F804369FED27
:10638000146A13F0010F07EE902A08BFD4F82035E5
:10639000F8EEE76A08BF07EE903A66EE866A04BF39
:1063A000F8EEE77AE7EEC66AFFF7CEFE04F5A463DF
:1063B00093ED000A07EE900AB8EEC00AF8EEE77A0D
:1063C00026EE400AA7EE860A30EE660A10BD00BF30
:1063D0000AD7233C10B504467AF066FD04F5005355
:1063E000D3F8902B801A41F2883290420FD80221C4
:1063F0002046FFF735FD50B104F5A044D4F89023B2
:10640000042A04D103F6843393ED000A10BD9FEDF6
:10641000010AFBE70000000008B52DED028B00F536
:10642000A0430146D3F8E025D3F814365268DFEDD7
:106430000D8A9B1A08EE103AFFF764FEB8EEC88A80
:106440000846A0EE288AFFF7C5FFBDEEC88AB8EE61
:10645000C88AA0EE288AFDEEC87ABDEC028B17EE42
:10646000900A08BD0000C842F0B52DED048B00F580
:10647000005489B000F5546694F84A1B0391054610
:10648000304644F0B7FD03990746304644F0C4FD5A
:10649000042F0399B0EE408A20D1002305A88DED8A
:1064A000050A0693079324F0ADFE05F5AE5005A945
:1064B000103022F0C9FDDFED877A8DED050AB4EECC
:1064C000E71AF1EE10FACDED060A8DED071A05DB9D
:1064D00005F5805393F82C35DF070CD494F87C3BFA
:1064E000002262F3000384F8942B84F87C3B09B00B
:1064F000BDEC048BF0BD94F87C3B98075FBF43F084
:10650000020384F87C3B05F52E5383ED008A04F6E4
:10651000983383ED001A94F8943B092B79D804F64C
:106520009C33D3ED000A9FED6C9AB0EE480A22F03E
:10653000E9F900BB05F52E5394F84A1BD3ED008A08
:10654000304644F087FD07EE900A9FED647AF8EE3E
:10655000E77A78EEC88A67EE877AF0EEE88A67EE27
:10656000897AF4EEE78AF1EE10FAC2BF94F8943B10
:10657000013384F8943B04F69C3394F84A1BD3ED22
:10658000008A304644F066FD07EE900AF8EEE77A9E
:106590009FED537A67EE897A78EEC88A67EE877A3C
:1065A000F0EEE88AF4EEE78AF1EE10FA02DD00235D
:1065B00084F8943B04F69C3383ED008A94F87C3B8A
:1065C000DA0794D52846FFF7D1FE04F6983696ED03
:1065D000008A30EE488A7AF067FCD4F8902B41F2BA
:1065E0008831821A8A42034604F6843204F68831DE
:1065F00036D982ED008A284681ED008A0221FFF714
:106600002FFC18B105F5A945AA6D6A65C4F8903B41
:106610006DE794F87C3B43F00103590784F87C3B19
:10662000C8D405F5A042D2F89023042AC2D1022191
:106630002846FFF715FC0028BCD043F0040311EEF8
:10664000100A84F87C3BF9F757FF05F54C561836CD
:10665000CDE90001234A062130464CF059FFA9E755
:106660009FED1F0A92ED007ADFED1F7A28EE008A77
:10667000A7EE278A82ED008AC4F8900BD1ED007A4C
:1066800038EE678AF3EE0E7AB0EEC88AB4EEE78A87
:10669000F1EE10FA7FF72BAF94F87C3B5B070CD53B
:1066A0003068F9F729FF05F54C541834CDE900019D
:1066B0000E4A062120464CF02BFF05F52D502422D2
:1066C00000213C3009B0BDEC048BBDE8F0409DF0EA
:1066D000E1BA00BF000000340AD7233CCDCC4C3DCA
:1066E000CDCC4C3EE0DB0B08CDCC4C3FFDDB0B08AA
:1066F00038B52DED028B0D460446FFF737FE00231B
:1067000020462B70B0EE408AFFF764FE022120463F
:1067100038EE400AFFF7A4FB28B104F5005494F8C2
:106720007C0B00F00100BDEC028B287038BD00002E
:1067300070B50B7803F00503042B05460C4616468E
:1067400015D105F5A04549F07FF9B2B24FF480119B
:1067500049F032F9D5F8E025636852689B1A13F5C1
:10676000FA7FC8BF6360237843F00103237070BDD4
:10677000F8B500F5805300F5A047D3F82065D7F8A9
:106780004C53B542044619D00E4A1268D26A92F8A8
:106790009C209AB100F5AC41751B25220431FFF70E
:1067A000C7FF07EE905AB8EEE70ADFED077A04F567
:1067B000305020EE270A083078F030F9C7F84C63E3
:1067C000F8BD00BF342C00200AD7233CF8B500F5F3
:1067D000A044054694F83FC30F4604F2E456BCF1CA
:1067E000000F53D004F204630FCB86E80F0001239F
:1067F00084F8403397E80F0004F2046686E80F003F
:10680000D4F80C3605F5AC46043693B9D4F81036F6
:106810007BB9D4F8FC35D4F80826C4F80C36D4F883
:106820000036C4F8103622B9D4F8F815304610F006
:10683000A9FD314628222846FFF77AFF94F804166E
:1068400011F0040102D1304610F02EFE05F5AB41E7
:1068500005F5AB4032466431743011F029F838B197
:1068600004F2E45604F2F45494E80F0086E80F00B2
:10687000284604F045FB2846FFF714FD284604F09F
:106880006FFE2846BDE8F840FFF7C2BA04F2F453A1
:106890000FCB86E80F00012384F83F3384F840C310
:1068A000A8E70000F8B500F500530446B3F9DE325E
:1068B000002B0E4633DB0B7813F0020F14BF4FF0A2
:1068C000FF33012304F5A04505F2E45785F8BC35F4
:1068D00005F2F4530FCB87E80F0096E80F0005F29E
:1068E000046787E80F0004F5AC41572204312046C5
:1068F000FFF71EFF2046FFF7D9FA2046FFF7D2FC2C
:10690000204604F02DFE002385F84033C5F8C0353D
:1069100085F845332046BDE8F84004F0F1BA4FF061
:10692000FF33CFE72DE9F043364B1B6885B00546B2
:10693000D86AFAF7FFFD002861D105F5005393F9F5
:10694000F83A5A1C54D0002B05F58C6711DD95F8E8
:106950007124242107EE903A01FB027292ED0B7A2A
:10696000F8EEE77AB0EEC77AB4EEE77AF1EE10FA15
:106970003EDC05F5805305F5955693F82C3513F05C
:10698000010406F1100629D0C3F340089B0732D456
:1069900095F8141495F858444FF0B00909FB0151CB
:1069A00091F8F1314CBB022B18D9684610F0E4FC89
:1069B000694630460AF030FA044678B195F8143446
:1069C00009FB03534246D3F80012684610F0DAFC84
:1069D0000AF0C2FC69460AF00DF9044638460CF08C
:1069E00039FF30460AF024F82846FBF781FD20469F
:1069F00005B0BDE8F0830024F0E74446EEE7002050
:106A0000F6E700BF342C002038B50C4B1B68054658
:106A1000D86A0C46FAF78EFD10B10024204638BD26
:106A20000AF09AFC21460AF0E5F804460028F4D062
:106A300005F5A740343025F0D3F9EFE7342C0020DA
:106A4000F0B500F5A045002385F83F3385F84033C5
:106A500005F2F453044600EE101A0FCB87B005F28E
:106A6000E45686E80F0002AE04F5AB42B8EEC00A69
:106A700030461749743244F007F996E80F0005F2E2
:106A8000046787E80F0004F5AC4140F25712043167
:106A900020460191FFF74CFE01992046FFF730FB9D
:106AA00001992046FFF70CFA04F500532046B3F98C
:106AB000DE32002BB4BF4FF0FF33012385F8BC3525
:106AC000FFF7F0FB204607B0BDE8F04004F048BDFA
:106AD0003C62002010B50349044644F0D5F8204636
:106AE00010BD00BF3C620020F8B500F5A04404F2E0
:106AF000F45305460E460FCB04F2E45787E80F0027
:106B000006F108012846FFF761FEB388D4F808268D
:106B100003EB830303EB83039B001BB2002BD8BF63
:106B20004FF4C873A4F83A33D4F8E0355968521AD0
:106B3000C4F80C239A680A32C4F80C26DB680A33BE
:106B4000C4F810360023C4F8203384F83C3384F8AA
:106B50005033C4F810330023C4F804334FF0FF332C
:106B6000C4F8FC3295F8712405F58C63242101FBEF
:106B70000233DB6AC4F83433F8BD000070B50E464A
:106B800008310546FFF722FEB38805F5A04443B35C
:106B9000642213FB02F3C4F80C33B4F93A33002B2C
:106BA000D8BF4FF47A7305F52D50D8BFA4F83A3307
:106BB000242200213C309DF06DF804F2246305F599
:106BC000A94093ED000A31464C3078F095FAD4F89C
:106BD0009033072B0CD128460421BDE87040FBF709
:106BE000FFB9D4F80C33002BD7DC40F6B833D2E72A
:106BF00070BD00000B7A00F5A04013F0020F14BF27
:106C00004FF0FF33012380F8BC3570477FB501F1A9
:106C1000080305460E460FCB6C4684E80F0005F5C9
:106C2000AB417431204610F0DFFC21462846FFF7C7
:106C3000CDFD31462846FFF7DDFF04B070BD0000F2
:106C40007FB501F1080304460E460FCB6D4685E87B
:106C50000F0004F5AB417431284610F0C5FC2946FD
:106C60002046FFF7B3FD20463146FFF7C3FF3379D7
:106C700007EE903A337E9B0748BF9FED0C7AF8EE03
:106C8000677A04F5A04448BF67EE877A9FED087ADB
:106C900067EE877AFCEEE77A17EE903AC4F8B435DF
:106CA0000123C4F8D43504B070BD00BF0000803BA0
:106CB00000A00C477FB501F1080304460E460FCB38
:106CC0006D4685E80F0004F5AB417431284610F09D
:106CD0008BFC29462046FFF779FD20463146FFF719
:106CE00089FFB38804F5A0444FF47A725343C4F883
:106CF000CC350123C4F8D43504B070BD2DE9F3417F
:106D000000F5AC450446043500F5AB400E46643052
:106D1000294610F029FC04F5A047C0B94FF0FF3315
:106D2000C7F8FC3206F10808404610F055FB03286E
:106D300002463AD1F168284610F024FBB388C7F820
:106D4000D435204602B0BDE8F041FFF771B91AF022
:106D500053F8FAF7D5FE012812D94FF0FF33C7F8E0
:106D6000FC321AF049F890F8F432DFED150AB0223F
:106D700002FB030090ED3C0A284610F0A3FED1E789
:106D800004F58058D8F8B00421F0A2FE08F5966307
:106D9000C7F8FC02D3ED007A9FED0A0ADFED080A7E
:106DA000F8EEE77A27EE800AE6E701AA00214046DE
:106DB00010F01EFB0028C1D001990022BBE700BFE4
:106DC00000007A440AD7233C7FB501F1080304464A
:106DD0000E460FCB6D4685E80F0004F5AB417431CC
:106DE000284610F001FC29462046FFF7EFFC20461C
:106DF0003146FFF7FFFE04F5A0440023C4F8D43564
:106E000004B070BD37B504460D467AF04DF8E06029
:106E1000D5ED027AF5EEC07AF1EE10FA15DD9FEDB0
:106E2000127A67EE877AFCEEE77AC4ED027A53F0C5
:106E30003BFAA2684FF47A73B2FBF3F30B4A0621D4
:106E400003B0BDE830404CF063BB62F02DFC002382
:106E5000009395F90D2095F90E3095F90C1062F01C
:106E6000BFFBA060E3E700BF00007A4420DC0B0812
:106E70002DE9F0412DED028B84B004460AF06CFA46
:106E800009F0BCFB04F5805304F5A04593F8A8373E
:106E90000BB9002875D0D5F8FC32013371D1D5F883
:106EA0002033002B49D079F0FFFFD5F82033C01AEA
:106EB000B0F5FA6F65D394F81424DFED5E7A9FED98
:106EC0005E8A4FF0B00808FB024292ED840A20EE81
:106ED000270A21F015FED5EDC17A30EE670A21F0C0
:106EE0000FFEDFED567A20EE080A04F54C5720EE2F
:106EF000270A21F0ADFDFDEEC07A183717EE906A33
:106F0000C5EDBF7AD5EDC17A67EE887A17EE900AA3
:106F1000F9F7F2FACDE9020194F8143408FB0343BF
:106F2000D3F80C02F9F7E8FA454ACDE900013346F7
:106F3000062138464CF0ECFA23E004F59070FAF79D
:106F4000DFFD02281DD994F81434B02202FB03435C
:106F500093ED837AF1EE047AB4EEE77AF1EE10FA6B
:106F60000FDD384B1B68D86A0368DB699847012836
:106F700003D079F099FFC5F82003D5F82033002B12
:106F800091D104F54053D5F8FC12D3F840054A1CC2
:106F9000036846D01B6B98472B4807F069FA20B16D
:106FA00004F5A740343027F09DF92046FFF764F937
:106FB000D5F80C338342064636DA07EE906A9FED29
:106FC000237AF8EEE77A04F54C5467EE877A1834A2
:106FD00017EE900AF9F790FA1D4ACDE90001204614
:106FE00006214CF095FA01244FF0FF33C5F8FC322E
:106FF00085F83C4305F2F4530FCB05F2E45605F255
:10700000046786E80F0087E80F00124862F0C8FCAA
:10701000002385F83F33204604B0BDEC028BBDE869
:10702000F0815B6B9847B7E7074807F001FA002843
:10703000C3D1F1E735FA8E3CE02E65420000C8422C
:1070400030DC0B08342C0020382C00200AD7233CDD
:1070500054DC0B08884D00202DE9F04700F5A046D0
:107060002DED028B4FF0FF33C6F8FC3206F20463BD
:107070008C4607460FCBBCF804509CF8049088B0AF
:1070800004AC2D0A84E80F0020D007F5AB4808F1C6
:1070900064082146404610F09FFC21464046B0EE71
:1070A000408A10F069FBDFED567AB4EEE78AF1EE24
:1070B00010FA0BDBEBB200EE903ADFED527AF8EE0D
:1070C000600A20EE270A204610F0FCFC07F5405A23
:1070D00096F84023DAF840059FED4B0A036807F560
:1070E000AB489B6A08F1740822B307F5AB4122460E
:1070F0006431984707F50052B2F90E33002B1CDDBE
:1071000007EE903A96EDC97AF8EEE77AB4EEE77AB0
:10711000F1EE10FA11DD07F5AB412246643140462D
:1071200010F0C6FBF0B90025284608B0BDEC028B74
:10713000BDE8F08722464146DBE7B9F1000F1CD1DC
:10714000002D3CD1B2F90C33DAF84005D6EDC60A71
:1071500000EE103A0368B8EEC00A1B6A9847B0EE1A
:10716000408A0EE0002DDED106F2E45406F2F45619
:1071700096E80F0084E80F00D6E707EE909AB8EE85
:10718000678A2146404610F027FCB4EEC08AF1EE33
:1071900010FA17DBB6F8F03303932146404610F09F
:1071A0001BFCBCEEC00A07F54C50039B174A8DED43
:1071B000000A062118304CF0ABF90125B4E79FED29
:1071C000128ADEE707F5AB4122466431404610F0F3
:1071D0006FFB05460028A6D0B6F8F033039321468E
:1071E000404610F0F9FBBCEEC00A07F54C50039B7B
:1071F000074A8DED000A062118304CF089F993E713
:1072000000000034E02E65420000000070DC0B0836
:107210008EDC0B0870B500F5005500F5A046B5F9F9
:1072200010130029ACBF01234FF0FF330029B8BF72
:10723000494286F8BC3589B2044604F07DFAB5F9B6
:107240000C3396EDC97A002BCABF07EE903ADFEDFA
:107250000E7AF8EEE77AFCEEE77AF8EE677AB4EEAB
:10726000E77AF1EE10FA08D804F54C501830074AC6
:1072700006214CF04DF9012070BD204604F0A8F91C
:107280000028F1D1F8E700BF00000000ACDC0B08DB
:107290002DE9F04100F5AB4700F5AC456437043506
:1072A00004462946384610F05FF904F5A04604F577
:1072B000405830B3D6F8FC124B1C22D0D8F8400509
:1072C00003681B6B9847D6F8D435012B47D0D6F806
:1072D000D435022B06D12046FEF736FFD6F8083605
:1072E000984243DD2046FEF72FFFD6F80836C01A35
:1072F0000028B8BF4042B0F5FA7FCCBF0020012083
:1073000035E004F5AB402946743010F065FBDFED45
:10731000197AB4EEE70AF1EE10FA16D53846294686
:1073200010F02AFA9FED147ADFED140AF6EE007AD7
:10733000E0EE077A28469FED120AFDEEE77AF8EEB6
:10734000E77A27EE800A10F0BDFBD8F840059FEDE4
:107350000D0A03682A469B6A39469847B3E72046D8
:10736000FEF7F2FED6F808369842B0DB0120BDE801
:10737000F08100BF00004843A00CB34500009643D5
:107380000AD7233C00000000F7B5374FD1ED026A61
:10739000D7F8F8359FED357A07EE903AF8EEE77AB0
:1073A0000546D7EE876A0E46F5EEC06AF1EE10FA92
:1073B00008DD52F079FF2E4A06214CF0A9F8012091
:1073C00003B0F0BDD1ED037A97EDC76AF5EEC07A50
:1073D000F1EE10FA13DDF4EEC67AF1EE10FA0ED5E6
:1073E00052F062FF0446D7F81C03F9F785F8214AEA
:1073F000CDE90001062120464CF08AF8DFE7DFEDF9
:107400001E7A337CB4EEE76AF1EE10FA54BFB0EEA8
:10741000677AB0EE467A0BB90020D1E7B5EEC06AC4
:10742000F1EE10FA0CDC86EE876A03EB830307EEBD
:10743000903AF8EEE77AF4EEC67AF1EE10FAEBD570
:107440002C7C002CE8D179F02FFD6B69C01A337CBD
:107450004FF47A7253439842DED901232B7479F0AA
:1074600023FD68612046ABE7387C00200AD7233C27
:10747000C4DC0B08D5DC0B080AD723BC38B505469D
:1074800073F0FEFA72F086F8044640B979F00CFD0C
:10749000EB68C01AAB68984284BFAC6001242046F8
:1074A00038BD000038B504460D4679F0FDFC04F502
:1074B000A0439FED077AC3F8D805D5ED027A67EEB1
:1074C000877AFDEEE77A17EE902AC3F8D42538BD07
:1074D00000007A4410B5044679F0E6FC04F5A043B8
:1074E000D3F8D825801AD3F8D42590424FF0000065
:1074F00084BFC3F8D405012010BD000000F5A043EF
:1075000093EDC97AD3F8D42522EAE27207EE902AE5
:10751000F8EEE77A0020B4EEE77AF1EE10FA44BF15
:10752000C3F8D4050120704710B500F5005300F5ED
:10753000A040B3F9DE32002BB4BF4FF0FF3301237C
:1075400080F8BC3500F2046400F2F4500FC884E8FF
:107550000F0010BD38B504462DED028BF0EE408AC9
:10756000B0EE608A09B301295ED0B5EEC08AF1EEB3
:1075700010FA69DDDFED357AB4EEE78AF1EE10FA44
:1075800062D8FCEEC87A04F54C5017EE903A304AB7
:10759000062118304BF0BCFFFDEEC87A04F500540C
:1075A00017EE903A84F8AB323CE0F8EE000A21F096
:1075B000A9F940B104F580444FF0FF33C4F83C3DD5
:1075C000BDEC028B38BD04F50053B3F9B42207EECD
:1075D000902AF8EEE77AF4EEE87AF1EE10FAC4D8E1
:1075E000B3F9B63207EE903AF8EEE77AF4EEE87ABD
:1075F000F1EE10FAB9DBDFED157A68EEA77A04F543
:107600008043FDEEE77A04F54C5017EE902AFCEE2D
:10761000E87AC3F83C2D062117EE903A0D4A18304F
:107620004BF076FF0120CBE7FCEEC07A00F54C5022
:1076300017EE903A084A0621183004F500544BF032
:1076400067FFC4EDB08AEDE70020B9E70000C8424B
:107650001BDD0B08F4DC0B0808DD0B08D1F80D303E
:1076600000EE903AD1F80930097A00EE103AFFF7AF
:1076700071BF000070B58B88012B04460D4611D1F7
:1076800000F590763046FAF73BFA02280AD994F8CA
:107690001414B02303FB01612046DC31BDE87040C7
:1076A000FFF7B2B909F058FE05F10801BDE87040D6
:1076B00009F0A0BAF0B500F5A046002789B004464D
:1076C00086F8457308460D4624F09CF940B3012323
:1076D00086F83C3304F54053D3F840050368DB6B70
:1076E000984786F84373C6F8C07503A80FF044FEA8
:1076F000B6F8F0134FF6FF73994208BF39460131CF
:1077000004F5A74001AA89B2343026F06DF928B1FA
:10771000BDF80600A0F115035842584186F83D0314
:107720006B885D2B00F0008133D81F2B2AD80F2BDC
:1077300001D800202BE0103B0F2BFAD801A252F801
:1077400023F000BF377801084D7801085778010809
:1077500061780108757801084378010825780108E7
:10776000337701083377010833770108337701084D
:1077700033770108337701083377010885780108EA
:107780006B780108532BD4D1012086F8430309B04C
:10779000F0BDBD2B18D8BB2B4BD8B22B7CD00CD84E
:1077A000702B74D0722BC4D1D5ED027AFDEEE77A3E
:1077B00017EE903AC6F8D4353BE0B32BB9D1294641
:1077C0002046FFF757FF34E0C33B9AB2112AB0D8E6
:1077D000112BAED801A252F823F000BFD3780108D4
:1077E00033770108D378010833770108337701082C
:1077F00033770108D378010833770108337701081C
:10780000337701080B7901083377010833770108D2
:107810003377010833770108A3780108337701082B
:10782000C3780108002386F8793329462046FFF7FC
:107830005BF90120ABE705F108012046FEF7C6FF22
:10784000F7E729462046FFF799F9F2E7294620464F
:10785000FFF7DCF9EDE729462046FFF7F1F9E8E705
:1078600029462046FFF726FAE3E729462046FFF798
:10787000ABFADEE704F5994129223831204605F0BC
:10788000F5FFD6E729462046FFF738FAD1E7294623
:107890002046FFF707FECCE729462046FFF7DEFE2D
:1078A000C7E7AB88012BC4D803F0010386F83E3349
:1078B00004F54C50AB88204A062118304BF028FEC6
:1078C000B7E7A988003918BF0121204600F098FBCE
:1078D000AFE7EB6896F8E91604F5AC44703473B979
:1078E0002B6963B96B6953B9204657F0AFFD042883
:1078F0009FD196F8E916204657F0B2FD99E705F1B9
:107900000802204657F0EAFE93E704F5AC4095EDF7
:10791000041AD5ED020A95ED030A96F8E91600223D
:10792000703057F0BFFD84E704F5994029462030B8
:10793000FFF768FA7DE700BF2CDD0B0800F58042F9
:1079400000F59943D2F80C2D20339A4201D1FFF76C
:10795000B1BE01207047000010B500F5804200F56F
:107960009943D2F80C2D20339A4204460ED100F5EB
:1079700099410822383105F079FF04F54C50044A4A
:10798000BDE81040062118304BF0C2BD10BD00BF4D
:107990003CDD0B08F0B506468FB009AD06F5A044F6
:1079A00028460F460FF0E8FCB4F8F0334FF6FF72AC
:1079B000934208BF0023013306F5A74007AA99B2F6
:1079C000343026F011F8A0B117B10023C4F8B8354F
:1079D00095E80F0001AE86E80F00D4F8103600934A
:1079E00004F2046494E80E00034802F031FD0FB085
:1079F000F0BD0120FBE700BFF878002070B5064617
:107A000006F5A045002103F097FED5F8C0457CB9E6
:107A1000304603F0DDFD10B90024204670BDD5F8D6
:107A2000B835012BF8DD79F03FFAC5F8C005F4E769
:107A3000D5F8D41561B179F037FAD5F8C035C01A48
:107A4000D5F8CC359842E7D90023C5F8D4350121C3
:107A50003046FFF79FFF04460028DDD006F54C5066
:107A6000044A062118304BF053FD002385F84533B6
:107A7000D3E700BF64DD0B0870B50A468B88190A8E
:107A8000137E0546DB0748BF01EB810105F5A044E5
:107A900048BF4900002603F04FFE84F8456328469E
:107AA00003F096FD10B90024204670BDD4F8D4151B
:107AB00051B1D4F8B835D4F8B4259342F3DD012B95
:107AC000F1DDC4F8D46501212846FFF763FF0446C1
:107AD0000028E8D005F54C50024A062118304BF03A
:107AE00017FDE1E77CDD0B0838B5054605F5A04438
:107AF000898803F021FED4F8D43583BBD4F8B83597
:107B0000002BB8BF5B42012B02DC0024204638BDAD
:107B100094F8BD2594F8BE3572B9002BF5D005F563
:107B20004C50D4F8F8256423062192FBF3F3183067
:107B30000C4A4BF0EDFC01E0002BF0D10121C4F820
:107B4000D4152846FFF726FF04460028DDD005F5AA
:107B50004C50054A062118304BF0DAFCD6E70021DC
:107B6000EFE700BF94DD0B08B2DD0B082DE9F0470D
:107B70004B881F2B8AB004460A4631D80F2B07D8F2
:107B800004F54C50954A042118304BF0C1FC88E0B4
:107B9000A3F110010F29F3D801A050F821F000BF84
:107BA000B37C0108757D0108817D01088F7D010886
:107BB000A97D0108C17C0108A77C0108817B01081F
:107BC000817B0108817B0108817B0108817B0108A1
:107BD000817B0108817B0108B57D01089B7D01083F
:107BE000702B00F0F5800CD8532B00F0E9805D2B52
:107BF000C6D100F5994020300AB0BDE8F047FFF744
:107C00003DBCB32B08D8B12B4BD8722BB8D10AB0DE
:107C1000BDE8F047FFF772BCD42B3BD8BB2BAFD9E4
:107C2000A3F1BC02182AABD801A151F822F000BF81
:107C3000A37C0108A37C0108817B0108817B0108EA
:107C4000817B0108817B0108817B0108A37C0108FD
:107C5000817B0108A37C0108817B0108817B0108ED
:107C6000817B0108A37C0108817B0108817B0108DD
:107C7000817B0108A37C0108A37C0108A37C010887
:107C8000817B0108817B0108A37C0108817B0108BD
:107C9000A37C0108DF2B04D040F6B83293427FF476
:107CA0006FAF01202FE020460AB0BDE8F047FFF794
:107CB000DFB8114620460AB0BDE8F047FFF7CCB95F
:107CC00004F5A04504F5A946D5F8903304F5AB4773
:107CD00004F5AC4804F5AB49072B06F14C0607F157
:107CE000640708F1040809F174090FD104F5A744E9
:107CF00008340194D5F80C33009342464B4639467C
:107D0000304677F0BDFA0AB0BDE8F08700230DF1E8
:107D1000270133488DF82730FEF7EAFCD5EDD27AFB
:107D2000D5EDC70A95EDCA1AD5F82CA3CDED060AF4
:107D300030EE670A04F5AD4074308DED070A8DED25
:107D4000051A71F01DFC0546204600F0A5FE9DF8C1
:107D500027309DED051ADDED060A9DED070ACDE9F8
:107D60000203CDE900A54B4642463946304677F03E
:107D7000DDF9C8E72046918803F0DEFC0020C2E769
:107D8000114620460AB0BDE8F047FFF775BE204611
:107D90000AB0BDE8F047FFF731BE114620460AB0F1
:107DA000BDE8F047FFF7A0BE20460AB0BDE8F047A7
:107DB000FFF730BA20460AB0BDE8F047FFF768BACF
:107DC00000F5994020300AB0BDE8F047FFF7DCBA73
:107DD0000AB0BDE8F047FFF77DBB00BFCCDD0B0864
:107DE000382C002070B500F5804200F59943D2F898
:107DF0000C2D20339A4205460E4602D00024204620
:107E000070BDFFF7B3FE04460028F7D005F54C50CF
:107E1000318818304FF060FDF1E7000021F0400399
:107E2000152B04D0A1F15E03584258417047012040
:107E300070470000102946D8DFE801F0090D111540
:107E4000191D212529452D31354139393D0000F5D0
:107E500099405C30704700F598403430704700F529
:107E600098403C30704700F598404430704700F52A
:107E700098404C30704700F598407430704700F5DA
:107E800098407C30704700F599400430704700F509
:107E900099401830704700F599402030704700F540
:107EA00099403830704700F599404030704700F5F0
:107EB00099404830704700F599405430704700F5BC
:107EC00099406430704700207047000000290DDBA6
:107ED000074890F8782BCBB29A4207D3D0F8743B7E
:107EE0000122595CA0F5005005F09CBD704700BF11
:107EF000384C00202DE9F34100F5005300F54C55B6
:107F000093F8483B03F0010603F0020803F004076E
:107F10005B07044605F1180535D01F4A062128469F
:107F20004BF0F6FA26B104F53A500C3073F0B6FB7C
:107F3000B8F1000F04D004F53F50243073F02AF953
:107F400027B104F544503C3073F0D2FF04F5A0444F
:107F5000012384F89937114A114B1249B8F1000FE7
:107F600008BF1A46002F08BF1946CDE900210E4A66
:107F70000621002E18BF134628460C4A4BF0C8FABB
:107F800002B0BDE8F0810A4A0621284602B0BDE8E9
:107F9000F0414BF0BDBA00BFF9DD0B08EEDD0B0878
:107FA0001CB40C08F5DD0B08E8DD0B080ADE0B0835
:107FB0001CDE0B0810B5044600F53A500C3073F087
:107FC00099FB04F53F50243073F010F904F5445048
:107FD0003C3073F0C7FF04F5A04393F899275AB1DA
:107FE000002283F8992704F54C50044ABDE810405C
:107FF000062118304BF08CBA10BD00BF3CDE0B08D8
:1080000009B1FFF777BFFFF7D5BF000000F5804348
:108010000A4AD3F80C1D91420DD093F8193D43B98B
:1080200000F599422032914203D100F5A04090F82A
:108030003E33184670470023FBE700BF1479002049
:1080400010B5044678F030FF054BD3F82C3DC01A2C
:10805000642804D82046BDE8104053F091BD10BDFF
:10806000386C002010B500F52C54D4ED0E7AF5EEE6
:10807000C07AF1EE10FA8AB04FF0000304F1380430
:1080800045D907930893099306AB019300F59550E2
:1080900007AB009303AA05AB04A9103008F030FE2B
:1080A00030B3DDED080A9DED070A99F031FADDEDF8
:1080B000090A99F02DFAD4ED007A9DED047A77EE55
:1080C000A76AB4EEE70AF1EE10FAF4EEC76AACBFA5
:1080D00001200020F1EE10FA0CD802309DED037A59
:1080E000F4EEC77AF1EE10FA0CD8003818BF012070
:1080F0000AB010BDF4EEC77AF1EE10FA9CBF013061
:10810000C0B2EBE7012894BF00200120F0E7002077
:10811000EEE7000010B5074B1A7A4AB901241C7229
:1081200049F04EF922461121BDE8104049F0A4B8AB
:1081300010BD00BFE883002010B5074B1A7A4AB182
:1081400000241C7249F03CF922461121BDE8104080
:1081500049F092B810BD00BFE8830020F0B5054695
:1081600085B005F59556684610360FF005F9694655
:10817000304608F0F7FEA0B13248334C334F71F06F
:10818000FFF940B105F52C53D3ED0E7AF5EEC07A28
:10819000F1EE10FA07D8002328462380FB73FFF77F
:1081A000CBFF05B0F0BD2846FFF75CFFA0B36378B6
:1081B0007BBB23780133DBB2082B237002D130461E
:1081C00008F00AFE2378092B02D1304608F0FCFDA6
:1081D0002378092B1DD94FF48573238049F0F0F8DB
:1081E0000222102149F048F878F05EFE6368C01A58
:1081F00047F23053984209D905F54C50144A0221F0
:1082000018304BF085F978F04FFE60602846FFF794
:1082100081FF6378FB73C4E72678002EF9D0013E16
:108220006378F6B22670002BF3D0002EF1D1667081
:1082300049F0C6F83246102149F01EF82846FFF7EB
:108240007BFFE6E72C830020E88300209584002054
:1082500050DE0B0800F5A040D0F89033042B14BF7B
:1082600090F8BC030120704773B500F5804501927A
:10827000A5F8241D044678F017FEC5F8280DD5F89A
:108280000C0D03685B68984785F8220DD5F80C0D36
:1082900003685B6898470F28019A0BD80F2827D8E6
:1082A000DFE800F01C261C1C1C1C1C1C1C264E2677
:1082B0000A260A0A18281BD104F50056019296F9DD
:1082C0002033ABB1D5F80C0D03685B68984785F88F
:1082D000220D96F92033019A022B29E01F4B93F8C7
:1082E0009A3703B304F598417431204605F0BEFA7D
:1082F000D5F80C0D95F8226D03685B68984704F576
:108300004C54864204F1180420D0D5F80C0D0368B3
:108310009B689847124A03460421204602B0BDE8F4
:1083200070404BF0F5B804F5005393F92033022B5D
:10833000D8D004F59841042B0CBF7C313431D4E7FC
:108340002046FFF787FF0028D2D1B5E7054A042170
:10835000204602B0BDE870404BF0DAB8387C00200F
:1083600060DE0B0882DE0B08F0B5044604F580469B
:1083700085B00F46154653F089FBD6F80C0DA6F8CC
:10838000247D03685B68984718281ED8DFE800F052
:108390000D0D0D0D0D0D0D0D0D1D52680D0D5757C9
:1083A0001D1D1D1D1D1D1D1D0D00314AD2F89013F0
:1083B000012921D104F5005393F82133023B012B0D
:1083C0001AD904F5405383F81413D6F80C0D294A32
:1083D000294B052D18BF13460268039392689047F6
:1083E00004F54C5418340090039B244A0421204681
:1083F0004BF08EF805B0F0BD92F89A373BB104F51A
:1084000098412A467431204605F030FADDE704F53C
:10841000005393F92133032B03D1204603F0E8F9ED
:10842000D3E7022BEBD0042B15D104F599412A4652
:108430002031E8E72046FFF70DFF0028C5D104F5FD
:10844000005393F92133032BE7D0022BD7D0042B11
:10845000EBD0012BB9D104F599412A463831D2E746
:1084600004F5005393F92133042BAED1DDE700BFAF
:10847000387C002098DE0B0873C30B08A0DE0B08C5
:1084800070B500F54C5504461835124A04212846AB
:1084900004F580464BF03CF80023A6F8243D04F593
:1084A000005393F86832032B12D196F8221D302224
:1084B000204605F0B7FAD6F80C0D03689B6898477C
:1084C000054A034606212846BDE870404BF020B817
:1084D00070BD00BFB4DE0B08CBDE0B0800F54053C7
:1084E00010B500220529044600F54C5083F81423EA
:1084F00000F118000CBF054A054A042104F5804428
:108500004BF006F80023A4F8243D10BDE4DE0B0870
:10851000F5DE0B0830B50B4687B00446052A18D89F
:10852000DFE802F0172A0350175D00F5A043D3F8E7
:108530009033042B20D02C4D95F8353DE3B12B49D9
:10854000A1F5107025F022FE28B1294B012283F8F5
:10855000BC2307B030BD2549A1F5107026F016F9EF
:1085600050B104F5994104222031A5F5804007B0AF
:10857000BDE8304005F07AB904F5A043D3F8903354
:10858000042BE6D004F5005393F9EB32022B0AD109
:10859000154B93F8353D33B11449A1F5107025F012
:1085A000F5FD0028D1D104F5994104223831204647
:1085B00005F05CF904F50A502B3007B0BDE83040F7
:1085C00041F0CEBB0B4A112101A877F047FE04F51C
:1085D000AA4001AA0121583073F076FDB9E707B02F
:1085E000BDE8304003F004B9386C00202C82002034
:1085F000387C002010DF0B0870B52DED048B04468D
:1086000078F04AFC4F4BB4F8BE101A884E4E8A429E
:1086100005464E4A06D01980002330601370BDEC29
:10862000048B70BD33684A49C31A8B4276D9012343
:10863000137053F02BFB53F0E3F9356053F026FB36
:1086400053F0DEF904F5405393F8133323B104F5E6
:10865000AA40583073F08CFC53F0FAF90428DED9A4
:1086600053F014FA0021204603F0ECFB00212046D1
:10867000F0EE409A03F0F0FB01212046B0EE409A64
:1086800003F0AAFD00212046B0EE408A03F0EEFB85
:1086900004F5AD407430F0EE408A70F07BFFDFED02
:1086A0002D7A0028B0EE690A4FF0040008BFB0EE42
:1086B000678A54F0E1FEB0EE490A132054F0DCFE64
:1086C000B0EE680A152054F0D7FE04F5AA45B0EEC6
:1086D000680A1A2054F0D0FE58354620B0EE480AF9
:1086E00054F0CAFE284673F0D1FC08BB01210846AD
:1086F00055F0C4F99FED170A022054F0BDFE9FED1E
:10870000150A032054F0B8FE204603F073FFBDECB9
:10871000048B2046BDE8704004F088BE1278002A21
:108720003FF47DAF44F6206293427FF678AF80E756
:108730002846FDF7FDFA04F5A04393F962352B2B8B
:10874000D4D06CE7F4830020F8830020F683002067
:10875000400D03000000000000F5804200F5994341
:10876000D2F80C2D20339A4204D100F5A04090F8A5
:10877000BC03E8B10F4B93F8680203F54053A0F136
:108780002702012A93F8A8370FD92C2809D00A28E4
:1087900009D0A0F13102504250410A2B18BF0020ED
:1087A00070470120F9E7012070470A3B58425841C1
:1087B000704700BF384C002008B500F5005393F80F
:1087C000502142B193F88C312BB1FFF7C5FF80F0F7
:1087D0000100C0B208BD0120FCE700002DE9F04710
:1087E00000F50055DFF8ACA295F88C91044600F531
:1087F000AD408AB0743070F0C3FEDAF89033042BC9
:1088000006464ED000284CD0BAF8F213AAF5A04084
:10881000FFF704FB014620B19AF8B8134B1E5942EA
:10882000594104F5055808F11008404661F01EFC56
:108830009AF8A8370A2B074603D1A6BB00238AF86B
:10884000A83795F85031002B38D195F956318C4D19
:10885000012B03D0063BDBB2012B11D895F868320F
:108860000A2B0DD104F58046D6F80C0D03681B6A5F
:10887000984728B1D6F8101D2B22204604F0F6FFA9
:108880009AF8A8370A2B04BF37238AF8A83795F837
:1088900068320A2B02D1372385F868320AB0BDE866
:1088A000F0870121BDE740EA0903DBB2002BC8D104
:1088B000744800F0F1F80028C0D0C2E7002EEDD0D7
:1088C00004F5A9404C3076F0A7FB0028E6D12046FD
:1088D000FFF742FF0028E1D1002F00F0BF806A4976
:1088E0003A46404660F09AFF95F95691B9F1010F6A
:1088F00007D040F38780A9F10603DBB2012B00F219
:1089000081805FFA89F9B9F1010F4ED104F58042F7
:1089100004F59943D2F80C2D20339A4209D104F57D
:10892000A04393F8BC3323B195F8EB32013B012B04
:10893000B4D904F599410A223831204606AE04F034
:1089400095FF30460EF018FD95F9692192BBB9F1FB
:10895000010F2FD004F5A049B5F96A31D9F8E01517
:10896000DFED4A5AD1ED017A002BF8EEE77A52DDBD
:1089700007EE103AF8EEC76AE6EEA57A3046FDEE4D
:10898000E77A17EE901A0EF0FDFC00234046CDE981
:10899000043361F007FC04A962F064F9002857D0A1
:1089A000049B0893059B099317E004F599410A225B
:1089B0004831C2E72046FDF733FA07EE900AE84651
:1089C00004F5AB42743221464046B8EEE70AFEF7A2
:1089D00081F898E80F0086E80F0095F95631012BD1
:1089E00010D031462046FDF78BFB31462046FDF77F
:1089F00059FF95F95631072B04D104F54054012352
:108A000084F8123348F0DCFC3A4609210AB0BDE88C
:108A1000F04748F031BCD5ED566A95ED595A95EDC1
:108A2000577A35EE076A36EEC57AB4EEC67AF1EEBD
:108A300010FA89BF37EE067A95EDD37A27EE257ABC
:108A4000F6EE006A94BFE7EE257AE7EE267A95E720
:108A5000D9F8E0359A680892DB68A4E7B9F1000F0D
:108A60003FF41CAF95F88C31002B7FF417AF04F561
:108A70004C50074A052118304AF04AFDC2E700BFB2
:108A8000384C0020382C00201CDF0B080000C842A6
:108A900025DF0B08387C002010B5044600F5AD40FA
:108AA000743070F077FD04F5A04494EDE57A48B198
:108AB000DFED067AB4EEE77AF1EE10FAACBF0120F2
:108AC000002010BDDFED027AF4E700BFCDCCCC3D35
:108AD0006666663F00F58043D3F80C1D00F59943A8
:108AE0006433994204D100F5A04393F888239AB9DE
:108AF00000F599432033994210D100F5A04393F833
:108B000088234AB1D3F89023032A07D1B3F8F2237C
:108B1000A2F116035A425A41104670470022FBE761
:108B20002DE9F84F00F5804200F59943D2F80C2D5D
:108B300020339A42054600F5A04704D100F50058BD
:108B400098F9C43233B90023C7F87C3387F87933F6
:108B5000BDE8F88F78F0A8F9D7F83043814634B1F2
:108B6000041B40F6C3139C4294BF002401242846F2
:108B7000FFF792FF834620B1002487F87843002650
:108B80003FE005F5AD40743070F0FAFC82460028F5
:108B9000F2D005F5A9464C36304676F03DFA00286D
:108BA00040D097F87863C6BB44B305F5805141F2D5
:108BB0007072D1F8A834002BB8BF5B42934206DC38
:108BC000D1F8AC34002BB8BF5B42934228DD05F5E9
:108BD000A74105F5AB40783174300EF0FDFEDFEDB6
:108BE000467AC7F87C93B4EEE70AF1EE10FA4FF03C
:108BF00000034CBF01260026C7F88033012387F805
:108C0000783305F59070F8F77BFF022833D9002CF4
:108C100046D10023C7F87C339AE75C465E46EDE711
:108C20003446EBE7304676F0DFF9064638B1002CE3
:108C3000A5D04FF4FA73C7F8803354469FE7D7F8AE
:108C40009033012B03D0032B0DD03446D9E7D8ED58
:108C5000D97AF5EEC07AF1EE10FAF6DD97F888339E
:108C6000002BF2D1E5E72846FFF734FF0028ECD1CE
:108C7000002CDED1C5E705F5FC5A05F5005B0AF1CD
:108C8000180A9BF8E610504606F03AFA0028C0D0C1
:108C90009BF8E610504606F02BFB0028B7D1B8E74A
:108CA000D7F87C3313B9C7F87C9351E7D7F8802302
:108CB000A9EB03039342FFF44BAF97F87933002BF2
:108CC0007FF446AF012287F8792398F8C432DB0796
:108CD00005D505F5AD400C217430F8F749FE05F5D2
:108CE0004C5018302EB1054A0221BDE8F84F4AF029
:108CF0000FBC034A3146F8E7000096423CDF0B0800
:108D000052DF0B082DE9F04F2DED028B054685B0A3
:108D1000002305F50058039378F0C6F8D8EDB07A33
:108D2000F5EEC07AF1EE10FAC4BF9FEDBD7A67EEA2
:108D3000877A05F5907BC8BFFCEEE77A0746584670
:108D4000CCBF17EE906A9626F8F7DAFE022840F2BA
:108D5000FC8095F814349FEDB37AB02202FB0353E4
:108D6000D3ED837A67EE877AFCEEE77A17EE903AD6
:108D70009E428CBF00260126B8F9B432022BB8BF40
:108D8000022307EE903A05F59550B8EEE78A03A95D
:108D9000F6EE087A103028EE278A08F0C1F804466B
:108DA00040B1DDED037AF4EEC87AF1EE10FAACBF13
:108DB000012400245846F8F7A3FE05F5AD49012823
:108DC00009F1740905F5A04A16D8484670F0D8FB99
:108DD00090B18CB99AEDE57ADFED937AB4EEE77A4B
:108DE000F1EE10FA08DDDDED037AF4EEC87AF1EE6B
:108DF00010FAACBF01240024484670F0C1FB00907B
:108E0000002800F0FA8095F8142405EB0212D2F83D
:108E1000C02172B158460192F8F772FE012800F2A3
:108E20009680019A41F28731BA1A8A428CBF002299
:108E30000122DAF82C1301B11AB9002C40F0898014
:108E4000344605F5804105F59942D1F80C1D2032D4
:108E500091421AD198F9EC22002A40F08280002237
:108E60008AF87A23DAF89023042A00F0A880072AE7
:108E700000F0B980032A08D12846FFF72BFE20B165
:108E800000248AF87943CAF830439AF87A2302B169
:108E90007CB907EE904A9FED657ADAEDE56AF8EE67
:108EA000677A67EE877A9FED627AE6EE877ACAED97
:108EB000E57A2846FFF7F0FD0446A8B19AF8980332
:108EC000CAF82C7308B9CAF89C7305F5804105F5FA
:108ED0009942D1F80C1D2032914205D1DAF83023A5
:108EE00002B108B9CAF830739AF8C0248AF89843D6
:108EF00064F3C3028AF8C0246AF08EFC21466AF04B
:108F000067FC4C4A28465471FFF70AFE2846FBF7D7
:108F10007FFC34B198F86A221AB977F0C5FFC8F817
:108F20006C0288F86A422846FFF7B6FD002875D122
:108F3000484670F02FFB80F00100C0B28AF8A00311
:108F400005B0BDEC028BBDE8F08F002614E70022CF
:108F50006FE71FF0ADF81EF0FBF900287FF470AF4B
:108F60006FE7524207EE902A05F6C802F8EEE77A5C
:108F700092EDDB7AF4EEC77AF1EE10FA11DDDFED57
:108F80002E7A9AEDE57ACAF88473B4EEE77A012274
:108F9000F1EE10FA8AF87A237FF764AFCAEDE57A2A
:108FA00060E79AF87A23002A3FF45CAFDAF884236A
:108FB00040F6B831BA1A8A423FF651AF52E705F58A
:108FC000A9404C3076F010F800283FF45EAF9AEDDF
:108FD000C77ADFED197AB4EEE77AF1EE10FA7FF78F
:108FE00054AF009C51E79AEDC77AFEEE007AB4EEDA
:108FF000E77AF1EE10FAF4D447E7DAF89023002C80
:1090000018BF3446012A07D005F5A9404C3075F049
:10901000E1FF00283FF439AF002436E700208DE758
:109020000000B4420000C8429A99993E9A99193EAC
:109030009A99593F95840020CDCC4C3E0020704732
:1090400000207047012070470020704701207047C2
:10905000034BD3F89003431E58425841704700BF5A
:10906000387C002030B587B002A80EF085F92D4875
:1090700075F0B0FF20B12C492C48FCF721FF1FE010
:10908000284875F0B1FFE8B1294C04F124052346C6
:1090900004F11002A4F11001A4F59470009575F08C
:1090A000C9FFCDE90045A4F2F45292EDC90A214965
:1090B00004F11003A4F11002A4F5947075F07CFF84
:1090C00007B030BD174802A975F0CCFF08B102A95E
:1090D000D2E7164802F07CFA0028CCD1164CD4F81E
:1090E0001836002BC7D004F2046204F2E45104F2F3
:1090F000F4500EF0DDFB0028BDD1D4EDCA7AB7EEF6
:10910000000A04F20461A4F5A04030EE670AFDF7FE
:109110003DF804F2E45204F20461A4F5A040FCF727
:10912000E7FECDE7048100203C820020382C00209F
:109130002C820020B4570020387C002008B50A4853
:1091400090F85D33013B012B03D8A0F50050F9F7EF
:1091500021FD0648F9F746FC0448F9F7E1FCBDE8B3
:1091600008400248F9F7FABF384C0020382C00209C
:10917000124A904208B50ED002F1080188420AD086
:1091800002F11001884206D002F13801884202D073
:109190005C32904206D10A4B93F91503B0FA80F085
:1091A000400908BD03681B6A984728B1054B93F82E
:1091B000120380F00100F4E70120F2E77478002048
:1091C000384C0020385C0020104A904208B518D076
:1091D00002F10801884214D002F11001884210D037
:1091E00002F1380188420CD05C32904209D0036809
:1091F0001B6A984738B1064B93F8120380F00100C0
:1092000008BD0020FCE70120FAE700BF74780020C9
:10921000385C0020024A0260024A4260704700BF88
:10922000A4DF0B08E83E002008B50368DB6D984713
:109230000648D0F80C2D00F698439A4205D0BDE8B8
:109240000840A0F58040FEF7B5BE08BD386C002090
:109250002DE9F041454CA4F558730025C11A4B4245
:10926000C4E9D955A4F500584B41002284F8E852CE
:10927000A4F83E5384F84253C4F8042384F80053FE
:1092800084F8795384F87A53C4F86053C4F870535F
:10929000C4F8142388F8B4354368D3F8FC31A4F833
:1092A000383304F2F45306460FCB04F2E45787E850
:1092B0000F0084F8415384F85053C4F8C05577F038
:1092C000F3FDA4F58057C7F8140D336830465B6989
:1092D00098474FF0FF3384F8440384F8455388F8E7
:1092E000145384F84353C7F83C3D336830469B6DB4
:1092F00098470546002836D0336830469B6B984720
:1093000084F88803D8F840050368DB6B9847A7F515
:10931000556072F02BFBA4F5A04002F0FFFCA8F50D
:109320006B6060F009FF94F8BC33CBB1A4F5A040AA
:10933000FFF7B2FBA0B904F2F46070F02BF978B932
:10934000D7F80C0D03685B6B984748B950F0ACFF39
:10935000074A06214AF0DCF804F56D7024F0C2FFDC
:109360000448F8F78DFE2846BDE8F081387C0020DF
:1093700064DF0B08382C002070B503681B6E0E46A6
:1093800015469847044650B995F900303BB9054851
:10939000054B00683246C06A29461CF037F8204663
:1093A00070BD00BF342C002088DF0B0810B50D4CB9
:1093B000204672F0D7F804F5AC7071F04FFE04F55A
:1093C0002C7072F07DFD084B03F5A042002182F85D
:1093D000001303F500530021C2F80413012283F89F
:1093E000D82D10BDC45A0020382C002008B52DED12
:1093F000028B1520B0EE408A54F03EF8B0EE480AD9
:10940000BDEC028B1A20BDE8084054F035B80000CE
:1094100008B5084890F915330121A0F5005033B183
:1094200002F0DAFEBDE80840462054F025B802F00C
:10943000FBFEF7E7384C00200420704700487047D7
:10944000C6490D0800487047C6490D08037A73B134
:10945000D0ED037AFDEEE77A17EE903A084AC2F8AB
:10946000A433437A3BB10369C2F8A8337047436819
:10947000D3F8F831F2E74368D3F8FC31F4E700BFE2
:10948000387C002008B50023038100F114014068F6
:1094900007F05CFD012008BD70B56E4E2DED048B0C
:1094A00006F59A4304460121304693ED159ADFED07
:1094B0006A9A02F0C7FC0121B0EE408A304602F001
:1094C000CBFCC8EE297A06F500556068B5F938334B
:1094D00004F1140108EE903AF8EEE88AB5F93A334F
:1094E00068EEA78AC0EE297A08EE103AB8EEC88A6C
:1094F00028EE278A07F02AFD95F93E3363B39FEDE6
:10950000577AF0EEE87AF4EEC77AF1EE10FA23D546
:10951000227A6368002A55D1012222720022E26079
:1095200094ED037ADFED4E7AD3F8F8314D4A4E4888
:1095300067EEC77A9FED4D7A67EE877AB0EE490AFB
:10954000FDEEE77A17EE901A0B44C2F8A43300231D
:10955000012271F097FF08E0002343482372F0EEE8
:10956000490AB0EE680A71F089FF042053F084FFC5
:1095700095F93E3343B19FED397AF0EEC87AF4EEB7
:10958000C77AF1EE10FA28D4002339486372F0EE5E
:10959000490AB0EE480A71F0CBFB132053F06CFF80
:1095A000B5F93C33002B03DD324E96F9523163BBE3
:1095B00028482021F8F7CAFF002843D1254802F0A7
:1095C0007DFA42E0D3EDC56A96ED467AD4ED037A92
:1095D000E6EE877AC4ED037AA2E7637A2BB901231A
:1095E00063726368D3F8FC3123611E4B2169C3F8B1
:1095F000A8136368D3F8FC010023091A1A461C4813
:10960000B0EE490A71F07AFCC7E70121A6F5405097
:1096100002F02CFC80EE297AB5F93C33002106F5E6
:109620009E7007EE903AF8EEE77AF0EE490A27EEE0
:10963000870A72F045FBBDEC048B2046BDE8704004
:10964000FFF7D4BE0348F9F7FDFB07EE900AB8EE2A
:10965000E70AF0E7382C002000A08C450000003419
:10966000E02E6542387C0020C45A00200000C84229
:109670001C5C0020385C00202DE9F04F2DED0C8B98
:10968000DFF8A0A39FEDDDDA9FEDDD9A97B00AF534
:109690009A4300F1140504460121504693ED15BA92
:1096A00002F0D0FB01215046F0EE408A02F0D4FBDC
:1096B00001215046B0EE408A02F0D8FBDFEDD17AAE
:1096C00088EEA77A0AF5005601A8B6F938330AF5EC
:1096D000A04B0AEE903AF8EEEAAAB6F93A33DFED7B
:1096E000CA8A6AEE87AA88EE277A0AEE103AB8EE9E
:1096F000CAAAB6F93C339FEDC58A2AEE07AA80EEC6
:10970000277A09EE903AF8EEE99A6AEE8D7A69EED8
:10971000879AF0EEEACAF4EEC8CACDED017AB0EE4F
:10972000CACA6AEE0D7AF1EE10FAF0EEE9BAB4EEBA
:10973000C8CACDED027A58BF4FF0010969EE8D7AA3
:1097400048BF4FF00009F1EE10FAF4EEC8BA9AEDF6
:10975000460ACDED037A54BF4FF001084FF00008E0
:10976000F1EE10FA54BF0127002721F051FC01A9A6
:10977000284620F06DFF284621F05CF8284620F0AE
:10978000D3FF20EE090A284620EE280ABDEEC00AC3
:109790008BEDE90A20F0E2FF20EE090A4FF07E533C
:1097A00020EE280ADFED9A8A0A93BDEEC00ACDEDBD
:1097B0000D8A8BEDEA0A0DF1280B59466068CDED54
:1097C0000C8ACDED0B8A07F0C1FB0021504602F058
:1097D00003FDB0EEC00AB4EEC80AF1EE10FA16D5D9
:1097E0005046FFF759F990B9F4EEC8CAF1EE10FAF5
:1097F0000DD5B4EEC8CAF1EE10FA08D5F4EEC8BA29
:10980000F1EE10FA44BF9BE80F0085E80F000AA8AC
:1098100021F074F8294612A88DED141A8DED120A64
:10982000CDED130ACDED151A21F07AF80DF1100ADD
:1098300051460EA88DED101ACDED048ACDED058AA6
:10984000CDED068A8DED0E0ACDED0F0ACDED111A84
:1098500020F038FEB6F93833DFED6E7A01EE103ABB
:10986000B6F93A3309EE103AB6F93C3308EE903ABD
:10987000B8EEC11AB8EEC99AF8EEE88A21EE271AB6
:1098800029EE279A68EEA78AF4EEC8CAF1EE10FA1C
:1098900021EE0D1A29EE0D9A68EE8D8A07D594F8FF
:1098A0002430DFED5B7A002B18BFB0EE671AB4EE00
:1098B000C8CAF1EE10FA07D594F82530DFED547AD6
:1098C000002B18BFB0EE679AF4EEC8BAF1EE10FAAA
:1098D00007D594F82630DFED4E7A002B18BFF0EE56
:1098E000678A9AE807000DF11C0B8BE80700F1EE80
:1098F000410AC2209DED070A1FF016F9C3208DED25
:10990000070AB0EE491AF1EE490A9DED080A1FF068
:109910000BF9B0EE681AF1EE680A8DED080AC42062
:109920009DED090A1FF000F9514658468DED090AD0
:1099300021F004FB12A928468DED120ACDED130A81
:109940008DED141A20F084FE284620F073FF06F5F2
:109950006963DDED076A93ED007A9FED290AC6EE93
:10996000877A06F6E8765846DDED086ACDED077A87
:10997000D6ED007A86EEA77ADDED096A8DED087ADC
:1099800086EEA77A8DED097A21F042FBB9F1000F3E
:1099900001D0CDED07AAB8F1000F01D08DED08AAD6
:1099A0000FB1CDED099AF0EE4B0A9DED070A1A486A
:1099B00071F064FD042053F05FFDF0EE4B0A9DED65
:1099C000080A164871F0B4F9132053F055FD002130
:1099D000F0EE4B0A9DED090A114872F071F920462C
:1099E000FFF704FD84F8249084F8258084F826701D
:1099F00017B0BDEC0C8BBDE8F08F00BF35FA8E3C84
:109A0000E02E654200A08C450000C84200000034F2
:109A100000000000CDCC4C3EC45A00201C5C00204D
:109A2000745D0020382C002010B50446FFF7F0FCD0
:109A30000B4B93F93E23022A0DD1B3F93C23002AA4
:109A400009DD03F5805393F9523123B12046BDE877
:109A50001040FFF711BE2046BDE81040FFF71CBDC7
:109A6000384C00200A2070470048704731EA0B0844
:109A70000048704731EA0B08012070470120704709
:109A8000012070470120704701207047034BD3F835
:109A90009003031F58425841704700BF387C002094
:109AA000F8B5194D05F2F4530FCB05F2E45405F265
:109AB000046684E80F0086E80F00002705F56D7046
:109AC00085F8447324F04EFE104B1C68E66A336838
:109AD00030465B689847A8B196F84D3093B1E36A79
:109AE0009B8F7BB150F0E0FBE36A094A9B8F062114
:109AF00049F00EFDE36A05F56D70998F24F01EFCA8
:109B0000E36A9F870120F8BD387C0020342C0020B8
:109B100074E00B0810B50A4C94F8B833012B0BD144
:109B200004F56D7021F0E2FEB4F8F233152B03D189
:109B300004F2CC4075F02EFB0023C4F8303310BD86
:109B4000387C002008B507F007FC90F87C32DB0772
:109B500004D5BDE80840024824F0A0BC08BD00BF01
:109B6000EC7F002010B5304C94F8B833012B0ED0A8
:109B7000A4F552710822A4F5A04003F077FE50F03E
:109B800093FBBDE81040294A062149F0C1BCB4F856
:109B9000F233162B05D0152B36D1D4F89033072B82
:109BA0000AD1234804F0E6F9214804F01FFBBDE880
:109BB00010401F4804F03CBAA4F5A040F9F72EFC71
:109BC000A4F5A040F9F736FBA4F54053D4F8A4134C
:109BD00093F97C2364235A4304F2CC4075F036FA9F
:109BE000C4F8A40304F2CC4075F072FB30B1BDE8B8
:109BF00010409FED100A462053F03EBCA4F5A04053
:109C0000BDE81040F9F706B91E2B18BF4FF0FF331F
:109C1000074818BFC4F8FC32F9F700FC0448F9F70C
:109C200009FB0348ECE700BF387C00208CE00B0800
:109C3000382C00200000000010B5144BB3F8F233AC
:109C4000532B04461ED102F0ABFE9FED110A4620B5
:109C500053F012FC9FED0E0A492053F00DFC9FEDCE
:109C60000C0A4A2053F008FC462053F0E5FC49203A
:109C700053F0E2FC4A2053F0DFFC2046BDE81040E0
:109C8000FFF794BBBDE81040FFF758BA387C0020BE
:109C900000000000082070470048704724E10B08CE
:109CA0000048704730E10B080120704708B50248B2
:109CB000FEF720F9012008BD382C0020014800F0F3
:109CC00057B900BFAC78002010B50446FFF736FA4C
:109CD0002046BDE81040FFF79BBB00000120704705
:109CE00000487047A4E10B0800487047ACE10B083E
:109CF000012070470120704710B5054B03F2046442
:109D000003F2F4530FCB84E80F00012010BD00BF15
:109D1000387C002008B50B4800F5A04200F5005340
:109D20000321D3F86C3B93FBF1F3C2F8A433F9F7AA
:109D3000E1FA0448F9F77EFABDE808400148F9F76E
:109D400069B800BF382C00200720704700487047D2
:109D500030C50B080048704720E20B08012070470F
:109D600001207047012070477047000008B50023AC
:109D7000037203610248FCF799F8012008BD00BF97
:109D8000382C002010B5184CD4F8543BB3F90830E7
:109D900023B9D4F8603BB3F90830E3B10023037270
:109DA0000361D4F8540B52F061F804F66C33D3ED30
:109DB000007A0E48F8EEE77A27EE800ABDEEC00A78
:109DC00080EDE90AA0F5A040F9F794FABDE810404B
:109DD000074801F01BBB037A002BE2D0A4F500502A
:109DE000F9F71CFBF2E700BF384C0020387C00205C
:109DF000382C002070B54E4DDFED4E7A95F81434B6
:109E00009FED4D7A2DED048BB02606FB035393EDA9
:109E1000848A9FED4A9A28EE278A05F5A553BDEE60
:109E2000C88A93ED070AF8EEC87A044667EE897A85
:109E300097EE870A1EF064FE237AF0EE408A002B2C
:109E400062D105F50053D3F8543BB3F90830002B29
:109E50005AD1284601F032FE002855D195F8143425
:109E600095F8581406FB035393F8F12100294BD1C0
:109E7000012A49D993ED837AF0EE087AB4EEE77AB5
:109E8000F1EE10FA40DBDFED2E7AB0EEE80AB4EE28
:109E9000E70AF1EE10FA37D5236993B377F004F8A7
:109EA0002369C01AB0F5FA7F32D8237A002B3CD050
:109EB000244DA5F1200696E80F0085E80F0094EDEB
:109EC000038AA5F110013046B8EEC88A0DF084FD72
:109ED00028EE098ADFED1C0A284670EE200AB0EE53
:109EE000480A0DF0EFFD194B9FED190AD3F8400514
:109EF000BDEC048B03682A4631469B6ABDE870407E
:109F0000184776F0D1FF20612369002BCDD0C5E73B
:109F1000104D84ED038A012323720023236105F190
:109F200010030FCB85E80F00BFE7BDEC048B70BDBD
:109F3000382C00200000C84235FA8E3C0AD7233C5A
:109F4000DB0FC93F3C82002000007A44385C0020CF
:109F5000000000001C820020052070470048704768
:109F600094E20B0800487047A4E20B0801207047F8
:109F700038B5474D2DED028BD5F8540B9FED458A32
:109F800051F074FFD5F86C3B07EE903AF8EEE77AA3
:109F900005F5405427EE800AA5F50050BDEEC00A35
:109FA00084EDE90AF9F7A6F9D5F8580B51F05EFFF0
:109FB000B5EEC00AF1EE10FADABF05F53763D3ED5E
:109FC000007AD5EDB37A3448CBBF20EE270A20EED5
:109FD000270A20EE080A28EE400ABDEEC00A84EDEA
:109FE000EA0AF9F757F995EDB37AD4F8A80305F51D
:109FF000376327EE087AD3ED007A27EE888AFDEEE4
:10A00000C77A17EE902AFDEEC87A17EE901A1EF066
:10A010002BFEC4F8A8032048FDF7F8FF20B1D4F8C0
:10A02000A8335B42C4F8A8331C4B93F8203D53B1CE
:10A0300095F92033022B06D1002301214620C4E9E3
:10A04000E93353F073FD51F021FE5F2152F0C6FE5B
:10A05000D8B152F093FE022817D194F84133A3B936
:10A0600094EDC57AD5EDDB7AB4EEE77AF1EE10FA2D
:10A070000BD5012384F84133BDEC028B084A094813
:10A08000BDE83840042149F043BABDEC028B38BD2D
:10A09000384C00200000C842382C0020386C0020CA
:10A0A000ACE20B08505F002010B50446FFF746F8FD
:10A0B0002046BDE81040FFF7ABB90000062070470E
:10A0C0000048704728E30B080048704738E30B0846
:10A0D0000120704701207047012070470120704720
:10A0E0007047000008B50248FBF7E0FE012008BDFC
:10A0F000382C002038B50E4C04F50055D5F8540B1B
:10A1000051F0B4FE05F66C32D2ED007AF8EEE77A43
:10A1100004F5A04327EE800A2046BDEEC00A83ED79
:10A12000E90AF9F7E7F82046BDE8384001F06EB9D2
:10A13000382C00200F20704700487047ACE30B0814
:10A1400000487047B4E30B080120704701207047B6
:10A150000120704701207047012070477FB50B4DEB
:10A1600005F54053002283F8122305F5AB43743301
:10A1700006460FCB6C4684E80F0000232846B360E8
:10A180002146FCF78FFB012004B070BD382C002065
:10A1900010B53B4CD4F86033002B2CDD76F084FEF8
:10A1A000D4F86033C01A40F6B733984223D8A4F5E8
:10A1B0004053D4F85403D3F86C2B51421EF054FD95
:10A1C000C4F8A403A4F5A040F9F794F8D4F86433D4
:10A1D000002B14DC2B48F9F72DF82B4890F812339C
:10A1E00093B30121A0F5405001F0F6FFBDE8104007
:10A1F000462053F041B92348F9F710F9E6E776F025
:10A2000053FED4F86433C01A40F6B7339842E1D80D
:10A210001E4BDFED1F6A93EDB37AD4F8580303F5B4
:10A220003763D3ED007A27EE267A67EEA67ABDEE85
:10A23000C77AFDEEE77A17EE102A17EE901A1EF095
:10A2400013FDC4F8A803C8E7A0F5805090F9AB321D
:10A25000012B04DCBDE810400A48F8F7DBBDD4F858
:10A260007033002BF6D076F01FFED4F87033C01A8E
:10A2700040F6B7339842EDD894EDDB0AB6E700BF5D
:10A28000387C0020382C0020385C0020384C00201E
:10A290000000C842D0ED027A0348FCEEE77A17EEE0
:10A2A000903A99B201F048BA382C002084B010B529
:10A2B00003AC84E80E000B4821466F22FCF738FA05
:10A2C0009DF80C1011F0040102D120460DF0ECF8BD
:10A2D00004482146FCF7E6FABDE81040012004B02E
:10A2E000704700BF382C0020B0EEC00AFDEEC07AE7
:10A2F00038B54FF6FF7205460C4617EE900A00215E
:10A300001EF0B2FC07EE900A002CF8EEE77A054B3F
:10A31000C5ED027A14BF4FF0FF32012283F8BC254D
:10A3200038BD00BF387C0020FEF79CBE0C20704773
:10A330000048704728E40B0800487047B5490D08ED
:10A3400001207047012070470120704701207047AD
:10A350000120704708B50C48FDF7E6F80A480B499C
:10A36000FBF7CEFE0848F8F7C7FA40B106484FF4AD
:10A370008051F8F7EBF810B10348FBF797FD02485E
:10A3800000F0BEFD012008BD382C00203C820020DA
:10A3900008B50D48F9F742F80B48F8F7ADFA50B197
:10A3A00009484FF48051F8F7D1F820B1BDE80840D2
:10A3B000054801F02BB80448F8F73CFFBDE8084019
:10A3C0000148F8F727BD00BF382C002008B50A481F
:10A3D0004FF48051F8F7BAF838B108480022D0F8A5
:10A3E000141600F204600CF0CDFFBDE808400248EE
:10A3F000002101F0A1B900BF382C0020387C0020DA
:10A40000881A10B51EF058FB104BD3F8B825002859
:10A41000B8BF4042002AB8BF524248F6A041B2FB42
:10A42000F1F24FF47A7102FB011188420CDC93F8CF
:10A430000426D20606D503F2046403F2F4530FCBCC
:10A4400084E80F00012000E0002010BD387C0020CF
:10A4500084B070B52DED048B86B00FAD85E80E008D
:10A460004E4CDFED4F8A0646D4F8400504F5005403
:10A4700004F5BA6393ED000A0368B0EEC00A5B6AA4
:10A480009847B4EEE80AF1EE10FAB0EE408A07DA27
:10A49000012006B0BDEC048BBDE8704004B07047ED
:10A4A000404928460DF0A4F902A8CDED030A8DED30
:10A4B000020A20F0A1FC04A88DED040AB0EE480ABF
:10A4C000CDED050A20F092FB13A928468DED000A78
:10A4D000CDED010A0DF08CF902A88DED020ACDED4B
:10A4E000030A20F02FFCB4EEE80AF1EE10FACFDBFD
:10A4F000B4EEC08AF1EE10FA9FED2B9ADFED2B8AB5
:10A50000DFED2B9A2BD802A8694620F05FFB04A848
:10A510008DED040ACDED050A20F0CAFB684620EE59
:10A52000098A20F0C5FB94F9BC3507EE903AF8EEA5
:10A53000E77A28EE288AA7EEA90A1EF0E1FA20EEB3
:10A54000090ABDEEC88A20EE280A18EE101AFDEEA0
:10A55000C07A304617EE902AFFF752FF99E738EE9F
:10A56000400A38EE088A80EE080A97F069F902A8D6
:10A57000B0EE408A20F09CFB94F9BC35F0EE007AF6
:10A58000B0EE697AA8EE677A07EE903AF8EEE77ACD
:10A59000A7EE270A1EF0B4FAC0E700BF385C00201F
:10A5A000000000342C820020E02E65420000C842EA
:10A5B000DB0FC93F10B504460848F8F79DF920B9EC
:10A5C0002046BDE81040FEF74DBD04484FF48051D1
:10A5D000F7F7BCFF0028F3D010BD00BF382C0020D7
:10A5E00000207047004870479CE40B080048704703
:10A5F000A4E40B08002070470020704738B5154CC4
:10A6000005460021204601F01DFC042052F034FFD5
:10A610000021204601F020FC132052F02DFF0021E4
:10A62000204601F023FC2846FEF7E0FE20460121EB
:10A6300001F0D2FD462052F01FFF6B6804F5A044E4
:10A64000D3F8F831C4F8A4336B68D3F8FC31C4F8FC
:10A65000A83338BD382C0020FEF7A8BE0B20704769
:10A66000004870475FDD0B080048704718E50B088D
:10A67000012070470120704701207047002070477B
:10A6800070B50B4E06F5A04505F2F4530FCB05F25D
:10A69000E45484E80F003046FBF7C2FB0146304625
:10A6A000FCF7CEF9002385F86836012070BD00BFA5
:10A6B000382C002038B53048F8F7B0FE2E48F8F7AF
:10A6C000B9FD2D48F8F7A6FB2B481021F7F73EFF00
:10A6D000E0B12A4AD2F8F835D2F808269342D4BF1E
:10A6E00000230123254C94F8682672B973B304F251
:10A6F000F4530FCB04F2E45585E80F00A4F5A04015
:10A70000FBF7D0FD012384F8683638BD1C4AB2F946
:10A710003C1B0029F9DD02F540529FED1A7AD2F870
:10A72000F835D2F8E8259B1A07EE903AF8EEE77A6A
:10A7300067EE877A07EE101AB8EEC77AF4EEC77A9A
:10A74000F1EE10FACCBF01230023CBE7A4F5405370
:10A75000642193F97C23D4F8A40312FB01F2D3F80B
:10A760006C1B8A42A8BF0A465142C3F86C2B1EF0EC
:10A770007BFAC4F8A403C8E7382C0020387C0020FA
:10A78000384C00200AD7233C38B52B4DB5F910338F
:10A7900083EAE371A1EBE37189B205F5405431B16D
:10A7A000002BB4BF4FF0FF33012384F8BC3523489E
:10A7B00000F0C2FF94F84233F3B995F9EB32022B63
:10A7C0001BD11F4D95F8353D9BB11E49A1F5107069
:10A7D00023F0DCFF68B1012384F8ED33282205F56E
:10A7E0004A61A5F5804003F041F828B9002384F8B8
:10A7F000ED33012384F8423338BD012B0CD10F48CF
:10A8000000F0E6FE40B10D48FBF7B6FC0028B8BFEB
:10A810004042B0F57A7FD4DB95F9EB32042BEBD1D3
:10A82000074D95F8353D002BE3D00649A1F5107092
:10A8300024F028F8CEE700BF384C0020382C002048
:10A84000386C00202C82002002207047004870479E
:10A850008CE50B0800487047AA490D08024B0022FE
:10A86000C3E9E922704700BF387C002038B5094DA4
:10A8700004462846F8F7B6F82846F8F751F9204676
:10A88000F8F766F92846F8F769FC2046BDE8384035
:10A89000FEF7BEBD382C00200D20704700487047E1
:10A8A00004E60B08004870470CE60B0801207047CF
:10A8B00001207047012070470023C37480F82430C2
:10A8C000012070470148002100F036BF382C0020DD
:10A8D000F0B5B54CD4F80026D4F8FC352DED088B36
:10A8E0001343D4F8F825134389B005460FD1AF4878
:10A8F000F8F794FDAD48F8F79DFC9FEDAD0A4620B2
:10A9000009B0BDEC088BBDE8F04052F0B5BD06F0D3
:10A9100023FD90F87C32DB07E9D5B5F90830E97CF6
:10A9200009EE103AB5F9103008EE903AB8EEC99A2F
:10A93000F8EEE88A002940F0D7809FED9EAA29EE24
:10A940000ABA0122FDEECB7AA4F5A040C4EDC37A89
:10A95000FBF792FA686800F57F700790B0EE408AC6
:10A9600020F0A6F9DFED947A20EE270A1EF046F8D3
:10A970000798F0EE409A20F0E5F9A4F5A040F0EE3B
:10A9800040AAFEF789F8002879D104F2F45696E837
:10A990000F0005F1140787E80F0096E80F0004F296
:10A9A000E45787E80F0004F2046787E80F00D4F843
:10A9B0000836824807EE903AF8EEE77AF0EE680A39
:10A9C00077EE8B7AB0EE690AFDEEE77A17EE903AF1
:10A9D000C4F808360DF076F8002384F8793395F939
:10A9E0001230724803EB830303EB83039B000121C6
:10A9F000A4F83A33F7F7F4FA94F88873002F73D178
:10AA00006F4B9FED707AB3F9B43207EE903AF8EEDF
:10AA1000E77A67EE877AF4EEE7AAF1EE10FA63DDE3
:10AA20004FF042FC064619EE900AF5F765FDCDE9B8
:10AA3000040118EE900AF5F75FFDCDE9020119EE69
:10AA4000100AF5F759FD604ACDE9000106213046AC
:10AA500048F05EFD76F028FAC4F8F872C4F8E40213
:10AA600076F022FA0123C4F8F40229EE8A0AEB7484
:10AA70001DF0EEFFBDEEC00A84EDBF0A34E076F0B3
:10AA800013FAD4F89C33C01A42F2107398427FF63E
:10AA90007CAFF0EE087AF4EEE7AAF1EE10FA7FF759
:10AAA00074AFBCEEC88A04F2046718EE103A9BB289
:10AAB00008EE103AB8EEC88A04F2F456B4EEC89A1A
:10AAC000F1EE10FA46D84FF0EFFB404A062148F06D
:10AAD0001FFD96E80F0087E80F000123EB740321A8
:10AAE000A4F5A040F7F77CFA304803F0C1FC28B188
:10AAF0002E480321F7F774FA0023EB74D4F890334F
:10AB0000012B40F0B480D4F8F835AA699FED29AA4A
:10AB10009B1A07EE903AD4F8FC320133F8EEE79A2C
:10AB20005CD0DFED2B7AE9EE0A7AF4EEE79AF1EEEB
:10AB300010FA0ADA274905F114000CF04DFFF4EE83
:10AB4000C08AF1EE10FA00F2928018480321F7F75C
:10AB500047FA8CE04FF0A8FB1F4A062148F0D8FCCA
:10AB600096E80F0005F1140C8CE80F0096E80F0032
:10AB700087E80F00D4F8083607EE903A39EE488A95
:10AB8000F8EEE77AF0EE680AE8EE0A7A3846B0EEB8
:10AB9000690AFDEEE77A17EE903AC4F808360CF031
:10ABA00091FF0121E9749BE7387C0020382C0020BC
:10ABB000000000000000C842E02E65423C820020F8
:10ABC000384C00209A99993E55E60B0814E60B087C
:10ABD000000048C32C82002030E60B08B5F90A308B
:10ABE00007EE903AF8EEE77A05F1140667EE8A7AF6
:10ABF000F4EEE79AF1EE10FA53DB434930460CF0DD
:10AC0000BBFDDFED427AB6EE008AA0EE278A96E819
:10AC10000F00BDEEC88A9FED3E0AB8EEC88A04F266
:10AC2000046728EE008A87E80F00F0EE680A3948CA
:10AC3000B0EE480A0CF046FFD4F8083607EE903A1A
:10AC4000F8EEE77A28EE0A0AE9EE0A7AFDEEE77AEC
:10AC500017EE903AC4F808361DF0FAFEBDEEC00AB1
:10AC600084EDBF0AD4F89033012B3FF45AAF2A4841
:10AC700003F0DEFB18B128480321F7F7B1F9D4F847
:10AC80009033012B17D1244803F074F9224803F0C4
:10AC9000ADFA214809B0BDEC088BBDE8F04003F0E7
:10ACA000C7B9194930460CF097FEF4EEC08AF1EEB0
:10ACB00010FAA2D9D6E795F824302BB917485EF0E0
:10ACC0006FFE012385F824301348F8F7A7FB1248DC
:10ACD000F8F7B0FA1048F8F79DF8114890F81433D7
:10ACE0006BB1002380F8143333220221A0F54050C9
:10ACF00009B0BDEC088BBDE8F040FDF735BB09B0ED
:10AD0000BDEC088BF0BD00BF2C820020A00CB34529
:10AD10000AD7233C3C820020382C0020884D00209C
:10AD2000385C002010B50446FEF774FA2046054B47
:10AD300040F8143B0CF020FB204603493EF03AFF5C
:10AD4000204610BD08E70B08A0E60B08032070475B
:10AD5000004870476CE70B080048704778E70B081D
:10AD6000F8B52A4D06460027A5F54050A5F8107302
:10AD7000F8F7C0FA7368A5F58052D3F8F811D2F845
:10AD80006C3B994205F500541FDBC4F8A43373688B
:10AD900092EDB37AD3ED7F6A9FED1D6AF8EEE66A15
:10ADA00027EE067AF4EEC76AF1EE10FA16DBBDEE76
:10ADB000C77A84EDEA7A1748FDF728F920B1D4F86C
:10ADC000A8335B42C4F8A833F8BD5B429942DCDD8E
:10ADD000012385F81033C4F8A473D8E702F537626D
:10ADE000D2ED007A67EE867AF4EEE76AF1EE10FAB9
:10ADF00089BF0123FDEEE77A85F81133002394BF64
:10AE0000C4EDEA7AC4F8A833D5E700BF385C002067
:10AE10000000C842382C002070B500212DED028BB7
:10AE200004463448344D01F00DF832480021F0EE6C
:10AE3000408A01F011F895F81033B0EE408AD3B192
:10AE4000B0EE680A042052F017FB95F8113393B363
:10AE5000B0EE480A132052F00FFB2648002101F003
:10AE600005F82046FEF7C2FABDEC028B2046BDE88D
:10AE70007040FEF7CDBA05F50056A5F54050F7F73E
:10AE8000B1FDD6F8A433002B0CDCD6F8A433002B8C
:10AE9000DBDA042052F004FBB4EEE80AF1EE10FA1B
:10AEA000CED4D2E7042052F0FBFAB4EEE80AF1EE79
:10AEB00010FAEADDC4E7114D0E48F7F731FED5F878
:10AEC000A833002B0CDCD5F8A833002BC5DA1320EF
:10AED00052F0E6FAB4EEC80AF1EE10FAB8D4BCE7C4
:10AEE000132052F0DDFAB4EEC80AF1EE10FAEADDF2
:10AEF000AEE700BF382C0020385C0020387C0020F2
:10AF000000F5A0400023C0F8B835C0F8B43580F88B
:10AF1000BD3580F8BE35704700F58043D3F83C3D21
:10AF2000002BCBBF07EE903A00F50050B8EEE70AD1
:10AF3000DFED037ADCBF90EDAE0A20EE270A704702
:10AF40000000C8422DE9F0412DED028B00F5955728
:10AF500084B09FEDC98A1037054603A938468DEDA8
:10AF6000038A05F0DDFFB0B19FEDC47ADDED037A11
:10AF700005F5A04367EE877AD3EDEC6A9FEDC07AC2
:10AF8000E6EE877AF4EE487AF1EE10FA48BFF0EE7A
:10AF9000487AC3EDEC7A2846F7F700FC05F58044C3
:10AFA000B0EE408AF0EE000A9FEDB30A1DF094FE69
:10AFB00004F65453D3ED007A38EE678A05F500564F
:10AFC000E0EE087AC3ED007A94F8203D002B40F0C3
:10AFD0009380D4F80C2D05F598437C339A4205D024
:10AFE00005F5994304339A4240F0868008212846AB
:10AFF000F7F7ACFA804630B1D6EDAE7A9FEDA17A84
:10B0000067EE877A73E002212846F7F79FFA014638
:10B01000002855D0D6F85C3B1B8B2846414608EEED
:10B02000103A01F0D9F8D6F85C0B4369B8EE488ABB
:10B03000B0EE401A2BB3012B28D0DFED937AF0EE5F
:10B04000671A96EDAE0A9FED8F7AF4EEC17AF1EEB3
:10B0500010FA20EE070A4FF0640124DBB6F8B422A0
:10B0600012FB01F2B0EE672A07EE902AF0EE400ADA
:10B07000B8EEE70A1DF08AFCBDEEC00A10EE103AE9
:10B08000ECE0DFED817AF1EE481ADAE78DED010AA6
:10B0900050F05EFE07EE900ADFED7B1A9DED011A7F
:10B0A000F8EEE77ACDE7B6F8B63213FB01F300EE1F
:10B0B000903AB0EE482AF8EEE00AF0EE671AD9E7C7
:10B0C000B6F9B422B6F9B6329B1A07EE903A284682
:10B0D000B8EEE78A01F080F8B6F8B432642213FBC8
:10B0E00002F307EE903AF8EEE77AE8EE007AFDEE2A
:10B0F000E77A17EE903AB1E005F5A043D3F8903324
:10B10000042B40F0A08005F5A9404C3073F0ACFF53
:10B11000C4F8380DD4F80C0D03689B6B98470028D1
:10B120005ED094F84C3D002B5AD0D4F80C3D05F578
:10B1300098453435AB4253D0D4F8383D9FED537A1F
:10B1400007EE903AD4F8483DF8EEE77A384627EE15
:10B15000878A07EE903AF8EEE78A68EE878A06F06B
:10B16000EBF8C8EE807A04F555639DED037A77EE2F
:10B17000877AB6EE007AB4EEE78AF1EE10FA4CBFA9
:10B1800077EEC87ADFED407A77EE877A93ED007A32
:10B19000FDEEE77AF8EEE77AB4EEE77AF1EE10FA30
:10B1A0000ADD37EE676ADFED3A6AB4EE666AF1EE01
:10B1B00010FA48BFF0EE477A04F55563C3ED007A04
:10B1C000D4F8383DDFED2F6A07EE103AB8EEC77AB3
:10B1D000A7EEA67ABDEEC77A17EE103AC4F8383D4E
:10B1E000D4F80C0D03681B6B984740B1B4F9442D9B
:10B1F000002AC2BFD4F8383D9B18C4F8383DB6F9D0
:10B20000B622B6F9B412D4F8380D64235A43594320
:10B210001DF02AFDC4F8380D06F60843D6F8180CC0
:10B2200093ED4A8A06F088F8C8EE007A04F5546473
:10B230009DED037A77EEC77AC4ED007A04B0BDECD9
:10B24000028BBDE8F081D4F80C2D05F59943483305
:10B250009A4206D1D4F83C3D002B02DDC4F8383DBB
:10B2600058E705F5994320339A427FF4C5AE284646
:10B27000FFF752FE00E700BFCDCCCC3DCDCC4C3E1D
:10B28000CDCC4C3F0000C842000000000AD7233C50
:10B290009A99993F30B500F5955587B01035002340
:10B2A0000446284603930493059304F009FF0028FD
:10B2B00043D003A9284605F061FE00283DD004F5DF
:10B2C000AE5393ED047ADFED216A8DED017AB0EE95
:10B2D000C77AD3ED077AB4EEE67AF1EE10FACDED47
:10B2E000027A06D5F0EEE77AF4EEE67AF1EE10FA9D
:10B2F0002AD401A81FF078FD03A901A81FF0BCFC07
:10B3000004F5005393EDB07AB5EEC07AF1EE10FA81
:10B31000C4BFDFED0F7A27EEC00A04F58044C6BF34
:10B32000A7EE270A0123002384F84C3DCABFFDEE97
:10B33000C07A002317EE903A04E004F5804400231D
:10B3400084F84C3DC4F8483D07B030BD00000034DF
:10B350000000C8422DE9F0412DED028B00F5A0461A
:10B3600007EE901AD6F8C03500F5AC45B8EE678AFE
:10B370000446043500F54057BBBB00F58043D3F8C5
:10B380000C2D00F5994320339A4204D000F59943DF
:10B3900048339A4229D196F8403333B304F5AB4091
:10B3A000294674300CF018FBD7F840050368F0EE1E
:10B3B000408A5B6AB0EE480A9847F0EE087A60EE81
:10B3C000277AF4EEE78AF1EE10FA0EDDBDEC028B7F
:10B3D000D7F840059FED0C0A036804F5AB412A46F7
:10B3E0009B6ABDE8F04164311847B0EE480ABDECF5
:10B3F000028BD7F8400596F9BC2503682946DB6A1D
:10B40000BDE8F041184700BF0000000070B50446D9
:10B410002DED028B04F5A04575F03EFDD5F82036E4
:10B42000474AC31A9342064672D907EE903AB8EEDD
:10B43000670ADFED447A9FED441ADFED440A20EEFF
:10B44000270A40F295101DF06FFBC5F8206604F541
:10B450000056DFED3F7AD6F8583BB3F9083008EED6
:10B46000103A96F91233B8EEC88AF0EE408A28EE08
:10B47000278A0BB1B1EE488A9FED367ADFED367A36
:10B48000B4EEC78AF1EE10FA52DA05F21C63D3ED7E
:10B49000006AF4EEC76AF1EE10FAB4EEE78AACBFC8
:10B4A00001230023F1EE10FA3FD905F21C6292ED60
:10B4B000007AB4EEE77AF1EE10FA36D82046FAF7C1
:10B4C000F5FC96F9133300EE103A06F5436306F6E1
:10B4D0003846D6ED000A93ED001AB8EEC00A40F2E5
:10B4E000A710F1EE600A20EE080A1DF01DFB28EE01
:10B4F000800ADFED1A8A20EE280A2046FDEEC07A87
:10B5000005F21C6517EE901AFAF7EAFC85ED008A41
:10B510002046FAF7FFFC2046F7F77CFCBDEC028BD7
:10B520002046BDE87040F7F785BE002BC6D1C8E7BE
:10B53000B4EEE78AF1EE10FAC3D90023B5E700BFF5
:10B540009F860100BD3786359A99193ECDCCCC3DFA
:10B550005304693900000034000000B40000C84200
:10B5600070B5044600F5A7404FF0FF31343022F0AB
:10B5700091FA431C054604F5A04603D1114BC6F8C9
:10B58000183370BD04F5AC4104F5AB4004316430B0
:10B590000CF0F2F89FED0C7AF6EE007AE0EE077A06
:10B5A000FDEEE77A17EE900A281A1DF085FA07EEED
:10B5B000900A9FED067AF8EEE77A67EE877AC6ED95
:10B5C000C67ADEE70000B442A00CB3450AD7233C9C
:10B5D00000F54050D0F8400503689B6B1847000009
:10B5E00070B500F540530446D3F8400503681B6965
:10B5F000984706462046FFF7EBFF04F5A0440546B2
:10B60000D4F8B80568BB3DB1D4F8F835C4F8C435F2
:10B61000274BC4F8C8350120C4F8B0651DF04CFABA
:10B62000D4F8B82594F9BC1500FB0123C4F8B8354B
:10B63000DDB1D4F81416D4F8F825521A02F2F31238
:10B6400040F2E6318A4210D8012203F5D23384F861
:10B65000BD2503F5F073002284F8BE25C4F8C83573
:10B6600070BDD4F8B035F01AD6E794F8BD25002A9D
:10B67000F6D1002BD4F8C825B8BF5B429342EFDB6C
:10B68000D4F8F815D4F8C435C4F8C415CB1A03F2AD
:10B69000F31340F2E630834202F5D2328CBF00232E
:10B6A000012302F5F07284F8BE35C4F8C825D7E747
:10B6B000E0A501002DE9F04100F58048044698F826
:10B6C000353DA3B300F5A045D5F80C3613B9D5F830
:10B6D000103663B304F5AB4604F5AC472046743628
:10B6E0000437FBF745F8394630460CF075F904F598
:10B6F000AB413A466431304685EDC90A0CF0A2F8F8
:10B70000DFED0C0A85EDCA0A7620B7EE001A1DF0AF
:10B710000BFA04F53053204683ED730AFFF760FF00
:10B72000D8F80C0D0368BDE8F041DB6A1847BDE8A6
:10B73000F08100BF00000000012938B5044600F583
:10B74000A04512D800F5005395F80426B3F9DE326F
:10B7500083EAE371A1EBE37189B2012998BF3C212F
:10B76000920731D5FF2385F8BC3507EE901AF8EE25
:10B77000677A05F5BA63C3ED007A2046FFF7EAFD64
:10B78000D5F8C03533BB2046FFF722FF40B995ED11
:10B79000CA7AF7EE007AB4EEE77AF1EE10FA19DD24
:10B7A00075F082FB04F58043C5F8C005D3F80C0D95
:10B7B00003681B6A984768B104F54C500021BDE846
:10B7C000384018304CF088B8002BB4BF4FF0FF332E
:10B7D0000123C8E738BD000010B500F5A9442C349A
:10B7E000204659F043FD2046BDE8104059F0AEBD5B
:10B7F00010B500F5A043044693F8C0349A0717D457
:10B800005B0700F54C504FF002014CBF094A0A4A51
:10B81000183047F07DFE04F5A9402C3059F0FAFCB1
:10B8200004F52C500121BDE81040043060F096B8BA
:10B8300010BD00BFECE70B0806E80B0870B500F57B
:10B84000A046054696F9AC449CB196F8C034C3F3C3
:10B8500080045B0729D4B6F9B234002B0BDC2846F0
:10B86000FFF7C6FF05F52C500121043060F076F893
:10B870000124204670BD2146FAF714FBB6F9B23414
:10B8800007EE903AF8EEE77AB4EEE70AF1EE10FA36
:10B89000E5D5D6F82C33002BE1D005F54C50044A01
:10B8A0000421183047F034FEE3E70024E1E700BF4D
:10B8B0001CE80B0808B52DED028B08EE901A30B38A
:10B8C000F2B1B0F9083008EE103AB8EEC88AF8EED6
:10B8D000E88A9FED100ADFED100A28EE800ADFEDFE
:10B8E0000F8A4FF4D470B7EE001A1DF01DF9C8EEA0
:10B8F000280A1DF075F820EE280ABDEC028B08BD61
:10B9000050F0AAFA07EE900AB8EEE78ADFE79FED5B
:10B91000020AF2E70AD7233C0000000000A08C4591
:10B9200037B500F50054054694F93F33002B52D04B
:10B9300050F0ACF950F0A0F9C4F8540B50F0A6F94F
:10B9400050F086F9C4F8580B50F0A0F950F08AF97D
:10B95000C4F85C0B50F09AF950F08EF941F2941152
:10B96000C4F8600BD4F8540B50F0DAF9D4F8580B43
:10B9700041F2941150F0D4F9D4F8600B41F29411D3
:10B9800050F0CEF9284600F021FC48BBD4F85C0BFF
:10B99000642150F0C1F950F079F9D02151F01EFA2C
:10B9A000C4F8640B50F072F9D22151F017FAC4F8C0
:10B9B000680B05F51B501C304921019051F09CFF8C
:10B9C00001984A2151F098FF0198462103B0BDE843
:10B9D000304051F091BF50F059F950F02FF9ABE7DA
:10B9E00005F5A043D4F85C0B93F89C37642173B140
:10B9F00050F092F96421462051F076FE64214920EE
:10BA000051F072FE64214A2051F06EFEC3E750F0FF
:10BA100087F9EFE710B500F500541E21D4F8540B58
:10BA200050F082F9D4F8580B1E2150F07DF9D4F86B
:10BA3000600B1E2150F078F9D4F85C0B1E21BDE894
:10BA4000104050F071B9000007B500F0BFFB01468F
:10BA500058B90190462051F069FD0199492051F0F3
:10BA600065FD01994A2051F061FD0021042052F04A
:10BA70002FF80021132052F02BF80021462052F01D
:10BA800027F80021492052F023F800214A2052F0E3
:10BA90001FF80021152003B05DF804EB52F018B830
:10BAA00010B5044652F05AFA51F0AAFE204601F0B1
:10BAB000BDFCBDE8104052F059B9000038B500F5A2
:10BAC0000055044695F93F330BB1002038BD0121E4
:10BAD000F6F73CFD90B104F58043D3F80C2D04F546
:10BAE00099435C339A4209D004F598433C339A4217
:10BAF00004D004F598434C339A42E6D12046F6F739
:10BB0000FBFE0028E1D0D5F8603BB3F90800DDE783
:10BB100038B52DED028B00F5804393F8203D002BC6
:10BB200040F0B9805D4A00F59943D2F80C2D5C33A2
:10BB300000F54C549A4204F1180408D0584A0321E5
:10BB4000BDEC028B2046BDE8384047F0E1BC00F573
:10BB500000559FED546AD5F8542BB2F90830002BEC
:10BB6000B8BF5B429BB207EE903A138B06EE903A59
:10BB7000F8EEE66AF8EEE77A66EE866AF4EEE67AC2
:10BB8000F1EE10FA17DCD5F8582BB2F90830002B7B
:10BB9000B8BF5B429BB207EE903A138B07EE103AA8
:10BBA000B8EEC77AF8EEE77A27EE067AF4EEC77AAF
:10BBB000F1EE10FA01DD3C4AC1E700F5AE50043069
:10BBC0001FF034FEDFED397A20EE270AF3EE0E7A0D
:10BBD000B4EEE70AF1EE10FA01DD354AAFE70420D2
:10BBE00051F02EFF132051F02BFF152051F028FFAC
:10BBF0004D2051F025FF4E2051F022FF4F2051F0F3
:10BC00001FFF502051F01CFF152051F049FC9FED03
:10BC1000298AB0EEC00AB4EEC80AF1EE10FA0BD5CC
:10BC2000102051F00DFF562051F00AFF112051F065
:10BC300007FF572051F004FF032051F041FCB0EE04
:10BC4000C00AB4EEC80AF1EE10FA0FD5022051F086
:10BC500037FCB0EEC00AB4EEC80AF1EE10FA05D512
:10BC6000182051F0EDFE192051F0EAFED5F8540BE2
:10BC7000811D0C303EF064FED5F8580B811D0C3050
:10BC80003EF05EFED5F8600B811D0C303EF058FE94
:10BC9000094A052154E7BDEC028B38BD386C002001
:10BCA00030E80B08CDCC4C3E50E80B08E02E654246
:10BCB00078E80B080000003494E80B0810B500F594
:10BCC000005494F916339BB1D4F85C0B50F03AF859
:10BCD000D4F85C2BB4F9183330B1B2F906009842AD
:10BCE000ACBF0020012010BDB2F906008342F7E787
:10BCF0000120F8E710B50446FFF7E0FF60B104F556
:10BD0000804475F0D1F8D4F82C3DC01AB0F57A7F94
:10BD100094BF0020012010BD0120FCE770B505464E
:10BD2000FFF7E8FF05F5005408B3D4F8543B9A89AF
:10BD3000DA80D4F8583B9A89DA80D4F8603B9A8943
:10BD4000DA80D4F8543B00261E81D4F8583B1E817B
:10BD5000D4F8603B1E8105F58043D3F80C0DC3F881
:10BD6000446D03685B689847D4F85C3B1E8105F519
:10BD7000AD4074306DF004FC80B300264FF086FFB8
:10BD8000437A13B94FF082FF837A94F91623012A7C
:10BD900023D106B10BB32846FFF7ACFF05F580446D
:10BDA00094F8263D38B30133DBB20A2B84F8263DE4
:10BDB0000CD105F54C501F4B1F4A0421183047F099
:10BDC000A7FB1E4A012384F8203D937294F8263D78
:10BDD0000A2B02D90A2384F8263D70BD2846FCF7B9
:10BDE0005BFE0028C9D14FF051FF4FF013FF061E34
:10BDF00018BF0126C2E7002BEFD0013BDBB2032BBB
:10BE000088BF032384F8263D94F8263D012B09D1F1
:10BE100005F54C500A4B084ABDE870400421183023
:10BE200047F076BB002BD8D1044A84F8203D9372AA
:10BE3000D3E700BF636C0D08A4E80B0895840020CD
:10BE400087EA0B0800F500500A4690F93E1BD0F82F
:10BE5000540BFFF72FBD000000F500500A4690F983
:10BE60003F1BD0F8580BFFF725BD000000F5005030
:10BE70000A4690F9401BD0F8600BFFF71BBD00008D
:10BE800010B54FF480610446F6F760FB04F50053EB
:10BE900028B1BDE81040D3F85C0B50F0D9B8BDE82C
:10BEA0001040D3F85C0B50F0DDB80000F8B500F599
:10BEB000005300F5A045D3F8603BB3F9087017B9FB
:10BEC000012385F8383700F5AD44743420466DF011
:10BED00057FB0646E0B9B7F57A6F2BDD74F0E4FF47
:10BEE000D5F83437074683B1C31A40F6B7329342C8
:10BEF0000DD9012231462046F5F714FDC5F8346707
:10BF000085F83867C5F8D47201E0C5F83407F8BD84
:10BF100017F57A6F0EDA74F0C7FFD5F834376BB1C6
:10BF2000C01A40F6B7339842F1D9012200212046C9
:10BF3000F5F71EFD0023C5F83437E8E7C5F83407E8
:10BF4000E5E7000070B52DED028B04464FF09EFE34
:10BF50004FF056FD30B9BDEC028B2046BDE8704075
:10BF6000FFF7DCBE04F5804595F8203D1BB974F061
:10BF70009BFFC5F8300D2046FFF7A0FE18B174F006
:10BF800093FFC5F82C0D2046FFF7C8FE2046FCF7AE
:10BF900013FC04F500560023C5F8443D96F91A3306
:10BFA00063B3D6F85C3BB3F90830322B26DD28B3F7
:10BFB000323B1BB207EE903A04F59550B8EEE78A93
:10BFC000DFED207A103028EE278A03F0B3FF38B374
:10BFD000B6F9B63296EDAE7A07EE903AF8EEE77A19
:10BFE00077EEC77A27EE888ADFED177A28EE278A60
:10BFF000BDEEC88A18EE103AA5F8443D2046FFF77A
:10C0000055FFD5F80C0D03685B689847BDEC028BB3
:10C01000014604F5AE404030BDE8704052F092BB9E
:10C0200096F9A93296F9AB229B1A07EE903AF8EEF0
:10C03000E77A27EE888ABDEEC88A18EE103AA5F88E
:10C04000463DDBE70AD7A33C0000C84270B500F5C7
:10C0500000540546D4F81C330BB9002041E094F994
:10C06000A832002BF9DA00F58043D3F80C0D0368F1
:10C070005B6898470138172832D801A353F820F09D
:10C080007DC10108B9C10108E1C00108AFC10108C3
:10C09000A5C1010891C1010887C10108E1C00108DB
:10C0A000E1C00108E5C0010873C1010869C10108C8
:10C0B0005BC001089BC101089BC10108E1C00108E8
:10C0C000E1C00108E1C00108E1C00108E1C00108C8
:10C0D000E1C00108E1C00108E1C00108C3C10108D5
:10C0E000012070BD05F5A045B5F8F263162EB4D059
:10C0F000D4F81C1311F0020301F0010205D0A6F1DF
:10C10000150CDCF1000343EB0C0311F0040043EACF
:10C11000020303D0A6F11F046042604143EA00021B
:10C1200011F0080007D01F2E1AD0A6F11100022826
:10C130008CBF0020012011F0100340EA020005D05E
:10C14000102E0FD0A6F1520253425341034311F473
:10C15000006014BF95F8BC13014643EA0100C0E734
:10C160000120E8E70123F1E7D4F81C03C0F34010F5
:10C17000B7E7D4F81C03C0F38010B2E7D4F81C036F
:10C18000C0F3C010ADE7D4F81C03C0F30020A8E74B
:10C19000D4F81C03C0F34020A3E7D4F81C03C0F379
:10C1A00080209EE7D4F81C03C0F3003099E7D4F850
:10C1B0001C03C0F3403094E7D4F81C03C0F3803074
:10C1C0008FE7D4F81C03C0F3C0308AE700F50050B5
:10C1D00090F8A802C009704738B504460D464FF0E4
:10C1E00055FD0368DB689847C8B104F50053D3F8E0
:10C1F0005C0B6DB14FF030FE07EE900AB8EEE70A27
:10C2000004F5A04494F89B370BB1B1EE400A38BD59
:10C21000B0F9083000EE103AB8EEC00AF0E79FED32
:10C22000010AF4E70000000038B52DED028B04464A
:10C230000D464FF02BFD0368DB68984700283FD080
:10C24000214BD3F85C3B5B69012B07D0BDEC028B23
:10C2500029462046BDE83840FFF7BEBF4FF4806155
:10C260002046F6F773F90028F0D004F50053DFED0F
:10C27000177AD3F85C0B93F9AB32028B08EE903A45
:10C2800000EE102AF8EEE88AB8EEC08A68EEA78AB7
:10C290004FF0ECFDB6EE001AA0EE011A04F5A04432
:10C2A000DFED0B0AB0EE680A1CF06CFC94F89B37CB
:10C2B00028EE000A0BB1B1EE400ABDEC028B38BD8E
:10C2C0009FED030AF9E700BF384C00200AD7233C52
:10C2D0000000000010B500F5A0430446D3F89023F9
:10C2E000042A0CD1FAF742F804F5546080EDA70A4D
:10C2F0003EF026FF2046BDE81040FAF7B5B803F23D
:10C30000246393ED000AEFE770B500F5804604461C
:10C31000D6F80C0D03689B6B0D46984748B9D4EDD1
:10C32000460A9FED1C0A64212846BDE8704051F082
:10C3300099B9D6F80C0D04F5994104F50052203155
:10C34000884292F8AA3292F974231FD104F5A041D1
:10C3500091F83C0350B94AB1D3B204F5A041D1F8E9
:10C3600090130139012998BFD3B207E091F948052C
:10C3700060B1D1F89013042908D1C3B207EE903A06
:10C38000D4ED460AB8EE670A6421CDE7002AF5D05D
:10C39000E3E700BF000000002DE9F04100F5804810
:10C3A000044604F59943D8F80C0D5C33984203D148
:10C3B00000252846BDE8F08103689B6B984750B183
:10C3C00004F5A04393F8C05415F0010503D00122F1
:10C3D00083F88823EDE704F5A9404C3072F078FF2C
:10C3E000054608B10125E4E704F5A04696F8883330
:10C3F000002BDDD0D8F80C0D03689B6B984718B95B
:10C40000002386F88833D4E794F8143494F85874E9
:10C41000B02202FB034393F8F121B7BB012A0AD9EA
:10C4200093ED837AF1EE047AB4EEE77AF1EE10FA46
:10C43000ACBF01270027D8F80C2D04F59943203311
:10C440009A4202D196F83C3323B104F59943643300
:10C450009A4240D104F50053204693F96883FCF7D3
:10C460001BFBA0B9204601F013FC0028BAD0002322
:10C4700086F8883394F8712404F58C63242101FB39
:10C480000233DB6AC6F8343393E72F46D3E774F000
:10C490000BFDD6F89C334FF4FA62C01A642313FBE9
:10C4A000082341F28832934238BF13469842D9D9C3
:10C4B0002046F9F7E1FEB0F5FA7FD3DD04F58053AD
:10C4C00041F26E72D3F8AC3403F6B7339342C9D855
:10C4D000002FC7D094E706F22463D3ED007AB2EEC2
:10C4E000047AF0EEE77AF4EEC77AF1EE10FA87DA22
:10C4F000002F3FF477AF04F59550103003F01AFD8C
:10C5000000283FF47DAF04F5005304F5FC5093F888
:10C51000E610183002F02EFFF1EE047AB4EEE70ACE
:10C52000F1EE10FAFFF65EAF6AE70000F8B52DED08
:10C53000048B0446084616461D46BDF9287050F087
:10C54000AFFF04F500543046B0EE408A50F0A8FF2B
:10C55000B4F94423002AF0EE408A37DAC2F16403CA
:10C5600007EE903A9FED207AF8EEE77A67EE877A49
:10C5700060EE278AD4EDD07A9FED1C1ADFED1C0AFD
:10C5800038EEC80ABC2020EE270A1CF0CDFA38EE9F
:10C59000288AB0EE409A94EDD00A9FED141ADFED90
:10C5A000140A28EE000ABD201CF0BEFA2846B0EEA0
:10C5B000408AB0EE490A50F05FFFB0EE480ABDEC89
:10C5C000048B3846BDE8F84050F056BFD2D002F197
:10C5D000640307EE903A9FED047AF8EEE77A67EE8F
:10C5E000877A28EE278AC5E70AD7233C00A08C4526
:10C5F00000A08CC500B52DED048B042083B050F055
:10C600004FFF0320B0EE408A50F05AFFDFED189A3A
:10C610009FED181ADFED180A8DED011AF0EE408A31
:10C62000B0EE480AA8EEA90ACF20CDED000A1CF012
:10C630007BFAB0EE409AB0EE480A9DED011ADDEDAE
:10C64000000AA8EEE90AD0201CF06EFA1820B0EE1D
:10C65000408AB0EE490A50F00FFFB0EE480A1920A8
:10C6600003B0BDEC048B5DF804EB50F005BF00BFD8
:10C670000000344200A08C4500A08CC5F8B52DED1B
:10C68000088B00F5005600F5A04596F9263B13F0FF
:10C69000040F03F0010203F0020440F0F580D5F826
:10C6A000A0777B1E5F425F41002A00F0EF804D20A3
:10C6B00050F0F6FE4E20F0EE409A50F0F1FEB0EE53
:10C6C000408AB6F94633DFED87AA0AEE103A152004
:10C6D000B8EECAAA50F0E4FE2AEE2AAA20EE0AAA70
:10C6E000002C00F0DB80F0EE488AB0EE699AB5EEDF
:10C6F000C0AAF1EE10FA40F3D6809FED7B1ADFED71
:10C700007B0A38EE0A0A4FF480701CF00DFA9FED98
:10C71000761ADFED760AB0EE408A40F2011038EE6C
:10C72000CA0A1CF001FAF0EE408A96F9273B632B07
:10C7300015DC07EE903A9FED6E7AF8EEE77AB4EEEC
:10C74000C79A67EEAA7AF1EE10FAF4EEC78A98BF9C
:10C7500029EE279AF1EE10FA98BF68EEA78AD5F86D
:10C76000A03796F9244B96F9256B022B00F0B48084
:10C7700024B2002C01DC002E6EDD032050F0A0FE60
:10C78000DFED5C7AB4EEE70AF1EE10FAB0EE40AA03
:10C7900062DB002F00F0A2809FED571ADFED570AF1
:10C7A00040F2271030EE000A1CF0BEF99FED541A3B
:10C7B000DFED520AB0EE40BA4FF494703AEE410AFF
:10C7C0001CF0B2F970EE007AB0EE4BAA07EE104AF8
:10C7D000F8EEC7AA9FED4BBA9FED431ADFED430A6F
:10C7E0006AEEA7AAB0EE690A40F22B10AAEE8B0AF5
:10C7F0001CF09AF907EE906AF0EE409AB8EEE70A5C
:10C800009FED391ADFED390A2AEE40AAB0EE490A47
:10C810004FF49670AAEE0B0A1CF086F9B0EE409A1F
:10C82000B0EE480A9FED301ADFED300A40F22D10CD
:10C83000AAEE8B0A1CF078F9B0EE408AB0EE680AD6
:10C84000AAEE0B0A4FF497709FED271ADFED270A27
:10C850001CF06AF9F0EE408AB0EE690A102050F040
:10C860000BFEB0EE490A562050F006FEB0EE480A24
:10C87000112050F001FEB0EE680ABDEC088B572085
:10C88000BDE8F84050F0F8BD01270DE7042050F056
:10C8900007FEB0EE408AF1EE409A12E7DFED178A0C
:10C8A000B0EE689A23E79FED101ADFED100A39EE1B
:10C8B000CA0A4FF482701CF037F99FED0B1ADFEDB6
:10C8C0000B0AF0EE409A40F2051039EE0A0A1CF00D
:10C8D0002BF9B0EE409A28E700244CE7F0EE407ABE
:10C8E00074E700BF0AD7233C00A08C4500A08CC58C
:10C8F000000000B4000000340000C8420000000046
:10C90000000048426666E63E38B52DED028B00F524
:10C9100000550446D5F8680BA0B304F5804393F89E
:10C92000202D7ABB93F8263D63BB4FF05BFB07EEEF
:10C93000900AB8EE678A462095F9A85250F0B0FDEB
:10C94000002DF0EE408A20DA04F5A9404C3072F058
:10C9500041FBE8B99FED101ADFED100A40F25110CB
:10C96000B1EE680A1CF0E0F8B4EE408AF1EE10FA7D
:10C97000C8BFB0EE480ABDEC028B6E20BDE838405F
:10C9800050F07ABD9FED058AD5E79FED040AEBE7ED
:10C990009FED010AE8E700BF0000C8420000000068
:10C9A00010B52DED028B4369002B4AD0037C0BB1EF
:10C9B00001330374037C002B41D0182B1FD803EBE9
:10C9C0004303C3EB03139B001CB2002307EE903A12
:10C9D000B8EEE78A0420B0EE480A50F04DFD07EEAD
:10C9E000904A1320B8EEE70A50F046FDB0EE480A30
:10C9F000BDEC028B1520BDE8104050F03DBD4A2B28
:10CA000002D8C3F13203DAE7632B01D8643BD6E7DF
:10CA10007C2B08D8643B03EB4303C3EB03139B005D
:10CA20001BB20024D2E7AE2B02D8C3F19603F2E783
:10CA3000C72B01D8C83BEEE700230374F1E71C467F
:10CA4000C4E7BDEC028B10BD10B59FED1C7AD0ED94
:10CA5000017AF4EEC77A0023F1EE10FA044643722D
:10CA60002BDB90ED007AB4EEE77AF1EE10FA24D9E0
:10CA700008F0E8F8217A07F039FDD4ED010AF5EE67
:10CA8000007A60EEA77AB4EEE70AF1EE10FA14D459
:10CA900094ED001A40F2A5101CF046F8F7EE007A6B
:10CAA000B4EEE70AF1EE10FA07D494ED007AC7EE7F
:10CAB000007A01236372C4ED037A10BD00000034D4
:10CAC000437A7BB391F9003090ED037A07EE903A08
:10CAD000F8EEE77A67EE877A9FED137AF4EEC77A7D
:10CAE000F1EE10FAD8BFF0EE477AFDEEE77A17EED6
:10CAF000903A0B7092F9003090ED037A07EE903A7D
:10CB0000F8EEE77A67EE877A9FED087AF4EEC77A57
:10CB1000F1EE10FA58BFF0EE477AFDEEE77A17EE25
:10CB2000903A1370704700BF0000C8C20000C842AE
:10CB3000437AF0EE407A5BB190ED030A9FED051A5F
:10CB4000DFED050A27EE800A4FF4E6701BF0ECBF1C
:10CB5000704700BF0000C8420000C8C2F8B50446D4
:10CB60000E46174674F0A0F9054604F59A40583071
:10CB700007F046FE04F5A044D8B3462050F090FCE0
:10CB8000DFED3D7AB4EEE70AF1EE10FA10DB97F92B
:10CB9000002094F98933193A934209DAD4F88C23A6
:10CBA000AA4205D0C4F88C53013384F8893344E099
:10CBB000462050F075FCDFED317AB4EEE70AF1EE75
:10CBC00010FA3AD896F90020002A36DAC2F1FF228C
:10CBD00094F98A3302F57F02E73293422DDAD4F8D2
:10CBE0008C23AA4229D0C4F88C53013384F88A33A9
:10CBF00023E0D4F88C33EB1AB3F57A7F1DD34620AB
:10CC000050F04EFC94F9893307EE903AF8EEE77A4B
:10CC1000B4EEE70AF1EE10FA01DD002B22DC46202B
:10CC200050F03EFC94F98A3307EE903AF8EEE77A3A
:10CC3000B4EEE70AF1EE10FA18D497F9000094F96F
:10CC400089230021821A1CF01FF8387096F9000021
:10CC5000002806DA94F98A13002201441CF014F823
:10CC60003070F8BDC4F88C53013B9EE7002BE4DD27
:10CC7000C4F88C53013BB9E700000034000000B455
:10CC800010B52DED028B00F5005282B092F9A8325A
:10CC900092F8A9228DF80630002B0446B0EE408AA7
:10CCA0008DF8072004DAFFF7D1F908B98DF80600EE
:10CCB00004F5A043D3F89023012A4CD0072A4AD088
:10CCC00004F5A9404C3072F085F9002854D104F5E0
:10CCD0002C500DF106010DF107022830FFF7F0FE90
:10CCE0002046FFF73BFF9DF906309DF90720DFED59
:10CCF000238A9342A8BF134607EE903A04F53054B6
:10CD0000B8EEE70A083420EE280A20468DF80630EF
:10CD100071F058FB9DF9073000EE103AB8EEC00AEA
:10CD2000204620EE280A71F057FB9DF9073001EEEE
:10CD3000103A9DF9063000EE903AB8EEC11AF8EEBE
:10CD4000E00A40F24D20B0EE480A1BF0EDFE02B0C2
:10CD5000BDEC028B10BDD3EDBB7AFDEEE77A17EE8A
:10CD6000902AD3EDBC7A8DF80720FDEEE77A17EE16
:10CD7000903A8DF80630AAE70023FAE70AD7233C59
:10CD800070B5044600F52C55283504F58046284634
:10CD9000FFF75AFED6F80C0D03685B6D984740B15B
:10CDA000462050F07DFB2846FFF7C2FE462050F09B
:10CDB00063FBD6F80C0D03681B6D984740B1462005
:10CDC00050F06EFB2046FFF75BFF462050F054FB0F
:10CDD0002046FFF7E1FA10B304F5005595F9143336
:10CDE00043B101212046FFF7F7F9BDE87040462026
:10CDF00050F042BB04F5A9444C34204672F0EAF8E6
:10CE000050B1204672F06EFA30B195F9A83200EEBA
:10CE1000103AB8EEC00AE8E79FED010AE5E770BDF9
:10CE20000000000010B504462DED028B462050F0A6
:10CE300037FB2046B0EE408AFBF72EFE80BB04F5A0
:10CE4000AD4074306CF09CFB50B304F5A853D3EDA7
:10CE5000028A1BF02DF990F813339FED137A0C2200
:10CE600002FB0300D0ED627AE8EEC77AF4EEC77AEF
:10CE7000F1EE10FA0CDC04F5005494F9AB3207EE35
:10CE8000903AF8EEE77AF4EEC87AF1EE10FA07D5A8
:10CE9000BDEC028B0548BDE81040012104F0D0BC78
:10CEA000BDEC028B10BD00BF0AE81C41E83E00202B
:10CEB0002DE9F04100F500550646D5F8643BA3BBCB
:10CEC000002706F58048D8F80C0D03689B6B98473F
:10CED0000446002852D006F59550103003F02AF889
:10CEE00080B308F63853D3ED007A9FED3F7AF8EE21
:10CEF000E77A67EE877AFDEEE77A17EE903A1BB293
:10CF000095F95B230AB19A421FDA95F95943FCB9A6
:10CF100006F5A042D2F89033013B062B2ED8DFE86D
:10CF200003F01E2D24602D2D1E004EF0AFFE036871
:10CF3000DB6898470028C3D0D5F8640B4FF052F84F
:10CF400047B2BEE795F9AB32DAE795F95A43DFE726
:10CF500024B29C42ACBF95F958430024D8E795F918
:10CF60005C33002B18BF1C4608E095F95C332BB1ED
:10CF70003046FBF7AFFD08B195F95C4387EAE773EC
:10CF8000A3EBE773DBB2A342C8BF3C4607EE904A6F
:10CF90000320B8EEE70A50F06FFA07EE907A02200D
:10CFA000B8EEE70A50F068FA95F98533D6ED460AEF
:10CFB00000EE103A6421B8EEC00A032050F052FB94
:10CFC00095F98533D6ED460A00EE103A0220B8EE08
:10CFD000C00A642150F046FB3046BDE8F041FFF73F
:10CFE00009BB92F94735BCE70AD7233C70B5044624
:10CFF0002DED048B462050F053FA5B4BDFED5B7A4E
:10D0000093F9F13A08EE903AF8EEE88A152068EEC6
:10D01000A78AB0EE408A50F043FA9FED557A20EE91
:10D02000280A04F5A045C0EE077A05F5F26604F576
:10D03000AA405830C6ED007A6FF028F808B10023F6
:10D040003360B5EEC08AF1EE10FA46D52046FFF700
:10D05000BDF8002800F083802046FEF7F7FF002887
:10D060007DD005F5F265D5ED007A9FED429A9FEDF2
:10D07000421ADFED420AB0EE480AA7EE890A4FF4E1
:10D080003B701BF051FDD5ED007A9FED3B1ADFEDB3
:10D090003B0AF0EE408A40F2ED20B0EE480AA7EEDF
:10D0A000C90A1BF041FDB0EE408A04F5AD45743568
:10D0B00028466CF06FFAE0BB28466DF03FFB022873
:10D0C00029D10321492050F031FDBDEC048B03210F
:10D0D000BDE870404A2050F029BD40D905F5F26501
:10D0E000D5ED007A9FED239A9FED251ADFED220AF8
:10D0F000B0EE480AA7EE890A40F2F2201BF014FDB8
:10D10000D5ED007A9FED1E1ADFED1B0AF0EE408A86
:10D1100040F2F320C1E79FED180A492050F0ACF926
:10D12000BDEC048B9FED140ABDE870404A2050F01E
:10D13000A3B9B0EE680A492050F09EF9B0EE480A53
:10D140004A2050F099F920464921FFF7DDF8BDEC5F
:10D15000048B20464A21BDE87040FFF7D5B89FED0B
:10D16000068AF0EE488AA0E7384C00200AD7233C14
:10D1700000A08C4500004842000000000000C8C22A
:10D180000000C842F8B52DED028B00F5A04604461C
:10D1900096F94535002B32DD00F5804200F59943C4
:10D1A000D2F80C2D20339A4229D196F94435002B20
:10D1B00025DD00F5A9404C3071F07EFFF8B104F593
:10D1C000AD4074306CF0DCF9C8B9124F9FED128A93
:10D1D00004463D682D190ED0B5F908004FF072FFD6
:10D1E00048B196F94535012B0CD1B5F90800B0EEE0
:10D1F000480A50F041F91434B4F5A07FE9D1BDECF0
:10D20000028BF8BD022BF6D1B5F90800032150F0CE
:10D210008DFCF0E7308900200000000037B500F5F4
:10D22000A043044693F8E8320BB39FED120A152091
:10D230004F2550F021F92046009550231322152147
:10D24000FFF774F9152050F0B9FB80B9284650F06B
:10D25000B5FB60B99FED070A4E2050F00DF99FED28
:10D26000050A4D2003B0BDE8304050F005B903B0C9
:10D2700030BD00BF0000000070470000F8B52DED84
:10D28000048B00F580450446D5F80C0D03689B6BB4
:10D29000984738B9D5F80C2D04F5984374339A4261
:10D2A00040F0BE8004F5AD4074306CF073F9002896
:10D2B00000F0B6802046FBF7EFFB002800F0B080BE
:10D2C00004F5A045D5F8A433002BB8BF5B42B3F5F5
:10D2D0002F7F00F3A580D5F8A833002BB8BF5B42A1
:10D2E000B3F52F7F00F39C8073F0DEFDD5F8603638
:10D2F000C31AB3F5FA7F0646C0F0928004F5B55321
:10D3000093ED057AF2EE007AB4EEE77AF1EE10FAD8
:10D3100000F1868095EDEC7AB4EEE77AF1EE10FA42
:10D320007ED404F5005707F6B47393ED048A04F530
:10D33000405304F51B54D3ED488A1C34B0EE480A20
:10D340000421204650F00EF9B0EE680A1321204661
:10D3500050F008F978EEC89A4D21B0EE690A2046DF
:10D3600050F000F938EE289A4E21B0EE490A2046D6
:10D3700050F0F8F8B0EE680A4F21204650F0F2F86D
:10D38000B0EE680A5021204650F0ECF8B0EE480AA2
:10D390001821204650F0E6F8B0EE480A1921204640
:10D3A00050F0E0F897F9263B03F00202DB075CBF80
:10D3B000F1EE489AB0EE489A6AB3B0EE498AF0EEC0
:10D3C000698AB0EE690A1021204650F0CBF8B0EE21
:10D3D000680A5621204650F0C5F8B0EE490A1121DE
:10D3E000204650F0BFF8B0EE480A5721204650F0D2
:10D3F000B9F8D5F86436C5F86066F31A42F21072CF
:10D4000093420DD9C5F86466BDEC048B2046BDE897
:10D41000F84050F08DBC9FED048AF0EE488AD0E7CA
:10D42000BDEC048BF8BD00BF0000000073B50446DE
:10D4300050F094FD054650F027FD2046FFF7D6FD3D
:10D440004E23009313224D2304212046FFF76EF84C
:10D450004F2315211322009320465023FFF766F82F
:10D460002046FFF70BF92046FFF78CFE4FF40051E2
:10D470002046F5F76BF810B12046FFF7CFFE04F514
:10D480000056D6F8F40A50B104F5804204F59943E9
:10D49000D2F80C2D5C339A4201D14FF0C7FF50F007
:10D4A00089FC4FF0DDFE284650F0F6FC96F9C83AAC
:10D4B0002BB1204602B0BDE87040FFF7DFBE02B0DE
:10D4C00070BD000073B5044604F5AA4550F046FD52
:10D4D000583550F0D9FC28466EF0D8FD04F5A0462A
:10D4E000002866D1D6F89033042B04D104F5A94066
:10D4F0004C3071F09BFD2046FFF742FC04F5804262
:10D5000004F59943D2F80C2D5C3304F5AD459A42ED
:10D5100005F1740523D028466CF03CF8F8B99FED6E
:10D52000310A46204FF0A8FF9FED2E0A49204FF008
:10D53000A3FF9FED2C0A4A204FF09EFF28466DF076
:10D54000FDF802280BD10321462050F0EFFA032109
:10D55000492050F0EBFA03214A2050F0E7FA204628
:10D56000FFF760FC2046FFF7A3FC2046FFF7CCF94D
:10D5700020464621FEF7C8FE28466CF001F890B917
:10D58000019028466DF0DAF868B102281AD10199A5
:10D59000462050F037FA0199492050F033FA0199AA
:10D5A0004A2050F02FFA204602B0BDE87040FFF745
:10D5B0003DBF2846F8F7BCFB96F962352B2B91D07E
:10D5C00002B070BD9FED070A46204FF055FF9FED5A
:10D5D000050A49204FF050FF9FED020A4A204FF004
:10D5E0004BFFE0E700000000F7F7C6B90148FBF782
:10D5F00003B800BF382C002008B5044A0F2342F0BE
:10D6000071F880F00100C0B208BD00BFB4E90B089A
:10D61000F8B500F540570446D7F8D05473F044FCF1
:10D6200004F5804304F50056B3F9241D8A1E92B216
:10D63000012A73D904F5A042D2F89023042A6DD0B0
:10D64000012993F8201DD3F82C2D08BFD3F8282DDD
:10D65000B1B1821A07EE902A96EDCA7ADFED416ADF
:10D66000F8EE677A27EE267AF4EEC77AF1EE10FA32
:10D6700006DD032202212046BDE8F840FAF774BE19
:10D6800096F92C23032A1BD1D3F80C3D04F59942BB
:10D690002032934265D1002D63D0401B07EE900AE3
:10D6A000DFED306AB8EE677AD6EDCA7A67EEA67A11
:10D6B000B4EEE77AF1EE10FA53DD05220321DAE742
:10D6C000012A4CD0022A4CD18DB1431B07EE103AEF
:10D6D000D6EDCA7ADFED236AB8EE477A67EEA67A0E
:10D6E000B4EEE77AF1EE10FAE7DC022A39D197F8C6
:10D6F000B433B3B3D7F8B8339BB31B4B1B6883B3B6
:10D70000C01A07EE900A96EDCA7ADFED166AF8EEB7
:10D71000677A27EE267AF4EEC77ACBE796F92023CC
:10D72000D6EDCA7A032A18BFD6EDC97A03290FD1DC
:10D73000FCEEE77A4FF47A7317EE902A401B5A43B7
:10D7400090420ED205212046BDE8F840FAF7C6BE49
:10D75000022906D193F8203D1BB90321F3E7002DE0
:10D76000B3D1F8BD00007A44A488002070B500F55C
:10D770000056044696F92033032B00F580450FD060
:10D78000B5F9243D63B900F5A043D3F89033042BD9
:10D7900017D095F8203DA3B103220121FAF764FDCB
:10D7A000B5F9243D012B0CD195F8203D1BB196F91C
:10D7B0002033032B05D120460321BDE87040FAF742
:10D7C0005FBE70BD70B500F6C806044630461AF05C
:10D7D00039FC04F54C53183360B3174A04F59555DA
:10D7E00018460121103545F093FE284602F048FA0C
:10D7F00004F58053032283F8C42440F20112A3F8F5
:10D80000B825B4F9A4301BB9B4F8A230A4F8A430F8
:10D81000B4F8A41030461AF0BDFC284602F030FBE4
:10D820008023C4F8743404F58C600121BDE8704095
:10D8300006F0DCB9014AD1E7BCE80B08E9E80B08BF
:10D8400038B50B6805465B6808460C469847064B9A
:10D85000D87023682046DB689847014605F5935049
:10D86000BDE8384038F040BB958400202DE9F74FE3
:10D8700000F580470446D7F80C3D8B420D4616460E
:10D880000CD100F5005494F86832934240F0B58012
:10D890004FF00109484603B0BDE8F08F0B68084619
:10D8A0005B69984704F54C5808F118088146B0B1F7
:10D8B00042F0CAF840F203124FF4801142F07CF8B3
:10D8C000524A0621404645F023FE1A2E1FBF504AF9
:10D8D000137843F0040313704FF00009DAE74D4B5F
:10D8E0001B68DB6A93F89C305BB304F5005393F834
:10D8F000502132B3B3F86C21D20722D593F88C3182
:10D90000FBB12046FAF728FFD8B1A6F12703DBB216
:10D910000A2B06D8012202FA03F340F223421342F3
:10D920000FD12B6828469B6898473B4A0346052140
:10D93000404645F0EDFD364A137843F0040313707A
:10D94000A8E7022E2BD0D7F80CBDD7F8103DC7F8AA
:10D950000C5D04F50059C7F810BD04F5A04A99F80C
:10D960006822009328469AF8A8378AF8A82789F8E9
:10D9700068620193FBF76CFC38BB284A04214046DF
:10D9800045F0C6FD009BC7F8103DC7F80CBD9AF8DE
:10D99000A83789F86832019B8AF8A83795E72B6881
:10D9A00028465B68984701462046FFF725FE8146DA
:10D9B0000028C8D12B6828469B689847184A034618
:10D9C0000521404645F0A4FD64E75846FBF72CFCD2
:10D9D000D7F80C0D03685B68984799F868220146F0
:10D9E00004F57F6042F0FEFFD7F80C1D2046FFF7DC
:10D9F00027FF002140464DF073FA1A2E1FBF044A3C
:10DA0000137843F00203137042E700BF04E90B08E8
:10DA1000B4840020342C00201CE90B0888E90B0892
:10DA200048E90B0873B505460A4801920E46FAF715
:10DA300001FA019A044630B10146284602B0BDE819
:10DA40007040FFF713BF2846314641F093FD204652
:10DA500002B070BD382C0020FFF7E4BF4FF4002364
:10DA6000F7B50446C0F8E03B00F53A500C306DF0D5
:10DA70007DFD04F53F5024306DF0F4FA4EF006F9C8
:10DA8000992229214FF0ECF94EF000F94EF0A6F85A
:10DA900004F591500C3057F059F904F5935038F0D3
:10DAA00007FA04F580432046D3F80C1DFFF7C8FEA3
:10DAB0002046FDF7C9FF04F58C6006F0DFFA4FF44D
:10DAC00080431921C4F8EC3F04F554603DF00AFE90
:10DAD00004F59A40583006F059FC04F5865004309D
:10DAE00051F05EFB04F54C5504F52E5018352030EE
:10DAF00050F0D8FF284649F053FF04F5585018302D
:10DB00005EF078FC0AF090FD4FF4806303630AF046
:10DB10008BFD0BF001FE04F50A5104F5FC50283191
:10DB2000183001F0BBF804F500538022C3F8E82058
:10DB30000423C4F8A43104F5907011F015FE2046BA
:10DB4000FDF768FF04F5AC40703052F01BF904F5A6
:10DB50005550043007F038FF04F52C5004305DF0C8
:10DB600039FF334B33491E68B06A03684FF47A7249
:10DB7000DB6A984701203BF0AFFE04F599411A2279
:10DB800054312046FFF772FE2B4A0621284645F005
:10DB9000BFFC2046FFF716FE04F5A74034301FF007
:10DBA0000DFB04F5A0434FF48072C3F8A824234B67
:10DBB0000093234B019302AB13E9060004F57F6049
:10DBC00042F02CFD73F070F904F5405504F5005750
:10DBD000C5F8D0042046FDF763FFD7F8441B29B1F0
:10DBE000706A03680222D3F880309847706A154B38
:10DBF0001A68036892F8F113D3F8AC30984797F895
:10DC000034131A222046FFF70DFF4EF03FF84DF077
:10DC1000C7FF95F9C9354BB104F557504FF0FF31A7
:10DC2000043003B0BDE8F04039F040BB03B0F0BDB4
:10DC3000342C0020EDD50108A4E90B08382C002075
:10DC4000E9D50108D888002000F57F6043F082BB49
:10DC500010B52DED028B044682B046204FF020FC1B
:10DC60002046B0EE408AFEF7B1FAFDEEC87A0146D2
:10DC7000CDED017A642240B9BDF904001BF004F82F
:10DC800040B202B0BDEC028B10BD6FF06301F3E750
:10DC90002DE9F04F054605F5005985B073F004F9FC
:10DCA00099F9688364231FFA88F803FB08F806468D
:10DCB00043F29C1305F5AD40984500F17400A8BFF0
:10DCC00098466BF067FC05F5A0440746A0B90146ED
:10DCD00005F5A54030224C3095F0DCFF95F8712415
:10DCE00005F58C63242101FB0233DB6AC4F834336D
:10DCF000384605B0BDE8F08FD4F8D0325BB1F31AE6
:10DD0000C82B08D905F5A540302200214C3095F0EC
:10DD1000C1FF0027ECE78F4BC4F8D062D3F820375F
:10DD2000C3B994F838A7BAF1000F13D1012384F8CE
:10DD3000E832D4F8D43240F6B832F31A9342E8D934
:10DD400005F54C50844A0421183045F0E1FBC4F835
:10DD5000D462DEE7002384F8E83295F8582495F879
:10DD6000143432B1B02202FB035292F8F121012A9D
:10DD7000CFD8B02202FB035393F8F131022BC8D95C
:10DD800004212846F4F7E2FB94F8DC1282460029CD
:10DD900060D1D9EDD97A9FED717AF0EEE76AF4EEB1
:10DDA000C76AF1EE10FA29D499F9002B09F6084355
:10DDB000012A93ED377A0ADCF4EEC77AF1EE10FA15
:10DDC0001CDD002784F8DC72C4F8CC7290E7D4F82C
:10DDD000E032F31AB3F5FA7F88BF84F8DD1294F8C5
:10DDE000DD32D9074DD5F1EE677AF4EEC77AF1EE60
:10DDF00010FA4BDC94F8DD329342E2DB012384F825
:10DE0000DC32D4F8D832C4F8CC62F31AB3F5FA6F26
:10DE100020D907EE908A9FED527AF8EEE77A05F561
:10DE20004C5B67EE877A0BF1180B17EE900AF2F74E
:10DE300063FBCDE9020109F60843D3F8DC00F2F7F1
:10DE40005BFB484ACDE900010621584645F060FBDE
:10DE5000C4F8D862D4F8CC3208F16402F31A9342C1
:10DE60001AD9D4F8D832F31AB3F5FA6FA9D905F54F
:10DE70004C503D4A0421183045F04AFBC4F8D862A2
:10DE80009FE7F4EEC77AF1EE10FAB3D5013384F8C8
:10DE9000DD32C4F8E062ADE7BAF1000F21D105F53B
:10DEA000805A41F64A52DAF8AC3403F6B73393425B
:10DEB0000AD905F54C502D4A0421183045F028FBAD
:10DEC000002384F8DD327CE72846FAF79FF840B952
:10DED000DAF8A834002BB8BF5B4240F6B832934260
:10DEE000E7DC95F81434D9EDD87AB02202FB03535D
:10DEF00093ED837AF4EEC77AF1EE10FA09D4DFEDF0
:10DF0000176AF0EEE77AF4EEE67AF1EE10FA7FF5B2
:10DF100000AFD4F8CC32F31A98453FF6FAAE17EEBC
:10DF2000100AF2F7E9FA05F54C551835CDE900016C
:10DF30000F4A0621284645F0EBFA0023C4E9BD63E9
:10DF400084F8DC32C4F8CC320023C4F8E462C4F8AC
:10DF50000433CDE6387C0020C4E90B08000000340F
:10DF60006F12833AE7E90B0819EA0B0826EA0B0857
:10DF700036EA0B0870B500F5A0450446D5F8FC322A
:10DF8000013303D10023C5F8A43370BDF5F746FA79
:10DF900004F5005095EDC57AD0EDDC7A90F97C233C
:10DFA000B4EEE77AF1EE10FA0AD5642312FB03F21D
:10DFB000D5F8A40351421AF057FEC5F8A403E4E7CC
:10DFC00004F58046D5EDCD1AB6F9EE3CB6F9EC6C09
:10DFD00003EB4301B142A8BF314607EE901A23EA92
:10DFE000E37394F87114B8EEE72A07EE903A04F55B
:10DFF0008C63242404FB013300F66C31D1ED000A5C
:10E0000093ED0B1A642112FB01F2F8EEE77A00EEB1
:10E01000102A32EE212AF8EEE00A77EEA11AB8EEC5
:10E02000C00A1AF0B3FCFDEEC07A17EE902ABFE7E3
:10E0300070B52DED028B00F50056054696F9AC3211
:10E04000002B3DD007EE903AF8EEE77A05F5A044B4
:10E05000C4EDBB7A96F9AD32ABB307EE903AD4F883
:10E06000F432F8EEE77AC4EDBC7AD3B172F01CFF5B
:10E07000D4F8F4329FED267AC31A07EE903AF8EE00
:10E08000677A67EE877A96EDB87AF4EEC77AF1EEA2
:10E0900010FA47BFD4F8EC32C4F8F0320023C4F8C9
:10E0A000F432D6F8B032DB0710D4D4F8EC32C4F82E
:10E0B000F032BDEC028B2846BDE87040F4F7AABEF2
:10E0C00096F9A932BEE796F9AB32C6E795F8712406
:10E0D000D4EDCD8A05F58C63242101FB023393ED49
:10E0E0000B8A05F5955005F580431030B3F9EE6CB9
:10E0F00001F020FF0028D8D007EE906AF8EEE77A0A
:10E1000077EEA87AF4EEC87AF1EE10FACDDCD0E71B
:10E110006F12833A70B500F5A0440646D4F89033E8
:10E12000012B02D0B4F93A0327E0F8F7A5F806F579
:10E130000053D3EDDE6AF5EEC06AF1EE10FAF1DDC0
:10E14000D4F80C53D4F810332D1ABBB107EE103AA3
:10E1500007EE905AF8EEC76AF8EEE77AB4F93A3368
:10E1600087EEA67A07EE903AF8EEE77A67EE277A1E
:10E17000FDEEE77A17EE903A18B270BD94EDC76ADB
:10E18000DFED177AB4EEE76AF1EE10FACAD507EEC2
:10E19000105ADFED147AB8EEC77A67EEC77A87EEC9
:10E1A000867AB5EEC07AF1EE10FABBDDB0F57A7F73
:10E1B000B8DBF4EEC76AF1EE10FAB3DB06F54C50AB
:10E1C000094A06211830642395FBF3F345F0A0F9C2
:10E1D000C4F8105372F068FEC4F8F802A2E700BF5A
:10E1E000CDCCCCBD0AD7233C58EA0B082DE9F84327
:10E1F0002DED028B00F5A04500F5305795F8503312
:10E200009FED5E8A0446083700F50058002B57D171
:10E21000D8EDDC7AF5EEC07AF1EE10FA50DD95ED2E
:10E22000C57AF4EEC77AF1EE10FA20DD00F59944D4
:10E2300094ED1C0ADFED527A20EE270A7034BDEE11
:10E24000C00A85EDEA0AB8EEC00A20EE080A384690
:10E2500070F01CF995EDEA0AB8EEC00A384620EED7
:10E26000080ABDEC028BBDE8F84370F019B990F8CC
:10E27000143498EDAE7AB02202FB0303D3ED836A27
:10E28000B4EEE67AF1EE10FA1ADBC6EE877AB5F94B
:10E290003A234FF4FA7107EE102AB8EEC77A67EE08
:10E2A000877AFDEEE77A17EE900AC5EDEA7A1AF062
:10E2B000DBFC07EE900AC5F8A803B8EEE70AC4E74E
:10E2C0004FF0010985F850932046FFF723FF0646DB
:10E2D00004F59550103001F02DFE58B12046F4F7AA
:10E2E000A9FFD5F8A833B34201DAC5F8A8634FF007
:10E2F000000901E0C5F8A86398F9DC326BB304F5B6
:10E300008054D5F8A433D4F8A8249FED1E1ADFED6D
:10E310001E0A9B1A002BB8BF5B4207EE903AB8EE7C
:10E32000E70AEA2020EE080A1AF0FEFBDFED177A72
:10E3300020EE270A93F066F8D5EDEA7A20EE000A7F
:10E34000F8EEE77A67EE807AFDEEE77A17EE903A1C
:10E35000B342C5EDEA7AB8BF1EB207EE906AB8EED6
:10E36000E70A384620EE080A70F090F8B9F1000F7D
:10E370007FF470AFBDEC028BBDE8F8830AD7233C75
:10E380000000C8420000B4420000000035FA8E3C94
:10E3900010B51F4BD3F89033012B0DD000F5804200
:10E3A00000F59843D2F80C2D74339A422DD100F524
:10E3B000A04393F8413333B300F5005200F5A04475
:10E3C00092F9693393B194EDC57AD2EDDB7AB4EE6C
:10E3D000E77AF1EE10FA09DA00F58051B4F9382342
:10E3E000D1F8AC1402F57A7291420CDD94F8413305
:10E3F0004BB100F54C50074A0521183045F088F81C
:10E40000002384F84133184610BD0023FBE700BF0A
:10E41000387C00207CEA0B0810B502210446F7F78F
:10E4200041FD04F52C500430BDE810405DF038BBD0
